:020000040800F2
:10800000203B0020ED500108794B01087D4B010811
:10801000994B01089B4B01089D4B01080000000093
:108020000000000000000000000000009F4B01085D
:10803000A14B010800000000A34B0108A54B01085B
:10804000B9510108BD510108C1510108C5510108CC
:10805000C9510108CD510108D1510108D55101087C
:10806000D9510108DD510108E1510108E55101082C
:10807000E9510108ED510108F1510108F5510108DC
:10808000F9510108FD51010801520108055201088A
:10809000114C0108095201080D520108A94B0108B1
:1080A0001152010815520108195201081D52010808
:1080B000C54B010821520108E94B0108255201086E
:1080C000295201082D520108315201083552010888
:1080D000395201083D520108415201084552010838
:1080E000495201084D5201085152010862F30F2212
:1080F00062F31F4200B500BF130096469446103944
:1081000028BFA0E80C50FAD85FEA417C28BF0CC019
:1081100048BF40F8042BC90728BF20F8022B48BFEE
:1081200000F8012B00BD30B4002513E050F8042BFB
:10813000D30744BFA9F101039A18091F042942F883
:10814000045BFAD213468C0744BF15809B1CC907F9
:1081500048BF1D7050F8041B0029E7D130BC7047A0
:1081600010B504462034A1F15002D2B200213C20C7
:1081700001F086F82246D2B2120942F01002002124
:108180003C2001F07DF804F00F04224600213C2041
:10819000BDE8104001F074B82DE9F04105460C46E9
:1081A00016461B19DBB22046E408891000EB51711A
:1081B000C910B0EBC10000D0641C1846801003EB5E
:1081C00050784FEAE808069FB3EBC80302D15FFA84
:1081D00088F812E008F101085FFA88F80DE02146FE
:1081E000C9B22846FFF7BCFF40233C22314638463F
:1081F00001F060F830460744641C2046C0B2404598
:10820000EDDB3846BDE8F08110B5040014D4DFF88A
:10821000FC02B0F90010224691420DD00480812268
:1082200000213C2001F02CF82246D2B200213C2053
:10823000BDE8104001F024B810BD3EB5069C0325F2
:108240000195009409B200B202F0B2F837BD10B542
:10825000A2B00022802102A8FFF748FF00240BE013
:108260000020019002A8009008238022E100C9B2FA
:108270000020FFF791FF641C2046C0B20228EFDB0C
:1082800022B010BD000000002DE9F841B3B0002479
:108290002246802103A8FFF729FF22460DF108019D
:1082A000A0A004F0AFFF050000F0A88028784228C5
:1082B00040F0A48068784D2840F0A08005F1360099
:1082C0000178FF2906D14178FF2903D18078FF2862
:1082D00000D1012400227F2103A8FFF707FF01231B
:1082E0000F2203E05B00DBB2521ED2B2082A2DDB64
:1082F0000026374601E00C467F1C3846C0B20C28E9
:10830000F0DA02EB420100EB8100284490F83EC015
:108310004FF0800E4FF0000821464046C0B20828BA
:10832000E9DA704600EA0C00002902D1002806D0E4
:1083300001E0002803D103A8845D1C438455761C0A
:10834000F6B24FEA5E0E08F10108E6E7642007F096
:10835000A6FBFFF77CFF0020019003A800900823F4
:10836000602200210846FFF717FF00227F2103A8A3
:10837000FFF7BCFE0123002202E05B00DBB2521CCF
:10838000082A2DDA0026374601E00C467F1C3846C5
:10839000C0B20C28F1DAA2EB820100EB8100284484
:1083A00090F892C04FF0800E4FF0000821464046F2
:1083B000C0B20828E9DA704600EA0C00002902D1B0
:1083C000002806D001E0002803D103A8845D1C43E7
:1083D0008455761CF6B24FEA5E0E08F10108E6E716
:1083E0000020019003A80090082360221946002075
:1083F000FFF7D2FE4FF4967007F051FB34B0BDE8A2
:10840000F0810000FEB504460D4616461F4614E0F6
:10841000303802E02D28FBD10C20394601913C492F
:10842000C0B201EB4010009010231A4629462046A6
:1084300000B201F0BDFF0E34761C3078002803D066
:108440002028E7D10A20E8E7F7BDFEB504460D462F
:1084500016461F4613E016F8010B203839460191E5
:108460002C49C0B200EB400201EB4200009008230F
:1084700006222946204600B201F09AFFA41D30785A
:108480000028E8D1F7BDFEB504460D4616461F4646
:1084900011E016F8010B2038394601911E49C0B28F
:1084A00001EB00100090102308222946204600B25C
:1084B00001F07EFF083430780028EAD1F7BD7CB5A2
:1084C000069D079C0026002D0DD0022D16D11646C4
:1084D0001D466E437443114D2646B61004EB567488
:1084E00015EBE4060AE016461D466E4374430C4D38
:1084F0002646B61004EB567415EBE4069DF82040B2
:108500000194009601F054FF73BD00000033002079
:10851000F4980008B0440108A0360108FC4D010899
:10852000CC5001084C4F474F494E2020424D50003F
:1085300000280AD0B0FA80F18840D1F19D01C90528
:10854000020672F1004241EB1020704710B5FF2384
:1085500013EAD0541DBF13EAD1529C429A4239E02B
:10856000A41ADA0780EA0103134042EA012142EA31
:108570000020421A3CBF641E01EB4202090AB2FB12
:10858000F1FE01FB1E221202B2FBF1F001FB1022F0
:108590006EF30F201202B2FBF1FE4EEA00207F3490
:1085A00006DDFE2C24DA53EA500050EBC45010BD17
:1085B000D4F1020401FB1E2240F08071192C1DDC55
:1085C00021FA04F0C4F12004A140114371F10042EA
:1085D000584110BD9C421ABF03EAD1529A420FE0A3
:1085E00080EA010E0EF00043400004D0490016D18D
:1085F00043F0FF4010BD490008BFD343180010BD31
:108600009C4205D1D21AF7D001F00041484010BD7C
:108610004A0212BF0846484000F0004010BD4AB967
:108620000902B1FA81F2914044B1A418C00140F0AE
:1086300000409EE7C90141F0004152420002B0FAF9
:1086400080F4A040141B94E7C0F3C75181B1FF2907
:1086500006D0C110400721F0E04101F160517047A0
:1086600041020CBF40F4E0016FF000410020704770
:1086700000F0004100020AD0B0FA80FC00FA0CF0D1
:1086800001F16051A1EB0C5101EBD0214005704785
:108690000CB430B583B00A4606A902910446002501
:1086A0000194009502AB01A9084878441E3007F0F8
:1086B000B3FD019A157000284EBF04460198041BB3
:1086C000204603B030BC5DF80CFB00BF6F03000018
:1086D0007CB505F0BAFE04460021684603F070FB45
:1086E000BDF800500B21684603F06AFB009E284647
:1086F000FFF71EFF6649FFF729FF0546654831462B
:1087000000F0EAFA06462846294600F0E5FA054652
:10871000204600F0CFFA6049FFF718FF01462846CF
:10872000FFF714FF01463046FFF710FFFFF78CFFFD
:108730004FF06632594B00F0DFFD00F083F901463F
:1087400089B2612900DB612080B276BD3EB5044666
:108750000C21684603F034FB9DF80050002C03D038
:10876000FFF7B6FF4E490880012D02D14C48008822
:108770003EBD05203EBD80B5012007F056FAFFF74B
:10878000D7FEFFF761FF4FF06632464B00F0B4FDB5
:108790000022454B00F0B0FD0022444B00F0ACFD40
:1087A0000022434B00F0A8FD00F04CF980B202BD5E
:1087B0003EB542F2107188423DDA0F21684603F05F
:1087C000FFFA9DF80000012825D13A4D28780328AA
:1087D00011DB002028700246374B0D2003F088FC87
:1087E000022003F00AFE002213460C2003B0BDE86D
:1087F000304003F07DBC06F0BFFE044680B206F0B8
:10880000D0FE014689B2204680B206F0EAFE287802
:10881000401C287037BD0022274B0D2003F068FC58
:10882000022003F0EAFD002213460C2003B0BDE84D
:10883000304003F05DBC37BD2048406870477CB5D0
:108840000B21684603F0BCFA009D1C4E7488002C76
:1088500010D03088FFF76CFE0146284600F03CFA45
:1088600005462046FFF764FE01462846FFF76EFEE8
:10887000706001E00020706000203080708073BD67
:108880000E490A88801808804888963048807047CA
:1088900000007A440000C842000020416666EE3FB6
:1088A0000233002066660A4000805B4000005940A9
:1088B0000000303F153300200000F03FAC320020B4
:1088C00070B44FF0004591EA030F40F1EF856B4023
:1088D000841A71EB030604D26E40001BB1411219D9
:1088E00073414FF4001C1CEB410F34BF7CEB43067B
:1088F00083E00C0DA4EB1356362E00F37C80012E82
:1089000045EAC32341DC43EA525312BFD20292022A
:108910005B08240545EAC12141EA5051D2EBC02051
:10892000994125D407D1B0FA80F610FA06F162D049
:108930000020203608E0B1FA81F6B140C6F12002ED
:1089400020FA02F21143B0404FEAF474B4EB4654FB
:1089500034F001064FEA74040AD8D6F50016760DF5
:1089600004F00044F04061FA06F25040F140484003
:10897000C00A40EA415021F0004128BF5FEA50059B
:1089800050F1000044EBD12135E0DB0A45EAC1217A
:10899000C90AB6F120050EDD42EA0242120CC5F109
:1089A000200603FA06F6EB4042EA06056D429841BE
:1089B00061F100010DE062FA06F5F240554063FAFC
:1089C00006FC82EA0C02F3405A406D42904161EB92
:1089D000030111F4801F05D1641E620502D06D00F1
:1089E0004041494121F48011430875F1004350F1A1
:1089F000000041EB045170BC70471CEB410F15D2D5
:108A000023F0004352EA43060BD04FEA4C0CBCEB78
:108A1000410F04D80C0D661E342EB7DDEBE7801A2B
:108A2000994150EA410608BF0021E4E708BF1CEB6A
:108A3000430F28BF6FF00001DDE70268531C03609D
:108A400011707047C1F30A5340F2FE329B1A14DDD5
:108A5000D3F120034FEAE17208DDC90241EA505127
:108A600041F00040D84080185040704703F2E13098
:108A700010B1D24382F000407047002070472E00B2
:108A8000C0F3C7517E390EDDC217D1F1200106DDDA
:108A9000000240F00040C840104450407047D043AE
:108AA00080F000407047002070470000F8B5044691
:108AB00015461E46C9B20E2905DB002090E80E00BF
:108AC00084E80E00F1BD714801EB410210EB820712
:108AD00006F0E2FF28187860002078707E80012080
:108AE0003870BD6097E8070084E80700F1BD0E28E4
:108AF00001DB012070470021644A00EB400398002D
:108B000011540846704710B50E2801DB012010BD36
:108B10005E4900EB400211EB82046088002806D019
:108B200006F0BAFFA16808186060012020700020DC
:108B300010BD10B504460E2C01DB012010BD06F05F
:108B4000ABFF524904EB440201EB82029168081822
:108B500050600020507010BD1FB54FF6FF742346C3
:108B60001F2200216846FFF7A1FF234640F2EB32A7
:108B700003216846FFF79AFF234640F22F12042193
:108B80006846FFF793FF2346492201216846FFF715
:108B90008DFF2346082206216846FFF787FF2346FC
:108BA00040F2292207216846FFF780FF234640F262
:108BB000632208216846FFF779FF234667220221D6
:108BC0006846FFF773FF234640F283120B21684685
:108BD000FFF76CFF234640F629420D216846FFF758
:108BE00065FF012340F2DC520A216846FFF75EFF71
:108BF0001FBD10B4C9B20E2905DB002191E81C008D
:108C000080E81C0008E0214A01EB410302EB8301EC
:108C100091E81C0080E81C0010BC70470E2806DAA2
:108C200000211A4A00EB400302EB830041707047B9
:108C300038B5002425E006F02FFFA9680818686001
:108C40001EE0124804EB440110EB8105287801284E
:108C500016D106F021FF6968814211D201206870A7
:108C60006888002805D04FF6FF71884201D0401E69
:108C7000688068880028DED1002028706860A860BD
:108C8000641C0E2CDDDB31BD0000000050300020E4
:108C9000C11768B14840401AB0FA80F29040D21C27
:108CA000C907C2F5846241EA025202EBD0214005B5
:108CB00070470000C2175040801AB0FA80F10AD005
:108CC0008840D1F19D01D20742EAC151020672F1FA
:108CD000004241EB10207047FF2212EAD05C1DBF1A
:108CE00012EAD153944593422BE09C44D30780EA87
:108CF00001021A4043EA002043EA0121A1FB0030AF
:108D0000C04238BF40007CF17F010BDBFE294ADA0C
:108D10005B0842EAC15153EA006373F1004C51EB26
:108D200010207047D1F1080CDCF120012FDB5B082B
:108D300010FA01F10B4320FA0CF073F1004150419D
:108D4000704794451CBF02EAD153934280EA010266
:108D500002F000421DD0400019D0490017D05BB985
:108D6000634514D00902B1FA81F39940BCEB030CBE
:108D7000C00140F00040C1E70002B0FA80FC10FAE8
:108D80000CF0B3EB0C0CC90141F00041B6E7100048
:108D9000704740000AD0490008D010F1807F94BF8E
:108DA00011F1807F02E042F0FF407047D0437047EE
:108DB00005281BD8DFE800F003070B0F131700206E
:108DC0007349088070470A20714908807047142051
:108DD0006F490880704728206D49088070475020EF
:108DE0006B4908807047B42069490880704738B5DE
:108DF00084B004460D460121084600F02AFCADF877
:108E00000450ADF808400020ADF80A00ADF80600A7
:108E100001A94FF0804000F05BFC01214FF0804041
:108E200000F004FD012211464FF0804000F0F4FCF8
:108E300001214FF0804000F0D4FC1C208DF8000090
:108E400001208DF8010002208DF8020001208DF82C
:108E50000300684608F0C9F905B030BD38B584B0E4
:108E600004460D460121042000F0F3FBADF8045048
:108E7000ADF808400020ADF80A00ADF80600454CFA
:108E800001A9204600F024FC0121204600F0CEFC80
:108E900001221146204600F0BFFC0121204600F0CF
:108EA000A0FC1E208DF8000000208DF8010001209C
:108EB0008DF802008DF80300684608F096F905B0B9
:108EC00030BD35480088704700203349088070471E
:108ED00031480188491C0180704738B502F0FCFE1A
:108EE00004462B4D02F02AFF002813D068880A3070
:108EF000688001462A8889B2914202D10021274A1E
:108F0000116080B2B0F5967F04DB002068800120FC
:108F10002249086068680A306860214988422ED377
:108F2000002C05D100221146084608F0ABF91EE0DE
:108F3000012C05D100221146FF2008F0A3F916E00C
:108F4000022C05D10022FF21104608F09BF90EE00B
:108F5000032C05D10022FF21084608F093F906E012
:108F6000042C04D1FF221146084608F08BF900209A
:108F700068600C48017801F0FD01017031BD0A49BB
:108F8000884204D30748017841F00201017031BDE5
:108F9000C4320020000800400A3300209C01214216
:108FA000E9620500800500201109050062B38B0706
:108FB00008D0521E11F8013B00F8013B00F024805C
:108FC0008B07F6D1830740F0208000BF103A07D30B
:108FD00030B4B1E83810103AA0E83810F9D230BCFB
:108FE000530724BFB1E80810A0E8081044BF51F8A7
:108FF000043B40F8043BD20724BF31F8022B20F891
:10900000022B44BF0B7803707047121F17D35B000D
:1090100009D151F8043B20F8023B1B0C121F20F829
:10902000023BF6D20BE051F8043B00F8013B1B0A6F
:1090300020F8023B1B0C121F00F8013BF3D238BF93
:10904000121D521E24BF11F8013B00F8013BF8D855
:109050007047000030B44FF6FF73002400E0641C3A
:109060008C420FD2025D53400022082AF7D21D46DF
:109070006D08DB072B4603D583F4204383F00103FF
:10908000521CF2E7180200EB132030BC7047F0B41A
:109090000B684C6800252E461CE027467F0987EAAE
:1090A0000417E71905F0030C52F82CC0AC448CEA05
:1090B0000707FB18204F7D191F467F0987EA031712
:1090C000DF19C5F3C12C52F82CC0AC448CEA070759
:1090D0003C19761C0746BE42DFD30B604C60F0BCE7
:1090E0007047F0B40B684C68134D454300261CE0F4
:1090F0001F467F0987EA0317DF19C5F3C12C52F811
:109100002CC0AC448CEA0707E41B0C4F7D192746A2
:109110007F0987EA0417E71905F0030C52F82CC001
:10912000AC448CEA0707DB1B761C8642E0D30B605D
:109130004C60F0BC70470000B979379E4786C86123
:10914000014648B1B0FA80F18840C91CC1F584617C
:10915000090501EBD02140057047000081B0009067
:109160000098411E00910028FAD101B0704780B5E7
:1091700001210C2000F062FA0820ADF80000142054
:109180008DF8030003208DF802006946374808F087
:10919000F1FD4FF40040ADF8000014208DF80300FD
:1091A00003208DF802006946314808F0E3FD0120F4
:1091B000304908603049086001BD38B52E4C0120A7
:1091C00020602C4D28600520FFF7C8FF002020609C
:1091D0000520FFF7C3FF0020286031BD38B5254CBE
:1091E00000202060244D28600520FFF7B7FF0120F4
:1091F00020600520FFF7B2FF0120286031BD38B59F
:10920000012420461C4908600520FFF7A7FF1B48E2
:109210000068002800D10024164D01202860052098
:10922000FFF79CFF002028600520FFF797FF2046EE
:1092300032BD70B505460F4C00202060064610E098
:109240002846C0B2C0090C4908606D000520FFF730
:1092500085FF012020600520FFF780FF00202060AF
:10926000761C3046C0B20828EADB70BD000C014015
:10927000000801408C812142BC0121423C01214275
:1092800070B504460D461646FFF797FF640020466A
:10929000C0B2FFF7CEFFFFF7B2FF2846FFF7C9FFC6
:1092A000FFF7ADFF3046FFF7C4FFFFF7A8FFBDE8AB
:1092B000704093E7F8B504460D4616461F46FFF783
:1092C0007CFF76003046C0B2FFF7B3FFFFF797FF91
:1092D0003846FFF7AEFFFFF792FF05E014F8010BE9
:1092E000FFF7A7FFFFF78BFF2846451EC0B20028F7
:1092F000F4D1BDE8F14071E7B0B581EA030C0CF0A0
:10930000004C40F2FF7515EA11541DBF15EA1357C2
:10931000AC42AF4239E0E41923EA455343F48013E9
:10932000C90241F0004141EA505EC7021100A7FBAB
:10933000020200284FF00000EEFB01204FF0000178
:10934000E3FB072118BF42F0010240180021494108
:10935000E3FB0E01A4F580640F0302D252004041EA
:10936000494154F101046CDD470872F1004250F1AB
:10937000000051EB0451A1F580115CBF41EA0C01E2
:10938000B0BD4CEA05510020B0BD05EA1357AC4210
:1093900014BFAF4241E050EA410E1CBF52EA430EF7
:1093A00002E061460020B0BD24423C441BD15FEA8C
:1093B000070EF6D0090302BF01460020AEF1140EDD
:1093C000B1FA81F7AEEB070401FA07FE0C37C7F1DB
:1093D000200100FA07F7C8404EEA000E23EA455381
:1093E00043F48013A2E733F00043B3FA83F704BFDA
:1093F000B2FA82FE77440B3FE41BB7F1200E2FBF79
:1094000002FA0EF3BB40C7F1200E22FA0EFE38BF5F
:1094100043EA0E03BA40641C82E750EA410E14BFCF
:1094200052EA430E6FF000014FF4001717EB430FA1
:109430008ABF194617EB410FB5E74CEA05510020EA
:10944000B0BDD4F10104B4F120070FDAC4F1200754
:10945000520828BF42F0010210FA07F501FA07F797
:10946000E1BF2A43E0403843E1400FE0352C98DC6F
:10947000C7F1200452EA400220FA07F218BF42F076
:10948000010231FA07F0A1400A43002172F10042C3
:1094900050F1000051EB0C01B0BD000070B44FF072
:1094A000004591EA030F7FF513AA6B40841A71EB14
:1094B000030603D2001BB141121973414FF4001C83
:1094C0001CEB410F34BF7CEB430442E00C0DA4EBDA
:1094D0001356352E4FDC45EAC323DB0A45EAC1218A
:1094E000C912B6F120050DDD63FA05F6EB4086EAF8
:1094F0000305124218BF45F00105C01851F10001E3
:109500000CD213E062FA06F5F2405540F3415A409E
:10951000B340F3405A408018594107D349085FEAE5
:1095200030005FEA350528BF45F0010501F58011DF
:10953000420875F1004250F1000041EB04514E0029
:1095400016F5001F70BC38BF70470020090D0905D3
:1095500070471CEB410F10D252EA43060BD0BCEB14
:10956000410F05D80C0DAB43661E342EB6DD02E06C
:10957000AB438018594170BC704770BC7047000005
:109580004849086840F0010008604A6846480240BF
:109590004A600A68454802400A60086820F4802052
:1095A0000860486820F4FE0048604FF41F0088609F
:1095B00070473F49086070473E4A136823F47C13A4
:1095C00018430843106070473B49086070473949A9
:1095D0000A68920850EA82000860704735480068BF
:1095E00000F00C00704733490A6822F0F002104383
:1095F000086070472F490A6822F4E062104308604F
:1096000070472C490A6822F4605242EAC0020A609C
:1096100070472A490860704726490A6822F4404288
:10962000104308607047264A0029116802D0084399
:109630001060704721EA000010607047214A00293D
:10964000116802D008431060704721EA00001060E2
:1096500070471D4A0029116802D008431060704706
:1096600021EA000010607047184A0029116802D0F2
:1096700008431060704721EA0000106070470146FF
:109680004009084A012801D1106804E0022801D1EC
:10969000106A00E0506A01F01F01C84000F00100AC
:1096A00070470000001002400000FFF8FFFFF6FEC8
:1096B000000042420410024060004242D800424290
:1096C00014100240181002401C1002400C100240FE
:1096D00010B40488DFF8A031984212D0DFF8B0212E
:1096E00090420ED0B0F1804F0BD0DFF89021904225
:1096F00007D0DFF88C21904203D0DFF88821904218
:1097000004D14FF68F7214404A881443DFF8782151
:10971000904208D0DFF87421904204D04FF6FF4207
:109720001440CA88144304808A8882850A88028586
:1097300098420FD0DFF8582190420BD0DFF8542127
:10974000904207D0DFF85021904203D0DFF84C213F
:10975000904201D1097A01860121818210BC7047B3
:1097600030B4038C4FF6FE7213400384058C83885B
:10977000048B4FF68C7214400A8814434FF6FD7226
:1097800015400A8915434A881543DFF8EC209042BA
:109790000FD0DFF8FC2090420BD0DFF8F820904289
:1097A00007D0DFF8F420904203D0DFF8F020904299
:1097B00010D14FF6F77215404A8915434FF6FB72E8
:1097C00015408A8815434FF6FF4213408A89134398
:1097D000CA89134383800483C9888186058430BC89
:1097E0007047002904D0018841F0010101807047D1
:1097F00002884FF6FE710A40028070470029B0F8D7
:10980000441004D041F40041A0F844107047C1F363
:109810000E01A0F844107047002A828902D011433B
:109820008181704722EA010181817047002904D0BB
:10983000018841F080010180704702884FF67F71F6
:109840000A4002807047038B4FF6F77213401943AA
:10985000018370478186704702460020138A0B40BF
:1098600092891140002B02D0002900D001207047BE
:10987000C943018270470000002C014000040040F1
:1098800000080040000C00400010004000140040A0
:1098900000340140004001400044014000480140C4
:1098A000094908607047094908607047084908601D
:1098B00070474AF6AA200449086070474CF6CC402D
:1098C000014908607047000000300040043000404B
:1098D000083000400448C06102210172034901625E
:1098E000034A4262086800472C32002054060020D8
:1098F00084060020000000E0F8180C0C0C8CCC78DA
:10990000F8E000000000001F7F78CCC6C3C1C06033
:109910007F1F000000000000303038FCFC00000019
:109920000000000000000000C0C0C0FFFFC0C0C0B9
:109930000000000000000070781C0C0C0C0C8CDC8B
:10994000F8700000000000C0E0F0F8DCCEC7C3C132
:10995000C0C0000000000070781C0C0C0C0C0C9CAB
:10996000F8F000000000003878E0C3C3C3C3C3E7C9
:109970007D3800000000000080C0E070381CFCFC56
:10998000000000000000000F0F0D0C0C0C0CFFFF7E
:109990000C0C0000000000FCFC8C8C8C8C8C8C8CE3
:1099A0000C0C00000000003171E1C1C1C1C1C1E374
:1099B0007F3E000000000000C0E070381C0C0C0C62
:1099C000000000000000003F7FE7C3C3C3C3C3E73C
:1099D0007E3C00000000000C0C0C0C0C0C0CCCFCB1
:1099E0003C0C0000000000000000C0F03C0F030031
:1099F0000000000000000000F0F89C0C0C0C9CF82B
:109A0000F00000000000003C7EE7C3C3C3C3C3E70F
:109A10007E3C0000000000F0F89C0C0C0C0C0C9C30
:109A2000F8F000000000000001C3C3C3E3733B1F54
:109A30000F03000000000000000000000000000014
:109A40000000000000000000000000000000000016
:109A5000000000000000000000000000F000000016
:109A60000000000000000101010101011F010101CE
:109A700001010100000000000000000000000000E3
:109A800000000000000101010101010101010101CB
:109A9000010101000038283880C0606060606040CB
:109AA00080000000000000001F3F606060606020D8
:109AB00010000000000000000000C0C0C0C0000096
:109AC00000000000000000000000303030300000D6
:109AD000000000000038283800FCFC8C8C8C8C8C3A
:109AE0008C00000000000000007F7F0101010101E7
:109AF00001000000FCFC0000000000C0C0000000ED
:109B00000000FCFC7F7F30180C0603010103060CEB
:109B100018307F7F00000C12120C00FEFE86868635
:109B20008686060000000000000000FFFF01010122
:109B30000101000000806010080464940404B44C27
:109B40000484848484848404040404040404844415
:109B50002464A42424242424242424E40408106059
:109B6000800000000000806010080484C4E4E4E485
:109B7000E4C4840404040404040404040404040485
:109B800004040404040484C4E4E4E4E4C484081085
:109B900060800000000718204080828180828285DA
:109BA00085888F8888888F858585858585858D952D
:109BB000A7B0AFA0A0A0A0A0A0A0A0BF80402018E8
:109BC0000700000000000718204080848C9C9C9CAB
:109BD0009F8F878383838383838383838383838329
:109BE000838383838383878F9F9C9C9C8C8440206A
:109BF0001807000000806010080464940404B44C4A
:109C00000484848484848404040404040404844454
:109C10002464A42424242424242424E40408106098
:109C200080000000000000F8F8808080F80080408C
:109C3000404040800080404040408000004040F86C
:109C400040400000D00040804040408000804040C4
:109C50004080000000071820408082818082828539
:109C600085888F8888888F858585858585858D956C
:109C7000A7B0AFA0A0A0A0A0A0A0A0BF8040201827
:109C8000070000000000001F1F0101011F000F124C
:109C90001212120B000C121212120F100000000F01
:109CA000100800001F00001F0000001F00478888E8
:109CB000887F000000E0F01010200000808080808D
:109CC00000008080F08080008080F0808000A00014
:109CD0008000808080800000008080808000000004
:109CE000000000000000806010080484C4E4E4E484
:109CF000E4C4840404040404040404040404040404
:109D000004040404040484C4E4E4E4E4C484081003
:109D100060800000000811111F0E000F12121212B5
:109D20000B0000000F10080000000F1008001F00BB
:109D3000001F000000001F004F909090907F0000D7
:109D40000000000000000718204080848C9C9C9C30
:109D50009F8F8783838383838383838383838383A7
:109D6000838383838383878F9F9C9C9C8C844020E8
:049D700018070000D0
:10A00000FFFFFFFFFFFFFFFFFFFFFFFF01F0004229
:10A010008B1AA3F16051B1F5801F0ADBB1F17F6F9C
:10A020001FD242EAC102C10071F1004142EB5070FF
:10A0300070470B15C3F10903212B10D2890241EAA5
:10A04000905180020128494141F0004121FA03F07A
:10A05000C3F12003994071F1004150417047100055
:10A0600070476FF0000013EB103F5CBF000E42EA38
:0EA07000C0507047004870470C070020704732
:10A08000042801D1014870470020704799FA000860
:10A090000146122902DADFF89C1408707047DFF8D5
:10A0A000940400787047DFF8900400787047024607
:10A0B000C021DFF88804FEF719B80A2251430128AD
:10A0C00007D101EBC101052091FBF0F101F54861D9
:10A0D00006E001EB8101A1F57A51092091FBF0F135
:10A0E000104691FBF0F002FB1012052A02DB401C27
:10A0F00000B2704700B27047000000002DE9F04345
:10A1000087B081460C46904601F0FCFD3C2190FB57
:10A11000F1F501F0F7FD3C2190FBF1F1C1EB0112EB
:10A12000A0EB8206DFF81074B888401CB88000B23B
:10A130001A28C0F2EC800020B880F888401CF88013
:10A14000B9F1010F2BD06DD3B9F1030F01D04BD36F
:10A1500068E000B2142801DD0020F880B7F906009D
:10A1600001460A290FDA00210191DFF8D4230146C4
:10A17000521A521E00920823024692B219465620E5
:10A1800000F016F94EE014294CDA00210091082362
:10A19000012219464C3080B2FEF74FF842E000B27F
:10A1A000102801DB0020F880B7F9061008460828BF
:10A1B0000DDA00200190DFF88C03009008230A22BA
:10A1C000C1F10F0109B2562000F0F2F82AE0102880
:10A1D00028DA0020009001230A22C1F1170189B278
:10A1E0005620FEF72AF81DE000B2102801DB0020FF
:10A1F000F880B7F906100846082809DA002001900F
:10A20000D148009008230A22562000F0D1F809E036
:10A21000102807DA0020009001230A2289B2562074
:10A22000FEF70BF8B8F1000F31D00821684601F0B5
:10A23000C7FDBDF800800021684601F0C1FDBDF8F2
:10A2400000005FFA88F8B8F1000F0ED1FEF770F940
:10A25000BE49FEF77BF9FEF7F7F902464FEA010324
:10A2600038A102A8FEF714FA38E0FEF7E5FAFEF787
:10A27000EBF90022B64BFEF723FBFEF7E3FB00B23F
:10A280004FEA000231A102A8FEF702FA26E00521FA
:10A29000684601F095FD0098FEF7F2FB80460A2122
:10A2A000684601F08DFDBDF9000000280DD0414643
:10A2B00009B20120FFF701FF0A2190FBF1F212B26F
:10A2C00098A102A8FEF7E4F908E00FFA88F80A203E
:10A2D00098FBF0F294A102A8FEF7DAF9002302AA93
:10A2E00019464820FEF7B1F8002C06D13A78521CE6
:10A2F0008EA102A8FEF7CCF903E08DA102A8FEF71B
:10A30000C7F9002302AA19463A20FEF79EF828460C
:10A31000C0B2642803DB01F0E3FC00252E46F6B250
:10A320003346EDB24FEA05020AA102A8FEF7B0F9E2
:10A33000002302AA08213820FEF787F807B0BDE8FD
:10A34000F08300002025322E30665600202532642E
:10A3500057200000253032643A2530326400000076
:10A36000002800D5704710B400291FD460281DDCD8
:10A3700011291BDA0B469B1001EB5374E4102346A2
:10A38000DBB2A1EBC401012404FA01F103EB4304A5
:10A3900000EB4410C12809DA684B002A1A5C02D08D
:10A3A0001143195402E022EA0101195410BC70470C
:10A3B0002DE9F64F83B0834688460F9C46460190B0
:10A3C0001946491E0846801001EB5071C910491CFE
:10A3D000BDF8100041430291BDF810705F44BFB258
:10A3E0004FF000094846ADF8000014E00022414655
:10A3F00009B200B2FFF7B4FF5EE0B0460BF1010B0B
:10A4000009F101091FFA89F9BDF80230BDF8000011
:10A41000401CADF80000BDF800000299884271D2DE
:10A420002046042839D8DFE800F026033823260028
:10A43000414609B2584600B2404A0D46AD1001EB04
:10A440005575ED1005EB450C00EB4C15525D891B65
:10A450000E9D8C464FEAAC0C01EB5C71C910BDF847
:10A4600010C00CFB01010198091A6D5C154314E042
:10A470000E9DEDB211E0414609B2891B0E9A0846C5
:10A48000801001EB5071C910BDF81050584600B251
:10A4900005FB01010198091A555C4FF0000AADF85F
:10A4A000023016E0A7EB0900E9079FD501224146DB
:10A4B00009B200B2FFF754FFADB26D0808F1010810
:10A4C000404600B2801BBDF80210884295D00AF1C8
:10A4D000010A504680B2082896DA20460428E1D0C6
:10A4E000E80707D50122414609B2584600B2FFF7F6
:10A4F00037FFE1E70022414609B2584600B2FFF7B4
:10A500002FFFD9E705B0BDE8F08FE0B5002001903E
:10A510000A4800901023602200210846FDF73CFE07
:10A5200000200EBD25644600256443004D256400CF
:10A53000412000001733002044070020902F002006
:10A540008E4E01085C4E01087A4E010800007A44E4
:10A550000000E03F3EB50D461446C01F09282ED826
:10A56000DFE800F0050505191E28282328280A2100
:10A57000684601F025FCBDF90000002805D040F236
:10A5800096202880D420208037BD4FF4AF702880DB
:10A590006420208037BD782028800020208037BDAF
:10A5A0000A2028800120208037BD05202880002037
:10A5B000208037BD012028800020208037BD00206A
:10A5C0002880208037BD000010B50446C91F092926
:10A5D00049D8DFE801F0050A0F141648181A1C477D
:10A5E00002EB82004000A08010BD02EB8200400020
:10A5F000208210BD02EB82004000608210BDE2812B
:10A6000010BDA28110BD628310BD228310BD104613
:10A61000A18A884227D0A282B4F90410002A10D05F
:10A620000120FFF74AFDA080B4F910100120FFF7C8
:10A6300044FD2082B4F912100120FFF73EFD608234
:10A6400010BD0020FFF739FDA080B4F910100020E4
:10A65000FFF733FD2082B4F912100020FFF72DFD23
:10A66000608210BDE28210BD0EB401464FF0FF3093
:10A67000C91F092920D8DFE801F005080B0E111FBA
:10A6800014171A1DBDF9040016E0BDF9100013E0FF
:10A69000BDF9120010E0BDF90E000DE0BDF90C008F
:10A6A0000AE0BDF91A0007E0BDF9180004E0BDF9A1
:10A6B000140001E0BDF9160003B070472DE9F04128
:10A6C00092B00746FFF7EBFC054605210FA8FEF701
:10A6D00090FA06AA0DF11A012846FFF73BFFDFF8B2
:10A6E000906B06F12404E078002814D00020E0707C
:10A6F00001F0FFFA2071304601F00FFEB6F91400A8
:10A7000060810520FEF78AFA012342F210720521CA
:10A710006846FEF7CBF9A8464046C01F0A2800F25B
:10A720005F82DFE810F00B00AD00D70043007E0031
:10A73000090136016C019D01D3010002DFF8341BD1
:10A740000878002807D000200870B6F904000A2114
:10A7500090FBF1F020812078002840F04182002316
:10A760000FF65C1219460846FDF76FFE0B23012217
:10A770000FF6C81107A8FDF78BFF002307AA19469B
:10A780004120FDF762FEB4F90A00002840F0CC80B9
:10A79000B4F908200FF6301107A8FDF779FF002360
:10A7A00007AA08212720FDF750FE19E2DFF8C41A96
:10A7B0000878002804D000200870B6F90E00208127
:10A7C0002078002840F00C8200230FF6041219466E
:10A7D0000846FDF73AFE0B2304220FF6601107A886
:10A7E000FDF756FF002307AA19464120FDF72DFE6D
:10A7F000B4F90820002A05D10FF6701107A8FDF75B
:10A8000047FF03E095A107A8FDF742FFB4F9080050
:10A810000A28C4DA002307AA08212120FDF715FE23
:10A82000DEE1DFF8501A0878002804D00020087014
:10A83000B6F90C0020812078002840F0D181002357
:10A840000FF6980219460846FDF7FFFD0B23052277
:10A850000FF6E80107A8FDF71BFF002307AA19461A
:10A860004120FDF7F2FDB4F908207CA107A8FDF70F
:10A870000FFF002307AA08212120FDF7E6FDAFE125
:10A88000DFF8F0190878002807D000200870B6F922
:10A8900010000A2190FBF1F020812078002840F080
:10A8A0009F8100230FF6400219460846FDF7CDFDB3
:10A8B0000B2302220FF6840107A8FDF7E9FE00230F
:10A8C00007AA19464120FDF7C0FDB4F90A00002887
:10A8D0002AD15DE7DFF89C190878002807D000200E
:10A8E0000870B6F912000A2190FBF1F0208120785F
:10A8F000002840F0758100230FF2F47219460846D3
:10A90000FDF7A3FD0B2303220FF6300107A8FDF787
:10A91000BFFE002307AA19464120FDF796FDB4F9B2
:10A920000A0000283FF434AFB4F908200FF2C871D0
:10A9300007A8FDF7ADFE32E7DFF8381908780028E0
:10A9400003D000200870207920812078002840F072
:10A95000478100230FF2A87219460846FDF775FDDE
:10A960000B2306220FF2D47107A8FDF791FE0023F6
:10A9700007AA19464120FDF768FDB4F90800002830
:10A9800040F0CA800023C0A208212720FDF75DFD0A
:10A9900026E1DFF8E0180878002804D000200870CD
:10A9A000B6F91A0020812078002840F01981002390
:10A9B0000FF2587219460846FDF747FD0B23072290
:10A9C0000FF2787107A8FDF763FE002307AA194666
:10A9D0004120FDF73AFDB4F90800002807D0002314
:10A9E0000FF2787208212120FDF72FFDF8E00023F7
:10A9F0000FF2707208212120FDF727FDF0E0DFF84B
:10AA000074180878002804D000200870B6F91800DF
:10AA100020812078002840F0E38000230FF2F862C4
:10AA200019460846FDF711FD0B2308220FF20C71A1
:10AA300007A8FDF72DFE002307AA19464120FDF7C0
:10AA400004FDB4F9082005A107A8FDF721FE0023A5
:10AA500007AA08212120FDF7F8FCC1E02533640096
:10AA6000DFF810180878002804D000200870B6F924
:10AA7000140020812078002840F0B28000230FF2DB
:10AA8000A06219460846FDF7E0FC0B2309220FF2ED
:10AA9000AC6107A8FDF7FCFD002307AA1946412079
:10AAA000FDF7D3FCB4F90800002807D000230FF20B
:10AAB000CC6208211520FDF7C8FC91E000230FF2BD
:10AAC000C86208211520FDF7C0FC89E0DFF8A41753
:10AAD0000878002804D000200870B6F916002081FC
:10AAE000207800287CD100230FF2406219460846E6
:10AAF000FDF7ABFC0B230A220FF2406107A8FDF71C
:10AB0000C7FD002307AA19464120FDF79EFCB4F9B2
:10AB1000080000283FF436AF0023B8A20821272000
:10AB2000FDF793FC5CE0DFF84C170878002801D0B3
:10AB3000002008702078002813D100230FF2F4526F
:10AB400019460846FDF781FC0B231A460FF2EC511B
:10AB500007A8FDF79DFD002307AA19464120FDF730
:10AB600074FC207801283BD19DF83D00002837D0A7
:10AB7000A078401CA0706078002807D000230FF256
:10AB8000C45208211520FDF760FC06E000230FF2F7
:10AB9000C05208211520FDF758FC6078401E804106
:10ABA000C00F6070A078052807DC01234FF4FA720B
:10ABB00005216846FDF77AFF0CE00020A070208098
:10ABC000304601F0AFFB012342F2107205216846C6
:10ABD000FDF76CFF00208DF83D000520FEF71EF804
:10ABE0002078012840F0F480A8F10708B8F1090F97
:10ABF00000F2D680DFE808F005050594186C804A5D
:10AC0000AFC3B4F908200FF26C5107A8FDF740FD5F
:10AC1000B4F908000A28C0F29780002307AA082187
:10AC20002720FDF712FCBBE0B4F908200FF24451D5
:10AC300007A8FDF72DFD002307AA08212120FDF715
:10AC400004FCB4F90800A1790246914200F0A88002
:10AC5000FEF71EF802460B46072001F049FAB4F948
:10AC60000800FEF727F8DFF8C81BFDF76FFCDFF8D8
:10AC7000C41BFEF731F8FDF703FFC0B2FDF7C4FABD
:10AC80002089A0718CE000BF4F464600B4F908202F
:10AC90000FF2E04107A8FDF7FBFC002307AA0821FB
:10ACA0002120FDF7D2FBB4F90800617902469142F8
:10ACB00076D080B2FEF77CF8B4F90800FDF7E8FF23
:10ACC00002460B46092001F013FA2089607167E003
:10ACD000B4F90800002806D0002348A20821272044
:10ACE000FDF7B3FB05E0002345A208212720FDF76F
:10ACF000ACFB2089207153E0B4F90800002807D08C
:10AD000000230FF2584208212120FDF79EFB47E067
:10AD100000230FF2504208212120FDF796FB3FE06F
:10AD2000B4F90820002A05D10FF2404107A8FDF729
:10AD3000AFFC04E00FF23C4107A8FDF7A9FCB4F911
:10AD400008000A28BFF669AF002307AA08212120BE
:10AD5000FDF77BFB24E0B4F90800002807D00023AE
:10AD60000FF2184208211520FDF76FFB18E00023B1
:10AD70000FF2144208211520FDF767FB10E0B4F92B
:10AD80000800002806D000231CA208212720FDF778
:10AD90005CFB05E000231AA208212720FDF755FBE4
:10ADA0002846112814D0002002900190009008231A
:10ADB0001A461146FDF783FB002002900120019006
:10ADC0000020009008231A4611465820FDF777FB13
:10ADD000A078002840F03181384601281CD1207825
:10ADE00001280FD12089401E208100B2BDF8181023
:10ADF000884221DABDF9180020811DE0204F4E0065
:10AE00004F464600002840F00E816D1E2846C0B215
:10AE1000062857DC112555E0022839D12078012871
:10AE20001AD12089801E208100B2BDF818108842F6
:10AE300002DABDF91800208128460A2874D1B4F935
:10AE40000800012805D0022803D0032801D00428D7
:10AE50006AD10020208167E0002840F0E4800120D2
:10AE60002070034641F2883205216846FDF71EFE38
:10AE70002846112840F0D7800020A0700120607083
:10AE800003464FF4FA7205216846FDF70FFECAE04B
:10AE900004282AD1207801280BD12089401C208148
:10AEA000BDF81A1000B281422FDABDF91A002081D4
:10AEB0002BE0002840F0B7806D1C2846C0B2122855
:10AEC00000DB07250120DFF8AC1308700020FFF736
:10AED000EEF82846C0B2FFF7DBF8012342F2107209
:10AEE00005216846FDF7E2FD9DE005284CD120785C
:10AEF000012821D12089801C2081BDF81A1000B2C0
:10AF0000814202DABDF91A00208128460A280BD1B5
:10AF1000B4F90800012805D0022803D0032801D085
:10AF2000042801D105202081012341F28832052126
:10AF30006846FDF7BBFD76E0002874D10120E07083
:10AF4000207900F0D2FE314684B068462422FEF714
:10AF50003DF80FBC01F0D6F9F08A002803D001209B
:10AF600000F0E4FE02E0002000F0E0FE02F023FC2E
:10AF70000020FFF79CF80020FFF78AF80022134614
:10AF80000C2001F0B5F84EE007281BD120780128ED
:10AF900049D1002020702846112805D0208902467A
:10AFA00029463046FFF710FBB6F9140060810020F7
:10AFB000FFF77DF8012342F2107205216846FDF784
:10AFC00075FD30E0082F2ED12078012817D1002000
:10AFD0002070314683B068462422FDF7F7FF0EBC8F
:10AFE0002846FFF741FB20810020FFF760F801238E
:10AFF00042F2107205216846FDF758FD13E0002863
:10B0000011D101209B490870E0700020FFF74FF834
:10B010000020FFF73DF8002213460C2001F068F8ED
:10B020000520FDF7FBFD2078012803D1012003F066
:10B03000E9F802E0002003F0E5F89DF83D00002863
:10B040003AD02078002812D101208A490870E07097
:10B050000020FFF72CF80020FFF71AF80022134613
:10B060000C2001F045F80520FDF7D8FD24E001286B
:10B0700016D100202070208902462946C9B23046E8
:10B08000FFF7A2FAB6F9140060810020FFF70FF86D
:10B09000012342F2107205216846FDF707FD0BE01F
:10B0A000A078002808D100202070012342F21072FD
:10B0B00005216846FDF7FAFC12B0BDE8F0810000FA
:10B0C0004D312054656D700025336443000000004D
:10B0D000536C6565702054696D6500004261636B57
:10B0E0006C696768740000004D322054656D700013
:10B0F0004D332054656D7000253364460000000018
:10B1000054696C7420416E676C65000053686F77FA
:10B110002054797065000000566F6C756D650000F5
:10B1200054656D7020547970650000004C6F772075
:10B1300043757200526573746F7265002532642F17
:10B1400025326400436F6D706C65746564000000A7
:10B15000202020202020202020000000506F776534
:10B1600072000000566F6C7420000000204F4646AD
:10B170000000000025336420000000004465677271
:10B18000656573204600000044656772656573203D
:10B19000430000002DE9FE438046894600F0B6FDDD
:10B1A000054603F035F907460A21684600F008FE17
:10B1B000BDF900403888022858DB7888002855D02F
:10B1C000DFF8206AB9F1000F13D000207080B7F9C2
:10B1D000040000EB80014800002C07D0014609B2B2
:10B1E0000020FEF76AFF03F07FFA02E000B203F0EE
:10B1F0007BFA3078002805D1B8F1030F02D1012085
:10B20000307075603078002830D07188084607EBC0
:10B210008000C28870688218954227D3491C7180CB
:10B22000388889B281420AD300207080788800284B
:10B2300005D04FF6FF71884201D0401E7880381D3E
:10B24000718830F9210000EB80014800002C07D004
:10B25000014609B20020FEF730FF03F045FA02E094
:10B2600000B203F041FA002030707560BDE8F7834A
:10B27000C8050020E43200202DE9F0478EB00746D3
:10B28000FEF70DFF824605210BA8FDF7B2FC012158
:10B29000684600F095FDBDF900800521684600F084
:10B2A0008FFD0098FDF7ECFB81460FFA89F903F05A
:10B2B0008FF906460A21684600F082FDBDF900407C
:10B2C000DFF82459BAF1030F04D0BAF1040F00F0EB
:10B2D000508100E20D210BA8FDF78BFC002C1FD044
:10B2E00041460120FEF7E9FE80462878002803D079
:10B2F00002280FD007D313E00221684600F060FD5A
:10B30000BDF900900CE00321684600F059FDBDF93D
:10B31000009005E00421684600F052FDBDF9009060
:10B3200000203146032900D10F2000EB0901002C39
:10B3300017D041450CDBA9EB0000804508DB0A2053
:10B3400099FBF0F20FF6D40103A8FDF7A1F91FE075
:10B350000A2098FBF0F20FF6C40103A8FDF798F954
:10B3600016E041450CDBA9EB0000804508DB0A2014
:10B3700099FBF0F20FF6AC0103A8FDF789F907E09D
:10B380000A2098FBF0F20FF69C0103A8FDF780F964
:10B39000002303AA19460846FDF734F86878002808
:10B3A0000CD19DF82D0000280AD0E878401E80417D
:10B3B000C00FE8700D20FDF731FC01E00020E870BF
:10B3C000EA7869783046FEF799FE3846022851D16E
:10B3D0002878002803D0022817D00BD31FE00221C1
:10B3E000684600F0EDFCBDF900000A2190FBF1F089
:10B3F000288114E00321684600F0E2FCBDF900005A
:10B400000A2190FBF1F0288109E00421684600F050
:10B41000D7FCBDF900000A2190FBF1F028812889B2
:10B4200000EB80014900002C06D009B20020FEF795
:10B4300044FE03F059F903E0084600B203F054F962
:10B440000020FEF734FE022003F0AFF80420FEF7E0
:10B450001FFE012341F2883205216846FDF726FBD5
:10B46000012002F0CFFE0020E8700120DFF87C17F9
:10B47000087073E0052819D10020FEF718FE00209F
:10B48000FEF706FE022003F090F8002213460C207F
:10B4900000F02EFE0D20FDF72AFB0120A8700020F1
:10B4A0006870E8700D20FDF744FB57E0012849D192
:10B4B0002878401C2870C0B2032801DB00202870C7
:10B4C000002068700120A8700020E8700D20FDF7B2
:10B4D00030FB2878002803D0022817D00BD31FE0B8
:10B4E0000221684600F06CFCBDF900000A2190FBC7
:10B4F000F1F0288114E00321684600F061FCBDF9F9
:10B5000000000A2190FBF1F0288109E0042168463F
:10B5100000F056FCBDF900000A2190FBF1F02881F3
:10B52000288900EB80014800002C07D0014609B2B1
:10B530000020FEF7C2FD03F0D7F80FE000B203F0E1
:10B54000D3F80BE0042802D100F0CAFB06E0082F74
:10B5500004D16878401E8041C00F68706878002868
:10B5600000F0B980A9783046FFF714FE0020A870DB
:10B57000B1E04FF4AF766420002C0FD040F6AC5110
:10B580000120FEF79AFD0A2190FBF1F64FF47A7143
:10B590000120FEF792FD0A2190FBF1F0B5F90810A9
:10B5A00032460B4612B29A4201DA2E8104E002467C
:10B5B00012B2914200DA2881B5F908209BA103A8B4
:10B5C000FDF766F8002303AA19462420FCF75BFF69
:10B5D0000020029001900220009010231A460021C2
:10B5E0000846FCF76CFF0020029001200190022029
:10B5F000009010231A4600215020FCF760FF3846C7
:10B60000012801D002280AD12889401E288101235F
:10B6100041F2883205216846FDF748FA0DE004281A
:10B6200001D0052809D12889401C2881012341F235
:10B63000883205216846FDF739FA9DF82D0000286B
:10B6400001D1072F47D10020FEF731FD0A242889B8
:10B65000604300B203F048F82878002803D002289D
:10B6600019D00CD322E0B5F9080044432046FDF779
:10B670000FFB02460B46022000F03AFD16E0B5F93A
:10B68000080044432046FDF703FB02460B46032017
:10B6900000F02EFD0AE0B5F9080044432046FDF70E
:10B6A000F7FA02460B46042000F022FD012002F0CA
:10B6B0007CFF0320FEF7ECFC0520FDF7AFFA00202D
:10B6C00002F0A0FD002068700120A8700020E87042
:10B6D0000D20FDF72EFA0EB0BDE8F0872DE9FF41F1
:10B6E00006216846FDF785FA9DF80100002856D02E
:10B6F000DFF8FC4425782846302834DA2E462F46D9
:10B70000DFF8F0840020019007EB08000090082388
:10B71000012200213046FEF74BFE0020019008F187
:10B720006000381800900823012219463046FEF7C1
:10B730003FFEC6F15F060020019008F15F00C01BCC
:10B7400000900823012200213046FEF731FE002040
:10B75000019008F1BF00C71B00970823012219467A
:10B760003046FEF725FE6D1C2570EDB2302D13DB43
:10B770004FF6FF7423464FF4C86206216846FDF772
:10B7800095F923463D2200216846FDF78FF90120F7
:10B79000DFF86414087003E00620FDF73FFA00208C
:10B7A00004B0BDE8F081FEB500250B21684600F02D
:10B7B00007FB009802F049FE06462946684600F05D
:10B7C000FFFABDF800700D21684600F0F9FA009C00
:10B7D00042F21170874206DA2A46DFF820340D2043
:10B7E00000F086FC0125322E06DA0022DFF8103444
:10B7F0000D2000F07DFC0125002C03D0022000F07C
:10B80000FCFD0125012000F007FC002806D10022E4
:10B81000DFF8F0330D2000F06BFC012500F054FA46
:10B82000022800D101252846FEBD00002533640012
:10B830000000204100007F432DE9F84390B0064608
:10B84000FEF72DFC044605210DA8FDF7D2F9DFF81F
:10B85000B853002C40F0A58006210AA8FDF7C9F9CD
:10B860009DF82900002844D0687804283ED8DFE8F5
:10B8700000F0030715233100FFF730FF687035E053
:10B8800000200190DFF88403009010236022002143
:10B890000846FEF78DFD0220687027E00020019029
:10B8A000DFF8500300901023602200210846FEF7C5
:10B8B0007FFD0320687019E000200190DFF850033D
:10B8C00000901023602200210846FEF771FD04203D
:10B8D00068700BE000200190C648009010236022A1
:10B8E00000210846FEF764FD012068700620FDF780
:10B8F00095F9012E06D0022E33D0042E1BD0052E32
:10B900003FD06BE10020FEF7D2FBFFF74CFF002891
:10B9100040F06481012028700320FEF7B9FB00226B
:10B92000B64B0C2000F0E4FB0D20FDF7ECF80120F5
:10B93000AE49087052E1012028700020FEF7B7FBE5
:10B940000720FEF7A5FB00224FF080430C2000F0FB
:10B95000CFFB012342F2107205210AA8FDF7A6F8D9
:10B960003CE1012028700020FEF7A1FB0120FEF73A
:10B970008FFB012341F2883205210AA8FDF796F8D2
:10B980002CE1012028700020FEF791FB0220FEF739
:10B990007FFB012341F2883205210AA8FDF786F8D2
:10B9A0001CE1022C40F087802878002822D001205A
:10B9B00000F0CCF9044600202870FEF778FB00BFA9
:10B9C0000FF2702299A102A8FCF762FE002302AADE
:10B9D00019460846FCF739FD0AA8A0470DF12802D0
:10B9E00096A102A8FCF754FE002302AA08211846DB
:10B9F000FCF72BFDA878002818D00020FEF757FB95
:10BA00005FF000038FA219460846FCF71EFD68464A
:10BA100000F053F9DDF804208DA102A8FCF738FEF0
:10BA2000002302AA08211846FCF70FFD300028D099
:10BA3000E878032825D8DFE800F00208111A30461C
:10BA400004281ED10120E8701BE03046022802D1F4
:10BA50000220E87015E00020E87012E0304604286B
:10BA600002D10320E8700CE00020E87009E03046C5
:10BA7000072804D10020E8700120A87001E0002010
:10BA8000E870002E06D0012340F6B83205210AA83E
:10BA9000FDF70CF89DF83500002800F09F8000208D
:10BAA000A870E870FEF703FB0020FEF7F1FA05200E
:10BAB000FDF7B4F892E0012C40F09080287800283F
:10BAC00000F0768002F0C1FC81460121684600F05A
:10BAD00077F9BDF900700A21684600F071F9BDF9E7
:10BAE00000800021684600F06BF9BDF8004000209E
:10BAF0002870FEF7DCFA00F0E7F8012843D100F0E7
:10BB0000D3F800F031FE00904846FDF7D3F84149E4
:10BB1000FCF71CFDFCF798FD02460B464EA102A85F
:10BB2000FCF7B6FD002302AA19460846FCF78DFC77
:10BB30002046FCF7FDFC3849FCF708FDFCF784FDC6
:10BB400004460D46B8F1000F0DD039460120FEF72E
:10BB5000B4FACDE900450A2190FBF1F242A102A816
:10BB6000FCF796FD08E0CDE900450A2097FBF0F2CE
:10BB700041A102A8FCF78CFD002302AA0821184667
:10BB8000FCF763FC14E000BF3FA102A8FCF780FDB6
:10BB9000002302AA19460846FCF757FC3EA102A85A
:10BBA000FCF776FD002302AA08211846FCF74DFC9D
:10BBB000002E06D0012340F6B83205210AA8FCF772
:10BBC00075FF9DF83500002808D00020FEF76FFAB9
:10BBD0000020FEF75DFA0520FDF720F811B0BDE862
:10BBE000F0830000CC32002044070020A432002063
:10BBF00018330020349B0008143300200000F03F6D
:10BC00000000104000002040E4320020F49B0008B7
:10BC1000B49C00080000204100007A4425336441B0
:10BC2000000000002533643D00000000537665727B
:10BC30003A257300322E31310000000048766572DB
:10BC40003A25730053756D4865617454696D6500DC
:10BC50002564206D696E0000523A252E316620540D
:10BC60007970653A2573000054656D703A25644615
:10BC700020563A252E30660054656D703A2564438F
:10BC800020563A252E306600523A2D2D20547970D8
:10BC9000653A4E6F6E65000054656D703A2D2D202B
:10BCA000563A2D2D00000000DFF8181C08884FF6CA
:10BCB000FF72904200D1888B7047DFF8081CD1E9F1
:10BCC0000023C0E900237047DFF8F80BC07A704703
:10BCD000DFF8F01BC8727047DFF8E80B807A704716
:10BCE0000020DFF8E41B08807047DFF8E01B0870D5
:10BCF0007047DFF8D80B007870470020DFF8D01BC2
:10BD000008807047DFF8C00B00887047DFF8B80B79
:10BD100040687047DFF8C01C0870704701B49DF898
:10BD20000000DFF8B81C087001B0704701B49DF83E
:10BD30000000DFF8901B087201B07047DFF89C0C20
:10BD400000787047DFF8980C0088704710B503281A
:10BD500033D8DFE800F0020E1A26DFF8784B2068AF
:10BD6000002804D10020DFF87C1C88472060206870
:10BD700010BDDFF8604B6068002804D10120DFF8B7
:10BD8000641C88476060606810BDDFF8484BA0689D
:10BD9000002804D10220DFF84C1C8847A060A0686E
:10BDA00010BDDFF8304BE068002804D10320DFF835
:10BDB000341C8847E060E06810BD002010BD000022
:10BDC0001CB50446002000900846C0B2102800F3BD
:10BDD0007780C9B200F27480DFE801F0090F1643E2
:10BDE0004A1D353C51585F21262C31666C00DFF826
:10BDF000A40C0088ADF8000062E0DFF8980CB0F900
:10BE00000200ADF800005BE0DFF8880CB0F9040038
:10BE1000ADF8000054E002F08AFC009050E0DFF83A
:10BE2000740C806800904BE0DFF8680C407F8DF860
:10BE3000000045E0DFF85C0C006A009040E0DFF8AD
:10BE4000580C00903CE0DFF84C0CB0F90E00ADF857
:10BE5000000035E0DFF83C0CB0F90C00ADF8000054
:10BE60002EE0DFF8300CB0F91000ADF8000027E04C
:10BE7000DFF8200CB0F91200ADF8000020E0DFF888
:10BE8000140CB0F91A00ADF8000019E0DFF8040C4A
:10BE9000B0F91800ADF8000012E0DFF8F80BB0F9C7
:10BEA0001400ADF800000BE0DFF8E80B007F8DF820
:10BEB000000005E0DFF8DC0BB0F91600ADF800007B
:10BEC000DDE90001C4E9000113BD2DE9F74183B0AC
:10BED0000446DFF87C5CAF8B062638467043284466
:10BEE00004A93246FDF762F87F1CAF83687D002805
:10BEF0002DD04FF08948DFF85C0CDFF8901C03F080
:10BF000097F9FEF783F84146FCF7E6FEFCF7B8FD2B
:10BF10006883DFF87C0CDFF8E01C03F089F9FEF79A
:10BF200075F84146FCF7D8FEFCF7AAFDE882DFF879
:10BF3000600CDFF8C41C03F07BF9FEF767F841469C
:10BF4000FCF7CAFEFCF79CFD288300206875BFB291
:10BF5000032F03DB0020A8830120287500220C2179
:10BF60006846FCF7C3F86946287D002826D00020E3
:10BF700010E006FB00F2009BAF5EFB1800934B68DD
:10BF8000AF1CBF5EFB184B608B682F1DBA5ED318C9
:10BF90008B60401C0328ECDB0098032290FBF2F03E
:10BFA000ADF81000486890FBF2F0ADF81200886818
:10BFB000114690FBF1F0ADF8140025E0002011E0EF
:10BFC00006FB00F2009BAF5EFB1800934B68AF1CB2
:10BFD000BF5EFB184B608B682F1DBA5ED3188B6059
:10BFE000401C80B2AA8B9042EADB009890FBF2F0F2
:10BFF000ADF81000486890FBF2F0ADF812008868C8
:10C0000090FBF2F0ADF81400204604A93246FCF78C
:10C01000CDFF06B0BDE8F08138B584B005460024F8
:10C020000320FFF793FE030004D003AA0DF10A01D9
:10C0300002A89847DDE902010A4601466846FFF773
:10C0400044FF280029D1BDF90800BDF90010A1F571
:10C050009672904203DB01F59671814200DA012469
:10C06000BDF90A00BDF90210A1F59672904203DBFA
:10C0700001F59671814201DA44F00204BDF90C0029
:10C08000BDF90410A1F59672904203DB01F596719B
:10C0900081422ADA44F0040427E0012D25D1BDF9BC
:10C0A00004100846002820DDBDF90000002802D554
:10C0B0004042ADF80000BDF90200002802D5404220
:10C0C000ADF80200DFF8880AB0F91A2091420BDAC5
:10C0D000B0F91610BDF90020914206DBB0F9180046
:10C0E000BDF90210884200DB0124204605B030BDB6
:10C0F0000146102900DD704780B50E2900F0B3809D
:10C10000102800F2B080DFE800F00911192938AEDC
:10C110006B77878F97474F57AE9FA70010461946FA
:10C12000FCF790FCDFF8D41B088001BD10461946CF
:10C13000FCF788FCDFF8C41B488001BD1046194697
:10C14000FCF780FCA0F57A7140F6C51289B29142E5
:10C1500080F08980DFF8A41B888001BD1046194655
:10C16000FCF770FCA0F57A7140F6C51289B29142D5
:10C1700079D2DFF8881B088201BD10461946FCF70A
:10C1800061FCA0F57A7140F6C51289B291426AD27B
:10C19000DFF8681B488201BD10461946FDF736FFDF
:10C1A000DFF8581B886001BD10461946FCF74AFCB1
:10C1B000DFF8481B487701BD1046194603F03AF8EE
:10C1C000002850D0DFF8341B11280A6A02D210432D
:10C1D000086201BD20F0004022EA0000086201BDB3
:10C1E00010461946FCF72EFC014689B279293ADA45
:10C1F000DFF8081BC88101BD10461946FCF722FC78
:10C20000014689B20B292EDA014689B200292AD0CB
:10C21000DFF8E81A888101BD10461946FCF712FCC8
:10C22000DFF8D81A488301BD10461946FCF70AFC0E
:10C23000DFF8C81A088301BD10461946FCF702FC56
:10C24000DFF8B81A888201BD10461946FCF7FAFBE0
:10C25000DFF8A81A087701BD10461946FCF7F2FB73
:10C26000DFF8981AC88201BD7CB504460A216846E9
:10C27000FFF7A6FDBDF90050002C02D0012C0BD019
:10C2800073BD0020FDF713FF0020FDF701FF022022
:10C29000BDE8764002F089B9FDF705FF06460020AB
:10C2A000FDF705FFF6B2002E03D0022E0FD007D304
:10C2B00013E002216846FFF783FDBDF900400CE062
:10C2C00003216846FFF77CFDBDF9004005E004212D
:10C2D0006846FFF775FDBDF90040002D04D02146EA
:10C2E0000020FDF7EAFE0446204602F0FDF9012099
:10C2F00002F01AFC80B203F03EF80120BDE876405F
:10C3000002F053B90FB480B5DFF8F00902A9242276
:10C31000FCF75CFE01BC5DF814FBDFF8E019242299
:10C32000FCF754BEDFF8801C02880A8082688A60AD
:10C33000427F4A77026A0A622422FCF747BEDFF88E
:10C340005407DFF8641C2422FCF740BE7CB51021A2
:10C350006846FFF735FDBDF9006007216846FFF725
:10C360002FFDBDF8004009216846FFF729FDBDF803
:10C370000050002E02D00120FFF7D8FCE4B2204686
:10C38000FCF7D6F8DFF8241CFCF7E0F8DFF8201CF7
:10C39000FCF7A2FCFCF774FBC0B2FBF735FFEDB273
:10C3A0002846FCF705FD03F0E7F8002821D003F04C
:10C3B000E3F8044603F0E0F805462046FCF7B8F839
:10C3C000DFF8F01BFCF7C2F80446284603F0E9F852
:10C3D000FCF7AEF801462046FCF77EFCDFF8D41BE4
:10C3E000FCF7B4F8FCF730F902460B460B20FFF7D8
:10C3F0007FFEBDE8734002F087B91FB5DFF8C44483
:10C40000617A02290AD0607201235022092168460C
:10C41000FCF74CFB207B40F0010020731FBDDFF8D0
:10C42000A814012806D10888401C08804868401CD0
:10C430004860704700200880486070472DE9FC4143
:10C440000C216846FFF7BCFC9DF8004007216846B8
:10C45000FFF7B6FCBDF90050ADB2DFF87C65B088DF
:10C460000146B42901DA401CB080707800280DD054
:10C47000002070702846FCF75BF8DFF82C1CFCF7F6
:10C4800065F8DFF82C1BFCF727FCB060307800283B
:10C4900033D00020B0803070B0702846FCF748F8E8
:10C4A0000746DFF80C8BDFF8001CFCF74FF801465D
:10C4B0004046FCF711FCB0603846DFF8F01AFCF794
:10C4C00045F801464046FCF707FCFCF7D9FAC0B234
:10C4D000FBF79AFE0C216846FFF772FC9DF80000FE
:10C4E00003280AD10020FDF7E2FD0120FFF71EFC22
:10C4F000002213460C20FFF7FBFDB07800285DD129
:10C50000002C17D0032C15D00020B08001207070B3
:10C510002846FCF70DF8DFF8941AFCF717F8DFF857
:10C52000901AFCF7D9FBFCF7ABFAC0B2BDE8F641B4
:10C53000FBF76ABEB0885A281FDB2846FBF7F8FFD6
:10C54000DFF8641BFCF702F8DFF8641AFCF7C4FBA1
:10C55000DFF8D01BFBF7FAFF0146B06803F06EF975
:10C5600003D803F07DF9B06001E00020B060B0684E
:10C57000FCF786FA00B2FBF747FEB088B4281DDB53
:10C5800001216846FFF71CFCBDF9000040F2F511DF
:10C59000884213DA0022DFF8903B0C20FFF7A8FD59
:10C5A000022002F002F80020FFF7C0FB0020FDF798
:10C5B0007EFD0020FBF728FE0120B070BDE8F3816E
:10C5C0001CB5044606216846FFF7FAFBBDF90000DA
:10C5D00080B2012C1CD100281DD0BD490A88521CF4
:10C5E0000A8092B2C0EB0013B2EB830F13DB002082
:10C5F0000880024603460C20FFF77AFD0022DFF890
:10C600002C3B0D20FFF774FD0220BDE81640F4E638
:10C610000020AF49088013BD2DE9F0414FF47A7531
:10C620002E46012003F096F9DFF8047B01203860E4
:10C63000022003F034FA052003F0F7FA0446002044
:10C640003860022003F02BFA052003F0EEFA0746CB
:10C65000002003F07FF9DFF88883B4F57A6F1FDAE2
:10C660002046FBF765FF05463846FBF761FF0146AC
:10C67000284603F0F5F80546C4F580543C192046D9
:10C68000FCF718FB01462846FBF760FFDFF824198A
:10C69000FCF722FBFCF7F4F90646A8F8006001E07D
:10C6A000A8F80050304680B2BDE8F081FEB50446DF
:10C6B0000D46164601F0B3FE02282CD101F0CAFE49
:10C6C000002828D101F0C1FEDFF8687AF97A00F07D
:10C6D000EBFAF872022807D101203070FFF79CFFB7
:10C6E000022001F062FF16E03078002803D0FFF747
:10C6F00093FF0020307002F0B6F9DFF8B018FCF7B5
:10C70000EBFAFCF7BDF900B2FCF7C2FA02460B46A1
:10C710000120FFF7EDFC002C25D1002D23D0DFF800
:10C72000144AE08B022803D1022001F03EFF13E0FF
:10C73000002811D101F089FE33280DDB0221684663
:10C74000FFF73EFBBDF9000001F0CEFF207A002884
:10C7500002D0012001F029FFE08B411CE1830E286B
:10C7600001DB0020E083F7BD10B40146002200E0A9
:10C77000521C1046C0B2072809DADFF8BC3903EBB7
:10C7800000100B464489A342F2D110BC70470FF64B
:10C79000D410FAE71FB5DFF89C49607A002849D029
:10C7A00002281CD04BD2607B00280BD10120FFF760
:10C7B000B5FA0123962209216846FCF777F9012092
:10C7C00060731FBD01283AD10020FFF7A7FA0020AF
:10C7D00060726073207B00F0FE0020731FBD607BE1
:10C7E00000280ED1A07B401CA0730120FFF796FA11
:10C7F0000123962209216846FCF758F9012060734D
:10C800001FBD01281BD10020FFF788FA00206073AC
:10C81000A07B042807DB0020A0736072207B00F05F
:10C82000FE0020731FBD0123322209216846FCF758
:10C830003DF91FBD0020FFF771FA0020A0731FBD56
:10C840001CB501216846FFF7BBFABDF900400D2178
:10C850006846FFF7B5FA0098DFF8D818002824D109
:10C86000C87A012802D00020887213BDB4F5FA7F7F
:10C8700002DA0220887213BDA4F2FF1040F22112E6
:10C88000904202D20320887213BDA4F22B3040F2F2
:10C890008742904202D20420887213BD40F2EF70AA
:10C8A00084420DDB0120887213BDC87B401E80418D
:10C8B000C00FC873C87B401E8041C043C00F887240
:10C8C00013BD000074050020BC320020500700207A
:10C8D0000633002078320020FEB504460121684668
:10C8E000FFF76EFABDF90070FFF703FA002872D067
:10C8F0000120FFF791FB0600DFF840580FD02878A1
:10C900000146022903DC0026401C287011E00020AB
:10C910006870A87802280CD10020A87009E0687817
:10C920000146022903DC0126401C687001E000205A
:10C930002870A87801281ED1300002D1B7F5FA7FFF
:10C9400019DA03F0A9F8696801F21451884212D388
:10C950000D216846FFF734FA009F4FF08072DFF830
:10C96000E0370D20FFF7C4FB0220A870082F02D18A
:10C970000020FDF79CFBA87806432CD12046012817
:10C9800019D10120A8700020FDF782FB022001F0E0
:10C990000CFE002213460C20FFF7AAFB0022DFF852
:10C9A000A4370D20FFF7A4FB0220FFF726FD03F0BC
:10C9B00073F86860F7BD002C0DD10120A87000222B
:10C9C000DFF880370D20FFF793FB0220FFF715FDFE
:10C9D00003F062F86860F7BD680500201633002098
:10C9E000043300200120000838B5FF208DF8000036
:10C9F00003F052F80446DFF83C5701F02BFD8DF8A8
:10CA000000009DF80000002805D101F01EFDE97A24
:10CA100000F04AF9E87203F03FF804F5FA71814238
:10CA200003D39DF800000028E7D1FFF7F5FDFBF7E1
:10CA30007FFD044602F017F8DFF87015FCF74CF99B
:10CA4000FCF71EF805462DB2284640F6D86188420C
:10CA50001EDA2046DFF8F01603F008F918D202E0DB
:10CA6000142003F01CF8052000F0C8F8032805D0B6
:10CA70000228F5D1DFF8BC0600F035F82846FCF7AF
:10CA800007F902460B460120BDE83240FFF730BBF4
:10CA900031BD00005432002078320020F8B5044641
:10CAA0000D460026374602E0032002F0F8FF2A4632
:10CAB0002146384603F04BFBAA2806D12846874278
:10CAC00008D000262F46FFB200E0761C3046C0B2E8
:10CAD0000328E9DBAF4204D1F6B2032E01DA0020CD
:10CAE000F2BDFF20F2BD38B584B00446102269467D
:10CAF000002003F073FBDFF8542669462020FCF782
:10CB0000F0FA06216846FCF7A5FA6D46E988024668
:10CB100092B2914206D100996160A988218060801B
:10CB2000002012E0062102A8FCF794FABDF80E10CE
:10CB3000024692B2914207D1A9686160BDF80C101B
:10CB400021806080002000E0012005B030BD0000A1
:10CB5000480500201C533B7416B582B01046009067
:10CB60006C46BDF80800A08006216846FCF772FA02
:10CB7000E080DFF8D82569462020FCF788FA0821F4
:10CB80006846FFF78BFF04B010BD00001857E63F62
:10CB9000E2274A911CB5DFF89C45207B00281FD175
:10CBA0006846FFF7A0FF01001BD10198217CFF29F7
:10CBB00002D0401C606004E06168884201D2401CE1
:10CBC0006060A08B4FF6FF71884201D12088A0835E
:10CBD000D4E900010A4601460020FFF7BDFF00E04E
:10CBE0000120207416BDDFF84C05007B002801D120
:10CBF00003F02BB900207047DEECEB3F3EB5054655
:10CC0000DFF83045207E00280BD1607C401C60742A
:10CC1000C0B203F0BFF8607C022827D10120207643
:10CC200024E0012822D1FFF7DEFF01280AD10220EB
:10CC3000207600206083012332220C216846FBF716
:10CC400035FF11E0608B401C60830021217680B2AB
:10CC5000854209D2084660830320207601233222D0
:10CC60000C216846FBF722FF00206074207E3EBD49
:10CC700010B4002101E0491CC9B2072911DADFF81C
:10CC8000B82402EB0112B2F90C300446A342F2DAE6
:10CC90000346B2F90E40A342EDDAB2F90A0010BC25
:10CCA00070474FF0FF30FAE7DFF8A424322808DBA2
:10CCB00010780346022B01DC401C107000205070DD
:10CCC00007E00020107050780346022B01DC401C66
:10CCD000507010780346022B02DD0123937004E0AC
:10CCE0005378022B01DD02239370002903D1002821
:10CCF00001D00120907090787047000054320020DD
:10CD00002DE9FF470C216846FFF75AF89DF80040CF
:10CD100010216846FFF754F8BDF900901FFA89F911
:10CD20000D216846FFF74CF8DDF80080002517E07C
:10CD3000DFF80074B8F1000F05D1F87A012802D1AC
:10CD40005020FFF75BFF387E022805D13846FFF7F9
:10CD5000CAFE01E0FFF71EFD3046FBF75FFF6D1CCA
:10CD60000A2D80F21E810FF23440465D314668463E
:10CD7000FBF73FFF9DF801000028F0D030460C285B
:10CD8000EAD8DFE800F06568D22E6107070A0709D4
:10CD9000070D0800E0E7CBE7DCE7FFF751FDDBE735
:10CDA000DFF89003C07A0128D6D1FEF7CBFF074603
:10CDB00001F059FE01467D48FBF78EFFFBF760FE50
:10CDC00000B2014640F6D9629142C5DAB7F5487F14
:10CDD000C2DAFBF75DFF02460B460120FFF788F938
:10CDE000BAE7FBF72CFDFFF729FB2046FFF7E8FB2E
:10CDF0002046FFF714FBCF4F387E022815D120467E
:10CE0000012812D1788C401C788480B23C2803DB46
:10CE10000120B87400207884B87C002805D0FFF782
:10CE2000B9FE002801D10020B874B8F1000F93D0EA
:10CE3000388C401C388480B203288DDB0020388475
:10CE40000220FFF7DAFA87E72046FFF745FD83E780
:10CE5000FDF75BFB80E720007FF47EAFB54FB9F1B3
:10CE6000000F0AD101F0F6FA00280DD101F0EDFA19
:10CE7000F97AFFF719FFF87206E007F12402494634
:10CE800009B20020FFF712FCF87A397D814202D006
:10CE900038750121F974022820D1F87C00283FF46C
:10CEA0005BAF0020F87401F0C3FA4FF6FF7A5346E7
:10CEB000672201216846FBF7F9FDA7F81CA0A7F837
:10CEC00000A000207860032038760022A14B0D20BE
:10CED000FFF70EF90220FFF790FA3DE701287FF4F3
:10CEE0003BAFF87C00283FF437AF0020F8744FF6D2
:10CEF000FF7A5346CB2201216846FBF7D7FD534604
:10CF000040F283120B216846FBF7D0FD00203876F3
:10CF1000534632220C216846FBF7C8FDFFF77CFB25
:10CF200000B2FFF7A5FEB88316E720007FF414AF28
:10CF3000FBF721FC0746FCF703F902460B460020ED
:10CF4000FFF7D6F80B216846FEF73AFF00984FF03E
:10CF50007E5102F08BFEBFF4FFAE42F211708742A9
:10CF6000FFF6FAAE01F071FA82463846FBF7E0FAB6
:10CF70000146FBF7B1FE7849FBF7E8FA0746504651
:10CF8000FBF798FE01463846FBF7E0FA0749FBF746
:10CF9000DDFAFBF759FB02460B460B20FFF7A8F81A
:10CFA000DAE6BDE8FF8700009C0500200000204174
:10CFB00000007F4300007A443EB50546080001D0DA
:10CFC0006648417008216846FBF713FE9DF8010092
:10CFD000002867D0002000E0401C0146C9B211299A
:10CFE00003D2012484402C40F6D05C4D2878401EAA
:10CFF0008041C00F28702878002839D00020FDF724
:10D0000056F82046012824D0042817D0082802D03A
:10D01000102825D02FE000200290022001900090DF
:10D0200010231A4600210820FBF749FA5FF000039D
:10D030004EA219461820FBF726FA1CE05FF0000309
:10D040004DA219460420FBF71EFA022001F0ADFAAA
:10D0500011E000234BA219461020FBF714FA0AE056
:10D060005FF000034AA219461020FBF70CFA02E019
:10D070000020FDF71CF8687800280ED000206870AA
:10D080002870FDF714F844F000442046FCF758F8E7
:10D0900002460B460D20FFF72BF80820BDE83E4066
:10D0A000FBF7BCBD37BD0000000010417CB50C2172
:10D0B0006846FEF785FE9DF800500D216846FEF794
:10D0C0007FFE009C01F0A1F80646254801782A461B
:10D0D000914203D005702846FFF7C6F8FFF710FE0F
:10D0E000002C1AD10C216846FEF76AFE9DF800005C
:10D0F000002803D002280BD005D373BD3046BDE80D
:10D100007640FEF799BB3046BDE87640FEF7B4B8EE
:10D110003046BDE87640FDF7D1BA31462046BDE83D
:10D120007C4049E70000B442000008400000304065
:10D130008481224274050020284D0108C00500208A
:10D140000000E0410000204000004844BC500108BD
:10D15000F8320020000010400024744908330020F9
:10D1600051070020554E4B3F000000005741524EE2
:10D17000494E4721000000004E6F20686F74706CAC
:10D18000617465004C6F7720566F6C74000000006E
:10D1900054696D65204F75740000000000030401A0
:10D1A00002090A070B0C0000002003E0491C642957
:10D1B000FCDB401CB0F57A7F01DA0021F7E770470D
:10D1C00080B54FF41852DFF8C81CDFF8C80CFBF725
:10D1D000FDFE00221021DFF84C0DBDE80840FAF7F3
:10D1E00085BF10B4002208E0835C1C46613C1A2C09
:10D1F00001D2203B8354521C92B20B469A42F3DB7D
:10D2000010BC70472DE9FF4104460D46DFF8846CE1
:10D2100006F580674FF0000802E0203708F10108AA
:10D22000404680B2102824DA0B22394601A8FBF7C9
:10D23000BDFE0B2101A8FFF7D4FF0B22214601A858
:10D2400004F0C8F80028E8D1022207F11C012846A2
:10D25000FBF7ACFE022207F11A016846FBF7A6FEB7
:10D26000BDF8000006EB402000F5007004B0BDE8FA
:10D27000F0810020FAE70146202903D00D2901D0D2
:10D280000A2801D1012070470020704730380A2851
:10D290008041C00F7047F8B5044600E0641C207858
:10D2A000FFF7E9FF0028F9D114F8015B2E462D2D78
:10D2B00001D02B2D01D114F8015B002707E007EB0B
:10D2C000870005EB4005303D2F4614F8015B2846EA
:10D2D000FFF7DCFF0028F2D12D2E02D17F42384625
:10D2E000F2BD3846F2BD30B40023154604E011F813
:10D2F000014B00F8014B5B1C1C46A4B2AC42F6D3B8
:10D3000030BC7047F0B403460024174608E01046CE
:10D31000401E2546ADB2A84201D05B1C491C641CCE
:10D3200008781D782646B6B2BE4201D28542EED0BC
:10D33000281AC0B2F0BC7047F0B402460020034681
:10D340001468054608E0012300EB8007304600EB37
:10D3500047003038641C6D1C2E460F46B6B2BE42E4
:10D360000AD22678A6F130070A2FECD31E46012EEA
:10D37000F0D11460F0BC70474FF0FF30FAE72DE9B0
:10D38000F04104460D461646284604F057F8074675
:10D390004FF0000802E0641C08F10108B0450BD210
:10D3A0003A4692B221462846FFF7ACFF0028F2D158
:10D3B000BFB2E019BDE8F0810020FBE770B504467C
:10D3C00004F03CF880B2002820D02044451E00E044
:10D3D0006D1EA54204D32878FFF74DFF0028F7D132
:10D3E00000206870264600E0761C3078002803D0C4
:10D3F000FFF741FF0028F7D1B44207D0AD1BAD1CA9
:10D400002A4692B231462046FFF76DFF204670BD96
:10D4100030B410F8013BA3F141041A2C00D22033A0
:10D4200011F8014BA4F141051A2D00D22034521EEF
:10D430001546ADB2002D01D0A342EAD01B1B92B21B
:10D440001A43104630BC70472DE9F0410746884624
:10D450003D2107F5C87004F00DF8002833D0401CBA
:10D46000FFF719FF0446A4B2002C01D0012C2AD1E9
:10D47000A8F81440002510E0022D0CD106EB860020
:10D480004000A8F8120006E0012DF5D106EB860059
:10D490004000A8F810006D1CADB2022D31DC3D211A
:10D4A00032206843384403F0E5FF00280BD0401CCD
:10D4B000FFF7F1FE0646B6B2002C06D130466438BE
:10D4C00080B2FB2815D300206FE04FF47A71012061
:10D4D000FCF7F3FD0A2190FBF1F08642F3DB40F606
:10D4E000AC510120FCF7E9FD0A2190FBF1F0B042BC
:10D4F000E9DB002DC8D106EB86004000A8F8040047
:10D50000C9E73D2107F1960003F0B4FF0028DAD007
:10D51000401CFFF7C0FE80B2002802D0411F7429D2
:10D52000D1D2A8F80E003D2107F1C80003F0A2FFF8
:10D530000028C8D0401CFFF7AEFE014689B20A2978
:10D54000C1DCA8F80C003D2107F1FA0003F092FFBE
:10D550000028B8D0401CFFF79EFE014689B2012981
:10D56000B1DCA8F81A003D2107F5967003F082FFA0
:10D570000028A8D0401CFFF78EFE014689B206297C
:10D58000A1DAA8F818003D2107F5AF7003F072FF8B
:10D59000002898D0401CFFF77EFE80B2002801D002
:10D5A000012890D1A8F816000120BDE8F0812DE9EE
:10D5B000F843ADF50C7D80460D46002427462246F3
:10D5C0004FF4E1711BA8FAF791FDDFF83C6B4FF4C3
:10D5D000007241463046FBF7E9FC2246242105A8AB
:10D5E000FAF784FD1DE008F101081FFA88F8B8F188
:10D5F000090F16DA06EB8800D0F80092484603F0CF
:10D600001DFF024692B249460EA8FFF701FF00280F
:10D61000E9D10EA91BA8322202FB08F8404403F00E
:10D6200035FFB7F5007F25DAA046224633210EA844
:10D63000FAF75CFD0EA903E008F101081FFA88F86B
:10D64000B8F1320FEDDAB7F5007FEADAF05D01F8F4
:10D6500008007F1C0A2801D00D28EDD1204601F8D2
:10D6600008000EA8FFF7AAFE9DF838000028D8D0C1
:10D67000A046BCE7214601E0491C89B2092906DA27
:10D680001BA832224A43805C0028F5D10124002CDB
:10D690005DD105A91BA8FFF7D7FE002800D1012402
:10D6A000002C54D105A984B068462422FBF78EFCD7
:10D6B0000FBCFEF727FEBDF918000A2190FBF1F21E
:10D6C0000FF678211BA803F016FFBDF924000A21EC
:10D6D00090FBF1F20FF674210DF19E0003F00BFFA9
:10D6E000BDF926000A2190FBF1F20FF6702134A853
:10D6F00003F001FFBDF822200FF670210DF58170B7
:10D7000003F0F9FEBDF820200FF670214DA803F0BC
:10D71000F2FEBDF82E200FF674210DF5B37003F064
:10D72000EAFEBDF82C200FF6702166A803F0E3FE98
:10D73000BDF82A200FF66C210DF5E57003F0DBFE35
:10D74000BDF828200FF66C217FA803F0D4FE00223C
:10D750004FF4C871284603F065FF002C13D0002653
:10D76000DFF8C077092E21DA07EB8600416C2846E6
:10D7700003F08BFF07F1140050F82610284603F041
:10D7800084FF761CEEE700260EE01BA832217143D1
:10D790000144284603F079FFDFF8700950F826109D
:10D7A000284603F072FF761C092EEEDB20460DF5AD
:10D7B0000D7DBDE8F0832DE9F043F5B00020ADF814
:10D7C000000002464FF4C87111A8FAF78FFC02213D
:10D7D00002A8FEF7F5FABDF908000A2190FBF1F264
:10D7E0000FF6581104A803F086FE04A911A803F04F
:10D7F0004CFFDFF83057696903F047FF032102A8A7
:10D80000FEF7DEFABDF908000A2190FBF1F20FF6EF
:10D810003C1104A803F06FFE04A911A803F035FF22
:10D82000A96903F032FF042102A8FEF7C9FABDF985
:10D8300008000A2190FBF1F20FF6201104A803F072
:10D840005AFE04A911A803F020FFE96903F01DFFA7
:10D85000062102A8FEF7B4FABDF908200FF60C1154
:10D8600004A803F048FE04A911A803F00EFF296ADA
:10D8700003F00BFF072102A8FEF7A2FABDF908206A
:10D880000FF6F80104A803F036FE04A911A803F06E
:10D89000FCFE696A03F0F9FE082102A8FEF790FA7F
:10D8A000BDF908200FF6E40104A803F024FE04A942
:10D8B00011A803F0EAFEA96A03F0E7FE092102A815
:10D8C000FEF77EFABDF908200FF6CC0104A803F09C
:10D8D00012FE04A911A803F0D8FEE96A03F0D5FEF0
:10D8E000102102A8FEF76CFABDF908200FF6B4016A
:10D8F00004A803F000FE04A911A803F0C6FE296BDA
:10D9000003F0C3FE0A2102A8FEF75AFABDF9082067
:10D910000FF6A00104A803F0EEFD04A911A803F07E
:10D92000B4FE696B03F0B1FE0FF694076A460DF181
:10D9300002013846FFF766FC0400DFF8586522D084
:10D9400011A803F07BFDBDF8001006EB411101F2B8
:10D950001C410870000A487006F58060201A00F526
:10D9600000700146491200EB9150801201212954A8
:10D9700011A803F063FD024611A92046FBF716FB30
:10D9800000F0D2FA5DE00FF644086A460DF102019C
:10D990004046FFF737FC0146DFF874474FF418594B
:10D9A00000291FD0FE2211A8FBF700FB00224946E8
:10D9B0003046FAF79BFB0C22414606F58860FBF7E0
:10D9C00005FBFE2211A906F52060FBF7FFFA0020F7
:10D9D00086F84B0406F25640046004210171FE21D2
:10D9E000817104E0002249463046FAF77FFB0C22A1
:10D9F000394606F58060FBF7E9FA0FF2FC7706225C
:10DA000039463046FBF7E2FA0622394606F5007041
:10DA1000FBF7DCFA11A803F011FD07463A4611A9FD
:10DA200006F5C060FBF7D2FA002086F80B0406F278
:10DA3000164004600221017187713F0AC77100F02E
:10DA4000A0FAE86B0021C17101724171A86BC1603D
:10DA50004161C1618161084675B0BDE8F0832DE97F
:10DA6000FF470C4600252E4600900A2102A8FEF72B
:10DA7000A7F9BDF90800002815D040F6AC510120E7
:10DA8000FCF71BFB80B20A2190FBF1FA1FFA8AFA1D
:10DA90004FF47A710120FCF710FB80B20A2190FB51
:10DAA000F1F7BFB202E04FF4AF7A6427A84606E070
:10DAB000A9F80600002508F101081FFA88F8B8F156
:10DAC000140F23DA0A216846FFF736FC10F1010F24
:10DAD0001CD082451AD3B84218D304EB8809A9F8A0
:10DAE00004000125761C1E228AA10098FFF747FC3E
:10DAF00000900028DFD00A216846FFF71DFC10F1D6
:10DB0000010F03D048F6A1418842D1D3002D03D0A4
:10DB1000002004EB8801C88026804046401E8041DA
:10DB2000C00F04B0BDE8F0873EB50020ADF804009A
:10DB300000F06EFC0546FAF78AFB01AA0DF106011A
:10DB40000FF29460FFF75EFB002817D04FF40072CD
:10DB50000FF29061FFF713FC009005216846FFF774
:10DB6000EBFB68804FF400720FF284610098FFF7BE
:10DB700006FC00902946FFF772FF04462046C0B21B
:10DB80003EBD2DE9F043E5B00020ADF800000FF2F6
:10DB900030666A460DF102013046FFF733FB0400A0
:10DBA000BC4D29D001A9FFF702FD002800F0A1809B
:10DBB00001A803F043FCBDF8001005EB411101F290
:10DBC0001C410870000A487005F58060201A00F5B5
:10DBD0000070D4490246521200EB9250801201228A
:10DBE0000A5401A803F02AFC024601A92046FBF7CB
:10DBF000DDF900F099F97CE00FF2D0546A460DF19E
:10DC000002012046FFF7FEFA01004FF4185721D019
:10DC1000FE2201A8FBF7CAF9002239462846FAF786
:10DC200065FA0C22214605F58860FBF7CFF9FE2244
:10DC300001A905F52060FBF7C9F9002085F84B0420
:10DC400005F25640DFF8C814016004210171FE217D
:10DC5000817104E0002239462846FAF747FA0C227F
:10DC6000314605F58060FBF7B1F90FF28C540C22B8
:10DC700021462846FBF7AAF90C22214605F500703B
:10DC8000FBF7A4F90024264605F5C06920E0A54865
:10DC900000EB8607D7F84480404603F0CFFB0246EE
:10DCA000414609EB0400FBF781F9404603F0C6FB4F
:10DCB00004197F69384603F0C1FB0246394609EB77
:10DCC0000400FBF773F9384603F0B8FB0419761C1F
:10DCD000092EDCD3002085F80B0405F21640DFF88E
:10DCE00030140160022101718471240AC47100F0B2
:10DCF00048F98C48C16B0022CA710A724A71806B64
:10DD00001146C1604161C1618161084665B0BDE8ED
:10DD1000F08300002C0000002DE9F841E9B0044632
:10DD20000E460025B6F5805F0FD15A4D4FF40072B4
:10DD3000294603F04FFB002800F0A4804FF4007246
:10DD400021462846FBF732F99CE0B6F5205F10D15A
:10DD5000DFF8C0534FF40072294603F03BFB002864
:10DD600000F090804FF4007221462846FBF71EF920
:10DD700088E0B6F5804F37D1DFF89C634FF400722E
:10DD8000314603F027FB00287CD04FF40072214677
:10DD90003046FBF70BF9634E012070702F4601E00F
:10DDA00020347F1C3846C0B2102811DA0C222146DC
:10DDB0006846FBF7FBF80B220FF20441684603F0BC
:10DDC00009FB0028ECD1A07E7082257F01203074F1
:10DDD000002D06D1307C012803D100203074308022
:10DDE00050E0012030704DE0A6F5004842F20100FD
:10DDF000804547D2274FB819A0F5F4454FF400727B
:10DE00002946204603F0E6FA002805D04FF40072B8
:10DE100021462846FBF7CAF8424C4FEA582808F139
:10DE20000208608A804527D105A92846FFF7BFFB75
:10DE3000002829D105A803F001FB618A07EB4111F5
:10DE400001F577710870000A487007F58060281A9C
:10DE500000F500700146491200EB9150801201213B
:10DE6000215405A803F0EAFA024605A92846FBF763
:10DE70009DF800F059F807E0601CA6F5FC46B60ACC
:10DE80000121815500F050F86AB0BDE8F081000032
:10DE9000009001085407002038B505460C46FFF7EE
:10DEA00083F94FF40071002C06D10A469B4928469D
:10DEB000BDE83840FBF77AB8B4F5805F06D10A4672
:10DEC00097492846BDE83840FBF770B8B4F5205FA5
:10DED00006D10A468F492846BDE83840FBF766B8A8
:10DEE000B4F5804F06D10A468B492846BDE8384034
:10DEF000FBF75CB8A4F5004042F2010290420AD25E
:10DF00000A4604F1006404F58B3421462846BDE836
:10DF10003840FBF74BB800222846BDE8384003F0F4
:10DF200081BB000040020020F8B503F0CFFB0024C5
:10DF30007C4900E0641C102C1FD2085D0028F9D039
:10DF400000200855784D15EB842003F04CFC7448F4
:10DF500010EB8426002700E0BF1CB7F5806F0CD2C1
:10DF600036F8021B17EB8420281803F02BFC04283A
:10DF7000F2D003F0B4FB0420F2BD03F0B0FB0020AC
:10DF8000F2BD38B5664C03F0A1FB002505E06648FC
:10DF900000EB852003F027FC6D1C092DF7DB002525
:10DFA00001E0AD1CADB2B5F5185F0BDA34F8021B19
:10DFB00005F1006000F5C83003F004FC0428F0D03F
:10DFC000042032BD03F08BFB002032BD10B5554C50
:10DFD000E36B1A78002A05D14002A0664902E16687
:10DFE000012018701878012833D1236CA06B806948
:10DFF00000280FD1A16E1846FFF74EFF4022C02126
:10E00000206C03F005FC4FF4E070A16B88614020A8
:10E0100020670CE04022C021206F184403F0F8FB79
:10E02000A06B816940398161206F403020674021B9
:10E03000012003F0CDFC3021012003F01FFCA06E75
:10E040004030A066E06E4038E0663848816840396C
:10E050008160E06E00280AD10020A16B88612067F2
:10E06000A0660320324908700020E16B087010BDE3
:10E0700070B52C4CA36BDD694035E66B3278002A15
:10E0800005D1400260674902A167012030703078F5
:10E09000012827D1002007E0264A125C266C725422
:10E0A000401CD969491CD961D969A942F4D3224DD0
:10E0B0002888616F41186167A26F101AA067C005B8
:10E0C00006D10020D861A1F50071206CFFF724FE75
:10E0D00016498A682888121A8A604FF44051022033
:10E0E00003F0E5FBA06F002803D011480078042856
:10E0F00008D10020A16BC861012103F0EFFD0020D1
:10E10000E16B087070BD0000BC02002054020020CA
:10E11000188DDD4054090020540B0020D84601081A
:10E12000540700204002002000900108883200209F
:10E13000203200204C3100202232002050727365C2
:10E140007454656D70313D25640000005072736534
:10E150007454656D70323D25640000005072736523
:10E160007454656D70333D2564000000536C656523
:10E170007054696D653D2564000000004261636B69
:10E180006C696768743D25640000000053686F7710
:10E19000547970653D256400566F6C756D653D253D
:10E1A000640000004C6F7743757272656E743D2594
:10E1B0006400000054656D70547970653D256400FD
:10E1C000434F4E4649472020545854004C4F474F28
:10E1D000494E2020424D500054454D504354524C1E
:10E1E000435356004379636C6554696D65732C0025
:10E1F00054696D6528532900F8FFFFFFFFFFFFFFFB
:10E20000FFFFFFFF7C49887070477C490878002237
:10E210000A7070477CB504460C216846FDF7D0FDB6
:10E220009DF800500D216846FDF7CAFD0098204674
:10E23000092810DA714E7078401E8041C00F70704E
:10E240000120FDF767FDFDF758FD0120FEF7D5F829
:10E25000032D00D0347073BD80B501210C20FBF775
:10E26000EDF94FF48060ADF8000048208DF8030010
:10E2700003208DF802006946614803F07BFD012010
:10E28000ADF8000069465F4803F074FD01BD10B4AD
:10E2900001460022104603460CE0D2B2824200D270
:10E2A00002461046002204E00C46DC40E407F4D4A9
:10E2B000521C5B1C1C46E4B2202CF5DBC90704D4BD
:10E2C000D2B2824200D202461046C0B210BC7047A1
:10E2D00070B5494D68684C49096841EA4001696078
:10E2E000A8684A49096841EA4001A96000241CE085
:10E2F000686810F1010F17D10420FFF78BFF4FF072
:10E30000FF30A86010E000280ED03079C0070BD590
:10E31000002CEDD1A86810F1010F05D10120FFF705
:10E3200079FF4FF0FF306860641C012C62DC05EB64
:10E3300084067068FFF7ABFF2855E87800280DD0F9
:10E34000287900F00100297A01F00101084205D086
:10E350000020E8704FF0FF306860A860287803283C
:10E3600013DB6878032810DB287900F00100297A94
:10E3700001F00101084208D00720FFF74BFF4FF0E2
:10E38000FF306860A86000202880285D01462029B1
:10E39000B9DBE8780028C7D1002C0ED128782028D6
:10E3A0000BDB6878062808DA0220FFF733FFA8782D
:10E3B0000028B9D10120E870B6E7012C0ED16878A9
:10E3C00020280BDB2878062808DA0520FFF722FF33
:10E3D000A8780028A8D10120E870A5E7287820288F
:10E3E00002DA687820289FDB0820FFF713FF01205E
:10E3F000E87099E770BD00003C050020FE32002067
:10E4000000080140000C0140280121420081214206
:10E41000DFF878097047DFF8780940797047DFF84E
:10E420007009C0787047DFF86809B0F92C007047B0
:10E4300010B5DFF85C4900220A2104F13C0003F02A
:10E44000F1F800202086A07110BDDFF84409B0F972
:10E450002E00704738B5DFF83849207801280AD1F6
:10E46000022020700120DFF82C19086001F014FB55
:10E47000E064012032BD022814D101F00DFBE16CF3
:10E480005A3188420CD303202070002001F0CDFBCC
:10E4900060860020DFF8FC18086001F0FDFAE064F7
:10E4A000022032BD03280BD101F0F6FAE16C0A31EB
:10E4B000884252D301202070002001F0B6FBA086D4
:10E4C000608EFAF735F80546A08EFAF731F8014666
:10E4D000284601F0C5F9DFF8C018FAF7FDFB4FF048
:10E4E0006651FAF7F9FBFAF7AFF8DFF8B028DFF872
:10E4F000B03803F0DDFCDFF8AC28DFF8AC3803F00F
:10E50000D7FCFAF79FFA00B2002800D500200028B7
:10E5100003DCB4F93610012905DC012806DDB4F965
:10E520003610002902DC0021A1712186218E04F120
:10E530003C020B4622F81300491C218689B20529AA
:10E5400003DB002020860120A0710021A079002893
:10E5500008461CD004F13C0305E0032032BD33F92A
:10E5600012205118401C0246D2B2052AF7DB09B22C
:10E57000052091FBF0F0E086E08EE08513E004F1E9
:10E580003C020346DBB232F913205118401C228EA4
:10E590000346DBB21546AB42F1D309B291FBF2F070
:10E5A000E085E08DE086002032BD012802D00228FF
:10E5B00009D07047DFF8D8070121C17000214170F0
:10E5C0000121017170470220DFF8C417C870A9E269
:10E5D000DFF8BC07807870471CB504460121684607
:10E5E000FDF7EEFBBDF900002146024602F10803EB
:10E5F0008B4203DB083A914200DB0446204616BDFD
:10E6000070B50546DFF88847A07803286BD8DFE8A7
:10E6100000F0021E60470020E07105F13200FAF7B9
:10E6200049FBA16801F022FB02D20120A07070BD5D
:10E63000323D2846FAF73EFB0146A06801F016FB82
:10E6400002D20220A07070BD0320A07070BDE079DE
:10E65000002810D12846FAF72DFB01460D46A16887
:10E66000DFF8480703F048FD294601F0FFFA3AD2E7
:10E670000120E07170BD012835D1A168DFF82C07B9
:10E6800003F03AFD01460E462846FAF713FB3146E1
:10E6900001F0ECFA27D20320A0700220E07170BDD7
:10E6A00005F13200FAF706FBA16801F0DFFA04D2A7
:10E6B0000120A0700020E07170BD1E3D2846FAF7D1
:10E6C000F9FA0146A06801F0D1FA0CD20220A0703C
:10E6D00070BD2846FAF7EEFA0146A06801F0AEF8E0
:10E6E00001D80320A07070BD0146B1F57A7F00DA31
:10E6F000704710B5DFF89846FAF7DCFAA060002002
:10E70000A0700120207110BDDFF884060021816017
:10E71000C16001614161816201834FF08241C16149
:10E72000DFF88C160162DFF88C1641627047DFF863
:10E730006006806870472DE9F843DFF85446E060D2
:10E740000546A068294601F08BF806462661DFF8E9
:10E75000681601F08BFA28D2DFF8601601F06EF827
:10E7600023D8A06AF9F770FF804689463046F9F74A
:10E770006BFFDFF84C26DFF84C36FAF7BDFD42465A
:10E780004B46FAF79DF8FBF741FCA062DFF838161C
:10E7900001F06CFA01D2A16207E0DFF8301601F057
:10E7A0004DF802D8DFF82806A0622079002810D0A2
:10E7B0000020A0622846A16801F058FA07D3A1689A
:10E7C00001F04EF84FF0804101F050FA01D20020E4
:10E7D0002071E0693146FAF77FFA05462565216A1E
:10E7E000A06AFAF779FA07466765D4F814803046CC
:10E7F000414601F035F8616AFAF76EFA8146C4F8CD
:10E8000058902846FAF73CF905463846FAF738F9A1
:10E8100045194846FAF734F945192583C4F8488064
:10E8200066612DB2002D02D50020208306E042F261
:10E830001170854202DB42F210702083B4F9180097
:10E84000BDE8F2832DE9F84303460D464FF0640C12
:10E8500028464008AE4600211C881646B44205D31F
:10E8600014469E1E36F81560B44209D20020BDE859
:10E87000F28386460A46101800EBD070401080B232
:10E880006246A2F1010C92B2002AEFD08542EDDB84
:10E8900033F8106032462746BA424CD203EB4002AE
:10E8A00032F8027C2246BE46724535D2F9F740FE68
:10E8B0004FF07C51FAF710FADFF8181503F01CFC42
:10E8C000F9F7C2FE804689462046F9F731FE044634
:10E8D0003046F9F72DFE0146204600F0C1FFF9F75A
:10E8E000B3FE0022DFF8F034FAF706FD04460D46C9
:10E8F000BE1B3046FAF7CCF902460B4620462946A5
:10E9000003F0D6FA02460B4640464946FAF7C6FDE2
:10E91000BDE8F443FBF77ABB9742AAD1401EFAF751
:10E92000C9F94FF07C51FAF7D7F9DFF8A814BDE820
:10E93000F44303F0E1BB22460ED003EB40014F88C5
:10E940003946914214D34AD001467246101800EB62
:10E95000D070401080B293E7F9F7EAFD4FF07C5198
:10E96000FAF7BAF9DFF86C14BDE8F44303F0C4BB5E
:10E97000401CFAF79FF94FF07C51FAF7ADF9DFF838
:10E98000541403F0B9FBF9F75FFE80468946204630
:10E99000F9F7CEFD04463846F9F7CAFD0146204690
:10E9A00000F05EFFF9F750FE0022DFF82C34FAF792
:10E9B000A3FC04460D46F61B3046FAF769F90246F9
:10E9C0000B462046294603F073FA02460B464046A2
:10E9D0004946FAF763FDBDE8F443FBF717BB401C5B
:10E9E000FAF768F94FF07C51FAF776F9DFF8E4139B
:10E9F000BDE8F44303F080BB38B50024254604E0AD
:10EA0000092001F012F904196D1C2846C0B2032830
:10EA1000F6DBDFF8C80321464FF6FF7289B2914258
:10EA200001D1048800E00480A4B2032094FBF0F03C
:10EA3000024692B24FF4A071DFF8A403BDE838405B
:10EA400000E738B50024254604E0022001F0EDF887
:10EA500004196D1C2846C0B20528F6DB0520B4FB5E
:10EA6000F0F080B232BD2DE9F84FFDF76BF90646A4
:10EA7000FFF7E7FF8146FFF7BFFF8046B6F57A7FD5
:10EA800002D1DFF860034BE0DFF85C73C7F8008069
:10EA90004FF4A55000FB09F0FAF7FAF8BF4AD34B40
:10EAA00003F006FA04460D46FBF7B0FAF9F7CCFD81
:10EAB00082468B460020CE4922462B46FAF7EEFCD2
:10EAC00004460D4606F596763046FAF7E1F82246FA
:10EAD0002B46FAF711FC0022C64B03F0E9F9024677
:10EAE0000B4650465946FAF7D9FCC34AC34BFAF7CE
:10EAF00003FC4FF03332C24BF9F7E2FE04460D46F9
:10EB00004046F9F7A1FD22462B46F9F7D9FEFBF75F
:10EB10007DFA04467C604846F9F70AFDB860204655
:10EB2000BDE8F28F00F014BC7CB505460C216846A8
:10EB3000FDF746F99DF8006000F0AEFF0446284658
:10EB4000F9F704FE012E1DD1AE4A1178012904D136
:10EB5000012151700021117051805178002910D08D
:10EB6000516832318C420CD35460518803460C46B4
:10EB7000641DA34202DB491D518002E00021517057
:10EB80005080508876BDB0F57A7F01DA5A2109E0CD
:10EB9000B0F5FA6F01DA5C2104E040F6B832904239
:10EBA00000DA5F2108467047FEB507460C2168462B
:10EBB000FDF706F99DF8005001216846FDF700F9C0
:10EBC000BDF90060724C6078032800F2C780DFE86E
:10EBD00000F0025C7492FAF777F9FFF744FF8A4974
:10EBE000FAF77AF8F9F74CFF6087B4F93A0041F286
:10EBF000941188420CDB0022844B0D20FDF778FA3B
:10EC00000220FDF7FAFB002213460C20FDF770FAF4
:10EC10003046FFF7F5FCB4F93A502846FAF74AF8BF
:10EC2000FFF789FDA0852846FFF7D6FC6087FAF735
:10EC30002FF802460B460120FDF75AFAB4F92C00D2
:10EC4000872801DD8720A085B4F92C00002815D085
:10EC50000020FFF769FF05465B2805DB2946B4F96C
:10EC60003A00FFF790FF0546280007D0012000F08A
:10EC70003DFB284600F07FFB00F057FBA08DF9F725
:10EC8000FFFD012020706070F7BDB4F92C0005284D
:10EC900010DB052F62DBF9F76EFD0646FAF750FA36
:10ECA00002460B460020FDF723FA012D02D1304623
:10ECB000F9F77EFD02206070F7BDB4F92C00B84270
:10ECC00007DA002000F012FBFFF72CFF0320607032
:10ECD000F7BD012D42D10020FFF726FF01465B283A
:10ECE00004DBB4F93A00FFF74EFF01460846BDE8E1
:10ECF000FE4000F040BBFFF796FB001DB8422DDA46
:10ED0000208F401C208780B2152825DB01206071F0
:10ED1000FFF7A0FB002821D1FFF797FB0546FCF782
:10ED2000D3FF01462846FDF7BFFF0546FCF7D0FF9D
:10ED3000022D0CD10022354B0D20FDF7D9F9022010
:10ED4000FDF75BFB002213460C20FDF7D1F90020F4
:10ED5000607120876070F7BD00206070F7BD10B54E
:10ED6000FFF75DFB0446FFF756FB012C0DD1002891
:10ED70000BD1274801784A1E9241D243D20F254B2E
:10ED80001A60491E8941C90F017010BDF83000207A
:10ED9000E00400209001214200404E479A99999941
:10EDA00099797840CDCCCCCCCCCCDC3F0000A040D5
:10EDB0008FC2F53C00006040010016430000C8C24D
:10EDC0007B14AE47E17A943F000048C301004843FA
:10EDD00000004843000080BF0000E03FFC320020FC
:10EDE000E83F010800007A449832002099F9304148
:10EDF00000C8A94080842E413F355EBA494C384056
:10EE00003333F73FA43200200000204100001040BF
:10EE1000133300208C0121422DE9F04D04460D46AC
:10EE20009046DFF88003DFF8801322462B46FAF77E
:10EE300063FA0F4627F00041DFF87023DFF87033E4
:10EE400003F0CCF9064662D2DFF8683307F00041E0
:10EE50000B4300223946F9F733FDF9F7F3FD5FEA7A
:10EE6000000A51D0F9F714FF0022D34BFAF744FA05
:10EE700006460F464FF0A040D04932463B46FAF7CF
:10EE80003BFA02460B4620462946FAF707FB0446A2
:10EE90000D464FF0C040CA4932463B46FAF72CFABD
:10EEA00002460B4620462946FAF7F8FA04460D4674
:10EEB0004FF00050C34932463B46FAF71DFA02466E
:10EEC0000B4620462946FAF7E9FA04460D4600208B
:10EED000BD4932463B46FAF70FFA02460B4620463A
:10EEE0002946FAF7DBFA04460D464FF00050B749C1
:10EEF00032463B46FAF700FA02460B4620462946C0
:10EF0000FAF7CCFA04460D460AF00300A7E06800C1
:10EF10004015401C0CD168004015401C02D129034B
:10EF200040F03C814FF0FF306FF00041BDE8F08DC4
:10EF300024F0000035F0004108BF002805D1B8F1E9
:10EF4000000F00F02B81A24D28E13946994B07F0C4
:10EF50000047304600223B43F9F7B2FC0F46490018
:10EF6000064641EAD0714000002908BF002817D0AA
:10EF700040F23342A2EB5150352804DB06F0000684
:10EF800007F000470CE0202803DD2038C740874009
:10EF900000E001D1002603E00028C4BFC64086403F
:10EFA00026F0000037F0004108BF002851D00020B3
:10EFB000814932463B46FAF79FF982468B464FF02D
:10EFC000A0407E4952465B46FAF796F902460B4648
:10EFD00020462946FAF762FA04460D464FF0C04033
:10EFE000774952465B46FAF787F902460B462046B8
:10EFF0002946FAF753FA04460D464FF0005071497E
:10F0000052465B46FAF778F902460B4620462946F7
:10F01000FAF744FA04460D4600206B4952465B4617
:10F02000FAF76AF902460B4620462946FAF736FAFD
:10F0300004460D464FF00050644952465B46FAF7CD
:10F040005BF902460B4620462946FAF727FA0446A2
:10F050000D4630463946F9F7F5FC00F0030025F07F
:10F0600000410029804405D500224FF00043101BC9
:10F0700063EB010100225FF0795304D54FF00047A4
:10F08000921A67EB0303994208F0010A05DABAF114
:10F09000000F7BD000244E4D78E022462B462046C0
:10F0A0002946FAF729F9BAF1000F06460F4631D082
:10F0B0004848494932463B46FAF71EF9474A484B09
:10F0C000F9F7FEFB32463B46FAF716F9454A464B3E
:10F0D000F9F7F6FB32463B46FAF70EF9434A444B42
:10F0E000F9F7EEFB32463B46FAF706F9414A424B46
:10F0F000F9F7E6FB32463B46FAF7FEF86FF05102AD
:10F100003E4BF9F7DDFB32463B46FAF7F5F80022B5
:10F110002F4B37E032463B4620462946FAF7ECF8BB
:10F1200082468B463648374932463B46FAF7E4F882
:10F13000354A364BF9F7C4FB32463B46FAF7DCF862
:10F14000334A344BF9F7BCFB32463B46FAF7D4F866
:10F15000314A324BF9F7B4FB32463B46FAF7CCF86A
:10F160002F4A304BF9F7ACFB32463B46FAF7C4F86E
:10F170002D4A2E4BF9F7A4FB52465B46FAF7BCF832
:10F1800022462B46F9F79CFB04460D465FEA887041
:10F1900004D585F000412046BDE8F08D2046294683
:10F1A000BDE8F08D83C8C96D305FE43F0000A0FF6B
:10F1B000FFFFDF410000E03F0000303EFB21B9418E
:10F1C000B410114026A6513E5C14D33C9A833B3BBD
:10F1D0000000F03F09260A1039BA213E3BA861C65B
:10F1E000F97D92BE63AC30909F01FA3EF6FB51165A
:10F1F0006CC156BFB10255555555A53FFFFFDFBF46
:10F20000B08F2FC310D8E53D8F0C73A1E1E55ABE36
:10F210004DADE44FE31DC73E3EE3B519A0012ABF43
:10F22000FAF010111111813F425555555555C5BF82
:10F230000122F1E5400D491840EA81200CD2490D28
:10F24000A1F58061491C40F0004005DBD1F11F01B0
:10F2500054BFC840C01770470020704738B588B009
:10F2600005460C4601210220FAF7F3F9012104209A
:10F27000FAF7E4F94020ADF8000004208DF803000F
:10F2800003208DF802006946424802F073FDADF894
:10F290000850ADF804400020ADF80A00ADF80600B3
:10F2A0003D4C01A92046FAF713FA6020ADF8100092
:10F2B0000120ADF812000020ADF81800ADF81600DE
:10F2C00004A92046FAF74CFA08212046FAF7BBFABF
:10F2D00001212046FAF792FA01212046FAF7A6FA10
:10F2E00001212046FAF77DFA09B030BD80B501460C
:10F2F000284800290CD00821ADF8001010218DF805
:10F30000031003218DF80210694602F033FD01BDA0
:10F310000821ADF8001004218DF8031003218DF8A9
:10F320000210694602F026FD01BD80B54020ADF80F
:10F33000000018208DF8030003208DF802006946B4
:10F34000144802F017FD01211348FAF757FA01BDDE
:10F3500080B500211048FAF751FA4020ADF80000BE
:10F3600004208DF8030003208DF802006946094847
:10F3700002F000FD01BD64280ADCC0EB0011480169
:10F38000642190FBF1F0014689B20348FAF762BAB2
:10F3900070470000000801400004004018B599B013
:10F3A0000CAA0221422000F083F90CAC6078E0281E
:10F3B00001D001207DE00DF102020221432000F086
:10F3C00077F9BDF80200C0F30231002907D00CAA7A
:10F3D000000B810001F01C01432000F069F90CA82A
:10F3E000BDF80210C1F3023100EB81020421432079
:10F3F00000F05EF90421072000F05FF9BDF802007B
:10F40000C0F30230010011D0ADF80000002007E089
:10F4100054F820106A4602EB80025160401CC0B2D2
:10F42000BDF80210C1F302318842F1DBBDF80200E1
:10F43000C0F302310A001DD100F00F02012A06D0EC
:10F44000032A09D0042A0CD0062A0FD012E0012288
:10F45000DFF8D4331A700DE00222DFF8CC331A70D3
:10F4600008E00322DFF8C0331A7003E00422DFF85B
:10F47000B8331A7000291BD000F00F00012817D1F3
:10F4800030226946DFF8A403F9F790FD0022DFF887
:10F49000A0330F20FCF72CFE00F06EF8044680B27B
:10F4A00000F07FF8014689B2204680B200F099F85A
:10F4B00000201AB010BDF0B585B0002214216846B6
:10F4C000F8F714FE12208DF80000684612214170F2
:10F4D000817013218DF80310D34CE1880A46120B7A
:10F4E000930003F01C039B1C43F08003037101F0A5
:10F4F000EF0343710B461B0A03F001030D466D0A2F
:10F500006D0005F00E052B43120102F070021A4344
:10F51000827107220023C1F3023704E0266B2E60BC
:10F52000121DD2B25B1C85181E46F6B2BE42F5DB38
:10F53000FF20287014206870FE20A8700F210B2077
:10F5400000F0BBF84021062000F0B7F84323222248
:10F55000E088C0F3023080000A300146C9B2684634
:10F5600002F08CFF0521062000F0A7F807210B20F0
:10F5700000F0A3F805B0F0BDAB498A8800E0521E48
:10F58000104640B201280ADB01EB800043681846B0
:10F59000800FF4D1C3F38920322148437047002003
:10F5A000704710B4002819D0002100E0491C9E4A81
:10F5B0000B46DBB29488A34210D20B46DBB202EBBF
:10F5C00083029268C2F38923322463438342EDD1DC
:10F5D000C2F3090202EB8200400000E0002010BCF0
:10F5E0007047F8B50246322392FBF3F60A460A2327
:10F5F00092FBF3F5ADB28C4CA288002A01D1022017
:10F60000F2BD00292FD0002801D10320F2BD002235
:10F61000042104F1300002F005F8012001E0401C53
:10F62000C0B2A18881421ADB04EB800253681A46FB
:10F63000C2F309029B0AC3F309033746BFB2BB42B8
:10F64000EDD1236B60F31E732363AA420BDB226BA5
:10F6500065F309022263226B65F3932222638142E0
:10F6600003DA0320F2BD0420F2BD0320216B60F316
:10F670001B61216361780846E28860F34B22E280D7
:10F680000120E28860F30E32E280E2884FF61060DB
:10F69000024042F04202E280491C01F00701617021
:10F6A000FFF709FF0020F2BD0146222002F074BEE0
:10F6B00003461046222202F092BE0A46014622204C
:10F6C00002F0C2BE38B50024254600F0B5F8224647
:10F6D0003021564801F0A6FF03210C20FFF7EDFF73
:10F6E000322000F0DCF903210C20FFF7E6FF0A20AE
:10F6F00000F0D5F90F210B20FFF7DFFF641EA441B6
:10F70000E40F08D003210220FFF7D7FF07210220D2
:10F71000FFF7D3FF07E003210220FFF7CEFF0B2105
:10F720000220FFF7CAFF012000F0B9F94020FFF7DF
:10F73000BBFF00F00F00022808DA6D1C284680B2DB
:10F7400040F22D118842D9DB012032BD072109206A
:10F75000FFF7B3FFEF210A20FFF7AFFFEF210E20E5
:10F76000FFF7ABFF01210F20FFF7A7FF002C1ED1F1
:10F770000B210220FFF7A1FF26210320FFF79DFFA9
:10F7800002210C20FFF799FF00210620FFF795FFCB
:10F790000F210B20FFF791FF3E20FFF785FF3F2051
:10F7A000FFF782FF4220FFF77FFF002032BD0721D5
:10F7B0000220FFF782FF25210320FFF77EFFDFE70E
:10F7C000F8B501210920F9F739FF48208DF8070025
:10F7D0002020ADF8040003208DF8060001A915488B
:10F7E00002F0C8FA0521012002F04BFB2020029014
:10F7F00001208DF80E0000208DF80C000C208DF8F3
:10F800000D0002A802F05CFE17208DF80000012018
:10F810008DF801008DF802008DF80300684601F0B4
:10F82000E4FC05B000BD0000CC310020D031002048
:10F830000000F03F000C0140C2E700004FF0807C68
:10F840001CEB400F94BF1CEB410F05E040EA010C9C
:10F850001CEB0C0F01D28142704718BF88427047E1
:10F8600090EA010F42F14E8481F00041421A3CBF00
:10F87000801A89184FF0004CC0F3C752FF2A24D0D9
:10F88000C1F3C75313B3D21AD2F1190327DD4CEADF
:10F8900001214CFA03F321EA0303D140C20D4CEAE3
:10F8A0000020401834BF20EA0C004CEA5000D2057A
:10F8B00053EA006373EB0C0C52EB1020420012F180
:10F8C000807F38BF7047C00DC0057047490212BF26
:10F8D0009A4200EB5120F8E7D2F11703D9D57047CF
:10F8E0006A494FF400620A614FF480520A610028AD
:10F8F00008680BD120F4404040F44050086008688C
:10F9000020F4402040F440300860704720F48040EC
:10F9100040F430400860086820F4802040F4302033
:10F920000860704780B501212120F9F787FE012189
:10F930004FF4004002F070FA0220ADF800000420FD
:10F940008DF8030003208DF802006946504802F04C
:10F9500011FA01BD80B501464D4800290CD00221A5
:10F96000ADF8001010218DF8031003218DF802105E
:10F97000694602F0FFF901BD0221ADF80010042133
:10F980008DF8031003218DF80210694602F0F2F998
:10F9900001BD1CB501210420F9F750FE1020ADF87F
:10F9A00000008DF8030003208DF80200394C6946F1
:10F9B000204602F0DFF91021204602F02BFA13BD99
:10F9C0001CB501210420F9F739FE0820ADF800002C
:10F9D00010208DF8030003208DF802002D4C69469D
:10F9E000204602F0C7F90821204602F013FA13BDA1
:10F9F00080B501210420F9F721FE8020ADF8000038
:10FA000010208DF8030003208DF80200694621487C
:10FA100002F0B0F901BD1CB50120F9F7FAFD012192
:10FA20004FF40000F9F715FE01210420F9F706FE56
:10FA300014208DF8040002208DF8050000208DF8B8
:10FA4000060001208DF8070001A801F0CEFB4FF45D
:10FA5000C050ADF8000003208DF8020018208DF88A
:10FA600003000C4C6946204602F084F94FF4C04074
:10FA7000ADF8000003208DF8020004208DF803008B
:10FA80006946204602F076F913BD000004080140E3
:10FA900000140140000801403E484068704710B51E
:10FAA0000446FFF7F9FF2418FFF7F6FF844204D35A
:10FAB000FFF7F2FFA042FBD310BDFFF7EDFF0B28CD
:10FAC000FBD2FFF7E9FFA042FBD310BD80B5F9F7E9
:10FAD00057FD102001F0F0FD012001F0E5FD0120AF
:10FAE000F9F767FD2120F9F7CAFD0028FAD00020B8
:10FAF000F9F779FD0020F9F784FD4FF48060F9F7FC
:10FB000079FD4FF420110020F9F756FD0120F9F797
:10FB10005BFD3920F9F7B3FD0028FAD00220F9F790
:10FB200056FDF9F75BFD0828FBD10120F9F771FDBF
:10FB300001214FF40000F9F78CFD01210520F9F7B0
:10FB400072FD012140F20C60F9F778FD01210320DC
:10FB5000BDE80440F9F77DBD80B501464FF0006077
:10FB600001F070FB4FF4A060BDE8024001F038BB2B
:10FB700080B508484168491C416001784A1C027000
:10FB8000142903DB00210170FEF7A2FBBDE8014050
:10FB9000F9F74EB8B432002010B586B0012140F21A
:10FBA0000C40F9F74BFD4FF48040F9F735FD272065
:10FBB000ADF8000000208DF803006946284802F0E7
:10FBC000D9F80220ADF8000000208DF80300694646
:10FBD000244802F0CFF8244C204602F0BBFC002061
:10FBE0000190ADF808004FF46020039000200490CD
:10FBF00001208DF8140001A9204602F0DAFC012151
:10FC0000204602F0F4FC204602F0FCFC204602F004
:10FC1000FEFC0028FAD1204602F0FEFC204602F04D
:10FC200000FD0028FAD106B010BD10B501460E4CFB
:10FC300007230122204602F004FD0121204602F0A4
:10FC4000F5FC0221204602F049FD0028F9D00221EE
:10FC5000204602F04AFD2046BDE8104002F030BDCB
:10FC600000080140000C0140002801404FF0807C5A
:10FC70001CEB400F94BF1CEB410F05E040EA010C68
:10FC80001CEB0C0F01D28842704718BF81427047AD
:10FC900081B041F21851484300900098411E0091F4
:10FCA0000028FAD101B07047F0B4024600200346A4
:10FCB00020E015782541454005F001054FF6FD7619
:10FCC000064000F0020080EA450080194BF6FF76FE
:10FCD000064000F4804080EA85373046381880B20C
:10FCE000400800EBC530641C2546EDB2082DE0DB72
:10FCF000521C5B1C1C46E4B20D46AC4201D20024EF
:10FD0000F2E7C04380B2F0BC7047B1490A8842F0C4
:10FD100001020A8000228A8403468A8C9A42FCD31C
:10FD20000A884FF6FE7002400A8070471CB5012118
:10FD30000420F9F783FCA74C4FF40071204602F031
:10FD400067F84FF40070ADF8000014208DF8030040
:10FD500003208DF802006946204602F00BF813BD1F
:10FD60001CB501210420F9F769FC9A4C4FF400718D
:10FD7000204602F04FF84FF40070ADF8000010205C
:10FD80008DF8030003208DF802006946204601F03B
:10FD9000F1FF13BD012802D0022801D07047DFE730
:10FDA000C4E71CB50020ADF800008B4C012020609A
:10FDB0001420FFF7AAFF0020206088480078002860
:10FDC00003D03220FFF7A1FF03E04FF4FF70FFF7ED
:10FDD0009CFF012020600220FFF797FF804C2068E5
:10FDE00000280ED0206800280BD00220FFF78DFFDE
:10FDF000BDF80000801CADF80000BDF80000FB2835
:10FE0000EDDBBDF80000FB2817DA0020ADF800009C
:10FE1000206801280BD00220FFF777FFBDF8000013
:10FE2000801CADF80000BDF80000FB28F0DBBDF839
:10FE30000000F02803DA012016BD002016BD0020C6
:10FE400016BD000080F31088704710B50120FFF741
:10FE5000F9FFFFF7A6FF04460020FFF7F3FF204657
:10FE600010BD10B55C4C002020600220FFF74DFF54
:10FE7000012020600320FFF748FF594804680A204A
:10FE8000FFF743FF2046C0B210BD10B5524C002012
:10FE900020600220FFF739FF012020600320FFF7D8
:10FEA00034FF4F4804683720FFF72FFF2046C0B2C9
:10FEB00010BD4A480078002800D0D2E7E5E738B501
:10FEC0000024082507E06408FFF7F3FF002801D0AD
:10FED00044F080046D1E2846C0B20028F3D12046AD
:10FEE00032BD38B504463C4D002028600220FFF7A3
:10FEF0000CFF2046401E8041C043C00F28600820F0
:10FF0000FFF703FF012028600520BDE83240FCE632
:10FF100038B50446304D002028600220FFF7F5FE7A
:10FF20002046401E8041C043C00F28603020FFF7AC
:10FF3000ECFE012028600A20BDE83240E5E62749B2
:10FF40000978002900D0CCE7E2E738B50446082557
:10FF500005E004F00100FFF7F2FF64086D1E28467B
:10FF6000C0B20028F5D131BD38B50446FFF719FFFE
:10FF7000050005D0CC20FFF7E8FF2046FFF7E5FF9E
:10FF8000284632BD38B50446FFF70BFF050005D003
:10FF9000CC20FFF7DAFF2046FFF7D7FF284632BD17
:10FFA00038B50446FFF7FDFE050005D0A520FFF794
:10FFB000CCFF2046FFF7C9FF284632BD0949097822
:10FFC000002900D1D0E7FF2900D1E9E7DAE70000F6
:10FFD000002C014000080140A4012142FB32002016
:10FFE00024012142123300202DE9F84384B08046D9
:10FFF0001446C146AA20FFF7E1FF060036D0FFF7FE
:020000040801F1
:100000005EFF0746FFF75BFF47EA0027FFF757FF52
:10001000002504E0FFF753FF09F8010B6D1C28468B
:10002000C0B20828F6DBFFF74AFF0546FFF747FF97
:1000300045EA002500220F216846F8F757F80B2201
:10004000414601A8F8F7B2FFAA208DF800006846E3
:1000500047703F0A87702046401E8DF80300241D1C
:10006000214689B26846FFF71FFE0746BFB2ADB210
:10007000AF4201D1022000E0304605B0BDE8F08378
:100080002DE9F84384B007460E461446B8460F20C3
:10009000FFF794FF002801D100203AE03046C0B2BB
:1000A000FFF753FF35462D0A2846FFF74EFF4FF066
:1000B000000905E018F8010BFFF747FF09F10109F6
:1000C0004846214680B28842F4D3FFF7F8FE8046C6
:1000D000FFF7F5FE48EA002800220F216846F8F7EE
:1000E00005F80C2239460DF10300F8F75FFF0F20E9
:1000F0008DF800008DF801608DF80250E41C214657
:1001000089B26846FFF7D0FD404501D1012000E0EB
:10011000002005B0BDE8F08338B504460D465520F3
:10012000FFF74CFF010011D02046C0B2FFF70DFFD2
:10013000240A2046FFF709FF681EC0B2FFF705FF3B
:100140000A20FFF7A5FDBDE83140B8E632BD2DE934
:10015000FC4104460D4616463619B6B24FF000086B
:1001600016E00822214689B26846FFF73DFF0746A0
:10017000022805D10821204680B2FFF7CDFF0746AF
:100180000A20FFF78CFC08F108081FFA88F80834E9
:10019000204680B2B0421DDA083086420CDAFF22D7
:1001A00008216846F7F7A2FF321BD2B205EB08011F
:1001B0006846F8F7FBFE05E0082205EB08016846F3
:1001C000F8F7F4FE0822214689B26846FFF758FF87
:1001D0000700C6D13846C0B2BDE8F68170B5044606
:1001E0000D461646F020FFF7E9FE002813D0204602
:1001F000C0B2FFF7AAFE240A2046FFF7A6FE00249D
:1002000004E0FFF75CFE05F8010B641C2046314654
:1002100080B28842F5D370BD2DE9F14FB0B092465F
:1002200004910DF142013A9A2B9199464A700020AF
:100230000AE01AF8011B0498309A904700280490AD
:1002400000F0B6860D98401C0D909AF8000050B151
:100250002528EED1002100220791089209910A92E7
:100260000B910C9204E00D9800F0A4BE41F0010146
:100270001AF8010F2028F9D023280CD02B2804D0FD
:100280002D2805D0302809D00BE041F00201EFE71E
:1002900041F00401ECE741F00801E9E741F0100109
:1002A000E6E72A280FD1D9F8002052F8040BC9F844
:1002B000002000280F9003D540420F9041F0040128
:1002C0000AF1010A14E00F92DFF828380AE00F98CB
:1002D000984205DA00EB800402EB4402303A0F92B8
:1002E0000AF1010A9AF80020A2F130000A28EED3A0
:1002F0009AF800002E2803D04FF0FF320E9229E02A
:100300001AF8010F2A2809D1D9F8000050F8042B57
:10031000C9F800000E920AF1010A1BE02D280CBF5B
:100320000AF1010A002000220E92DFF8C8470BE014
:1003300040B90E9AA24205DA02EB820503EB4503AF
:10034000303B0E930AF1010A9AF80030A3F1300213
:100350000A2AEDD3ADF84010DFF89C07784400F589
:10036000F3609AF8001001F085F808B11AF8010B53
:100370008DF842009DF84200682805D19AF80000E7
:1003800068280CD1622106E06C2804BF9AF80000AE
:100390006C2804D171218DF842100AF1010A12A8CB
:1003A00006901AF801BBBBF125012CD01C3900F0D6
:1003B000D081091F022940F2CC81133900F0238536
:1003C000093900F0C681891E00F0B885491E00F089
:1003D0006585491E022940F2BC81091F00F05E8537
:1003E000491F00F02881491E00F00D85491E00F0CC
:1003F000D080C91E0DD0891E00F00585C91E00F0F1
:10040000028500F0A6BD25238DF84830012100F0BB
:10041000ABBDD9F8000050F8044BC9F80000002C1F
:10042000059440F0A3802B994878002800F099802B
:100430004FF0FF340FF6843002F05AF9201A40F0E2
:10044000B78500F092BD6D1E40F0A9853096079DDE
:1004500012AF75B1309E17F8012B02A9304600F09B
:1004600073FE002801D46D1EF5D10028309640F0AF
:100470009F850A9D3020002D8DF804000CDD309EF4
:10048000012301AA02A9304600F06EFE002840F0C8
:100490008F856D1EF4D13096059F089D75B1309EF5
:1004A00017F8012B02A9304600F04EFE002801D4B7
:1004B0006D1EF5D10028309640F07A850B9D3020D6
:1004C000002D8DF804000CDD309E012301AA02A945
:1004D000304600F049FE002840F06A856D1EF4D1D8
:1004E000309605980899099D471875B1309E17F800
:1004F000012B02A9304600F027FE002801D46D1E12
:10050000F5D10028309640F053850C9D3020002D09
:100510008DF804000CDD309E012301AA02A93046AB
:1005200000F022FE002840F043856D1EF4D1309685
:100530009DF8400041077FF588AE2020002C8DF803
:1005400004007FF782AE309D012301AA02A928464C
:1005500000F00AFE002840F02B85641EF4D130958F
:1005600073E60FF66440059000F0FFBC0E9D002D71
:1005700004D5204600F062FF044607E02A462046E4
:1005800002F0D6F8002814BF041B2C46089400F093
:10059000ECBCD9F8001051F8040BC9F8001020F099
:1005A0000004002121F0FF3512ABCDE9024505938F
:1005B000DDE9022306993C2413B90AB90E9898B1D3
:1005C00002F00F053035641EEEB23A2EA8BF273573
:1005D000120942EA03721B090D5508BF002A03D015
:1005E00005980D19A842EBD308190590C4F13C02F7
:1005F0000E98089282420ADABDF84010821A4FF62D
:10060000EF7001400A92ADF8401000F0AEBC002837
:1006100040F1AB849DF8400000F01400102840F039
:10062000A4840F9B07990A985B1A1B1A9A1A002A2E
:1006300040F39B84E5E32B99487820B14FF0FF34D9
:100640000FF65430F8E69DF84200622861D0682821
:1006500017D06A283FD06C2806D0712847D074285C
:100660002CD07A281DD064E0D9F8001051F8040B82
:10067000C9F80010002868D14FF0FF340FF6303071
:10068000DAE6D9F8001051F8040BC9F8001020B9C7
:100690004FF0FF340FF61830CEE60D99018000F0D0
:1006A00064BCD9F8001051F8040BC9F800100028F8
:1006B0004BD14FF0FF340FF6F820BDE6D9F800100B
:1006C00051F8040BC9F8001000283ED14FF0FF3458
:1006D0000FF6DC20B0E6D9F8001051F8040BC9F889
:1006E000001080B94FF0FF340FF6C420A4E6D9F80B
:1006F000001051F8040BC9F8001020B94FF0FF3476
:100700000FF6AC2098E60D9AD317C0E9002300F04D
:100710002CBCD9F8001051F8040BC9F8001020B90E
:100720004FF0FF340FF6882086E60D99017000F037
:100730001CBCD9F8001051F8040BC9F8001020B9FE
:100740004FF0FF340FF6682076E60D99016000F057
:100750000CBCD9F80020D21D22F00702C9F80020F5
:10076000D2E900010832C9F80020CDE90201C80F22
:1007700002D007982D210AE0BDF84000810702D57C
:1007800007982B2103E0C00705D50798202112AA5E
:100790001154401C0790DDE90223079912A8CDE906
:1007A0002C2308444BF020016129059021AC0BD08B
:1007B0000E99002902D506210E9105E001BF4BF0EC
:1007C0002001672901220E92DDE902235900491513
:1007D000491C0DD11A030BD0ABF1610503211A2D71
:1007E000089102D20FF6E41110E00FF6E4110DE0CB
:1007F00059004915491C0DD11A030BD1ABF1610504
:1008000003211A2D089119D30FF6CC110322F8F702
:10081000CDFBAAE3DDE90201CDE92E01DDE92E23BE
:1008200023F00047B7F5801F22F000060DD200220A
:10083000002F08BF002E009203D116E00FF694118E
:10084000E4E76A4601F0A0FF0FE0DFF8DC08DFF81C
:10085000DC1800EB17500090DDE92E234FF0FF303D
:100860001940DFF8CC7810403943CDE902014BF054
:10087000200061280DD1059830210170821CBBF148
:10088000610F05920CBF7821582141700798801C98
:100890000790DDE9020120F0000231F0004308BFBB
:1008A000002A02D10026002568E14BF02008B8F1AB
:1008B000610F40F0B4800E98002847BF21210191BC
:1008C000401C0190019FDDE92C017F1C00220023C8
:1008D000DDE9024501F082FC00998DF8842038BFE3
:1008E00085F00045091F002F00910DF1850653DDAD
:1008F000204629460022002301F07EFF4CD248000A
:10090000400D00F11C0212D0002A10DD40F2FF73EE
:100910009A4206DBDFF81C1805F000400143002076
:1009200011E06FF31E5141EA025120460BE024F022
:10093000000035F0004108BF00280FBF29461C22E7
:10094000294601F071FF04460D46F8F77BF8FF1FBA
:10095000002F804609DDF8F79BF902460B4620463A
:100960002946F8F79BFD04460D46F01D0721B8F116
:10097000000F0CDD491E5EBF08F00F0200F8012DCC
:100980004FEA2818F3D502E0002200F8012D491E95
:10099000FAD5C61D002FABDC0DF18500361A019883
:1009A0008642D8BF304600280DF1850430D4B042CD
:1009B00006DA0DF185010A5C082AA8BF0F2100DACA
:1009C0000021024621AB134400E0401E13F80159F8
:1009D000521E8D42F9D00F2904D10DF185018B5C97
:1009E0005B1C8B54002A04D50099091D21AC401CC6
:1009F0000091411E0CD46218ABF13A0613783033E3
:100A0000DDB23A2DA8BFF318491E02F80139F5D519
:100A10000E99002940F1B080421E0E92ACE0009980
:100A2000DFF8142747F29750414391FBF2F2DDE9DA
:100A30002C45009225F00045D2F1070204DD204646
:100A4000294600F04EFB0BE052420020DFF8EC1686
:100A500000F047FB02460B462046294601F028FAE3
:100A60000446B8F1660F0E9806BF009F0A370627A6
:100A70003F18142FC8BF142730200D468DF884006E
:100A80000DF18506002F39DD20462946FEF7D2FB01
:100A900001460A4606F1080304200A26B2FBF6F6D0
:100AA00006EB860EA2EB4E02303203F8012C0A222E
:100AB000B6FBF2F202EB820EA6EB4E063036401E7B
:100AC00003F8026DE9D1083F002F03F10806D9DDD4
:100AD0000846F8F735FB02460B4620462946F8F74C
:100AE000DDFC0022DFF85836F8F706FC04460D4618
:100AF000CAE700BFCBCCCC0CB44600000DF185009A
:100B0000361A0DF1850404E00098401E761E009010
:100B1000641C20783028F7D0B8F1660F02D1009914
:100B2000491C04E0B8F1650F0CBF012100210E98AB
:100B300008188642B8BF701E00281DD4B04204DADF
:100B4000215C3429C8BF392100DC30210246631EF4
:100B50009D1800E0401E15F80169521E8E42F9D022
:100B6000392902D1A15C491CA154002A04D500995D
:100B7000491C1C46401C00910646009DF9F77AFA74
:100B8000406A0778DDF8388030B2002802DC0126A0
:100B90000FF248644BF02000662808BF6D1C16D089
:100BA000672846D128B210F1040F48DB404546DAE9
:100BB0009DF840006D1C010703D430B24045B8BF1A
:100BC000804628B2B8EB000848BF4FF000080FFA83
:100BD00085FBBBF1000F00F3B5800898411C08911C
:100BE000302205990A54B8F1000F03DC9DF840004B
:100BF000010704D50898411C089105990F5418EB7A
:100C00000B0FB8BFC8F100052DB268420B90A84485
:100C100032B29045B8BF4646059B089836B2099651
:100C2000324621461844F8F7C1F9A8EB06000C90AB
:100C3000D2E0BBF1610F17D14FF0700B19E030B269
:100C4000404504DA9DF840100A0758BF8046B8F1C5
:100C5000010848BF4FF00008BBF1670F14BF4FF009
:100C6000450B4FF0650B04E0BBF1410F08BF4FF09F
:100C7000500B0898411C0891B8F1000F059914F821
:100C8000012B0A5403DC9DF8400001071AD508988F
:100C9000411C0891B8F1000F05990F5412DD761E22
:100CA00030B280450598089BB8BF464632B221460F
:100CB0001844F8F77BF9089936B271180891A8EB37
:100CC00006000B9005980899084429B2002980F87D
:100CD00000B003D42B224270821C04E02D2242700B
:100CE0000D46821C6D4200212CAB28460AE00446CA
:100CF0000A2094FBF0F000EB8005A4EB450403F818
:100D0000014B491C00B20028F1DC012906DC4BF044
:100D10002000652804BF302002F8010B00292CAB0D
:100D200008D1302002F8010B06E0491E585C303033
:100D300002F8010B0029F8DC059908980844121AFA
:100D4000099249E030B229B288421CDA0598089B22
:100D500032B221461844F8F729F9089936B27118C9
:100D6000ABEB0606B8F1000F08910B9603DC9DF87B
:100D70004000020704D5059847540999491C099178
:100D8000CDF8308028E00598089B2AB22146184407
:100D9000F8F70CF90898761B5844B8F1000F089042
:100DA00003DC9DF840100A0703D5411C0891059902
:100DB0000F5430B280450598089BB8BF464632B202
:100DC00004EB0B011844F8F7F1F8089836B2301824
:100DD0000890A8EB06000B909DF8400000F014006E
:100DE000102840F0C280079A08990B988A18099930
:100DF00082180C988A1882180F98824280F2B58067
:100E0000821A0A92B1E09DF84200622808D0682850
:100E10000ED06A2814D06C281FD0712810D01CE086
:100E2000D9F8001051F8040BC9F80010C0B21AE04C
:100E3000D9F8001051F8040BC9F8001080B212E084
:100E4000D9F80020D21D22F00702C9F80020D2E90B
:100E500000010832C9F8002006E0D9F8001051F866
:100E6000040BC9F800100021CDE902019DF84000F3
:100E700001075AD5DDE90223002B08BF002A54D010
:100E80004BF02000782850D1079812A930220A543C
:100E9000401C431C079301F800B046E09DF8420057
:100EA000622808D068280ED06A2814D06C281FD079
:100EB000712810D01CE0D9F8001051F8040BC9F8C3
:100EC000001040B21AE0D9F8001051F8040BC9F82C
:100ED000001000B212E0D9F80020D21D22F0070263
:100EE000C9F80020D2E900010832C9F8002006E064
:100EF000D9F8001051F8040BC9F80010C117CDE95A
:100F00000201002902D507982D210AE0BDF8400012
:100F1000810702D507982B2103E0C00705D5079864
:100F2000202112AA1154401C079012A807990144CD
:100F3000059102A8594600F04FF816E001200790ED
:100F4000D9F8000050F8041BC9F800008DF84810CB
:100F50000BE025210122BBF1000F8DF8481007920C
:100F600003D08DF849B0022107910F9A07980A998A
:100F70000C9C121A0898521A0B99121A0998521AB4
:100F8000121A9DF84000141B41073FF560AA20206B
:100F9000002C8DF804007FF75AAA309E25460123C5
:100FA00001AA02A9304600F0DFF800283FF44BAA5E
:100FB0004FF0FF3031B0BDE8F08F00007072696E05
:100FC00074665F733A2062616420257320617267E2
:100FD000756D656E740000002DE9FC4307466F29AE
:100FE0003E6908BF082405D041F02000782814BFCE
:100FF0000A2410243C25D7E90023642918BF692955
:101000009046994605D1002B03D5D8F1000869EB2D
:101010004909B9F1000F08BFB8F1000F0CD1386BC6
:1010200050B9082C39D197F83800010735D5302050
:101030003B2586F83B0030E08DF8001040464946DD
:101040002246E31701F08EFC3032D0B26D1E3A28F2
:10105000019504DB9DF80000A0F151018A1872553A
:10106000404649462246E31701F07CFC80465FEA91
:10107000010908BFB8F1000F03D0F8687119884260
:10108000DCD3082C09D197F83800010705D5705D2D
:10109000302802D06D1E30207055C5F13C02BA6177
:1010A0007119F960386B824208DA821A3A624FF697
:1010B000EF70398F01403987BDE8F38300280ED5E2
:1010C00097F8380000F01400102808D17B6B79697C
:1010D000386A5B1A1B1A9A1A002AC8BF3A62BDE81E
:1010E000F3832DE9D04306460F4614464FF000081F
:1010F000DFF8509012E0E00707D542464B463046F5
:101100003946F8F7F9F806460F4640464946424642
:101110004B46F8F7F1F8641080468946002CEAD176
:1011200030463946BDE8D08302FCFFFFFFFF0F8049
:101130000000E03F0000F07FA08601000000F03FCB
:1011400084D797410000244010B503460C46114651
:10115000A0689847A06020B1E06A401CE0620020CF
:1011600010BD4FF0FF3010BDF8B505460E461746CE
:101170001C4600205CB117F8011BB068A847B0609E
:1011800030B1F06A401CF0620020641EF3D1F2BD61
:101190004FF0FF30F2BD00007072696E74665F73CD
:1011A0003A20256E20646973616C6C6F776564000A
:1011B0007072696E74663A2062616420256E2061E7
:1011C0007267756D656E7400000000006E616E00E0
:1011D0004E414E00696E6600494E460030000000E8
:1011E0001B4908431B490860704770B403781C46CC
:1011F0000122C17800291BD016490B6803F4E06373
:10120000C3F5E0631B0A4578C3F104018D40817882
:101210000F26DE4031400D432D010F490D55017859
:1012200001F01F0082400D48491140F8212007E0DD
:1012300003F01F0302FA03F30948641140F8243055
:1012400070BC7047074A114008430749086070475F
:101250000000FA050CED00E000E400E000E100E031
:1012600080E100E080FFFF1F08ED00E0002057490B
:1012700008604FF44D7000E0401E014689B200291D
:10128000FAD17047000240EA0140104317217DE087
:101290000123136000BF00BF00BF00BF00BF00BF3D
:1012A00000BF00BF00BF00BF00BF00BF00BF00BF46
:1012B0000023136000BF00BF00BF00BF00BF00BF1E
:1012C00000BF00BF00BF00BF00BF00BF00BF00BF26
:1012D00000BF00BF00BF00BF00BF00BF00BF00BF16
:1012E00000BF00BF00BF00BF00BF00BF00BF00BF06
:1012F00000BF00BF00BF00BF00BF00BF00BF00BFF6
:1013000000BF42E0314A0346CB40DB07C0D5012392
:10131000136000BF00BF00BF00BF00BF00BF00BF21
:1013200000BF00BF00BF00BF00BF00BF00BF00BFC5
:1013300000BF00BF00BF00BF00BF00BF00BF00BFB5
:1013400000BF00BF00BF00BF00BF00BF00BF00BFA5
:1013500000BF00BF00BF00BF00BF00BF00BF00BF95
:101360000023136000BF00BF00BF00BF00BF00BF6D
:1013700000BF00BF00BF00BF00BF00BF00BF00BF75
:1013800000BF00BF00BF00BF00BF491E0A4652B2E7
:10139000002AB7D56AE71CB501210420F8F74EF9F9
:1013A0004FF48070ADF8000010208DF8030003208A
:1013B0008DF80200064C6946204600F0DBFC4FF435
:1013C0008071204600F026FD13BD0000A0012142DF
:1013D000000801400300002013F0030F09D0521E43
:1013E00022BF13F8010B11F801CBB0EB0C00F3D0C6
:1013F000704711F0030F14D1121F22BF53F8040BD2
:1014000051F804CB6045F7D0121D0AD200BA9CFAFD
:101410008CFCB0EB0C0038BF6FF0000088BF0120DF
:101420007047521E22BF13F8010B11F801CBB0EB2D
:101430000C00F6D0521C08BF1046704700F10103A3
:10144000810704D010F8011B820781B1FAD102682C
:10145000A2F10131914311F0803104BF50F8042F03
:10146000F6E709BAB1FA81F100EBD100401CC01ACD
:1014700070470000C9B202788A421AB11CBF10F846
:10148000012FF9E718BF0020704700005FEA000C49
:1014900011F8012B00F8012B12B111F8012BF9E71B
:1014A0006046704730B40024002803D52D220A700E
:1014B000012440420A2290FBF2F3012205E00A25B2
:1014C00093FBF5F302EB82056A00002BF7D1002AAB
:1014D0000CD090FBF2F303F130050D55641C02FBB8
:1014E000130318460A2392FBF3F2F0E70020085595
:1014F000084630BC70470CB42DE9FC4104468846D0
:1015000000263746002C01D1304687E008AD2BE09D
:1015100018F80600E0557F1C25E0A0F57A7142F22C
:10152000283291421FD20A2190FBF1F10A2202FBDC
:10153000110030302071104691FBF0F002FB1011C9
:101540003031E1702E21A170114690FBF1F102FBC8
:10155000110030306070104691FBF0F002FB10116A
:10156000303121700527761C18F80600002852D06B
:101570002528CDD1761C18F80600632806D06428EB
:1015800013D066281FD0732805D0C1E755F8040B87
:10159000E0557F1CE7E755F8041B0022885C002813
:1015A000E1D0E055521C7F1CF8E755F8040B694662
:1015B000FFF778FF00216846405C0028D3D0E05553
:1015C000491C7F1CF7E755F8040B411E0929CAD3B3
:1015D000A0F10A015A29C6D3A0F16401B1F5617FD7
:1015E0009BD20A2190FBF1F10A2202FB110030305C
:1015F000E070104691FBF0F002FB10113031A17049
:101600002E216170114690FBF1F102FB1100303088
:1016100020700427A7E70020E0552046BDE8F6012A
:101620005DF80CFB62F30F2262F31F42401810F0CA
:10163000030308D0C91A1FD3DB0748BF00F8012DE8
:1016400028BF20F8022D130030B414461546103977
:1016500028BF20E93C00FAD8490728BF20E90C0040
:1016600048BF40F8042D890028BF20F8022D48BF4C
:1016700000F8012D30BC7047C91818BF00F8012DC3
:10168000CB0728BF00F8012D7047034600E05B1C24
:101690001A78002AFBD111F801CB83F800C013F8A7
:1016A000012B002AF7D17047DFF8DC100A6802F03E
:1016B0003802104308607047DFF8CC100A6822F047
:1016C00010020A600A68104308607047DFF8BC0027
:1016D000DFF8BC100160DFF8BC1001607047DFF874
:1016E000B800016841F080010160704738B50446D8
:1016F0004FF4302000F054F80146042913D1DFF8EC
:101700009850286840F0020028606C60286840F01B
:10171000400028604FF4302000F042F82A6841F67B
:10172000FD710A402A6032BD70B504460D464FF483
:10173000005000F035F8014604290ED1164E3068ED
:1017400040F00100306025804FF4005000F028F890
:10175000326841F6FE710A40326070BD0F49086080
:10176000704704200D490A68D20701D5012070474F
:101770000A68520701D5022070470968C90600D5DA
:1017800003207047000000000020024004200240B7
:1017900023016745AB89EFCD102002400C200240A9
:1017A00010B50446FFF7DDFF02E0FFF7DAFF641E25
:1017B0000146012901D1002CF7D1002C00D10520D0
:1017C00010BD000038B504460D461048FFF7E8FF8D
:1017D000052802D03420FFF7C1FF29462046BDE886
:1017E0003440FFF7A1BF10B50446A0050CD107484F
:1017F000FFF7D6FF052802D03420FFF7AFFF2046C1
:10180000BDE81040FFF772BF10BD0000A0860100C8
:1018100010B40F4B03EB4103521C521007E0017848
:10182000447841EA042123F8041B801C521EF6D19F
:1018300010BC7047064B03EB4103521C521004E0EE
:1018400053F8041B20F8021B521EF9D17047000008
:10185000006000404FF6F8710840DFF8E4110860BE
:10186000704710B4DFF8DC3153F8204048F68F128F
:101870001440214343F8201010BC704710B4DFF827
:10188000C43153F82040A4B248F6BF721440CA06CF
:1018900001D584F01004890601D584F0200444F4B5
:1018A000004444F0800443F8204010BC704710B45A
:1018B000DFF8903153F82040A4B24BF68F721440F9
:1018C000CA0401D584F48054890401D584F40054F9
:1018D00044F4004444F0800443F8204010BC7047B6
:1018E000DFF8602152F820304BF68F710B4083F403
:1018F000405343F4004343F0800342F820307047E4
:10190000DFF8402152F8203048F68F610B4043F455
:10191000004343F0800342F820307047DFF8242171
:1019200052F8201049040AD552F8203048F68F7139
:101930000B4043F4404343F0800342F820307047AB
:10194000DFF8002152F8201049060AD552F820305D
:1019500048F68F710B4043F4004343F0C00342F854
:1019600020307047DFF8D820126892B202EBC00234
:10197000DFF8D40000EB42004908490001607047DD
:10198000DFF8BC20126892B202EBC002DFF8BC00A4
:1019900000EB42004908490001607047DFF8A010E1
:1019A000096889B201EBC001DFF89C0000EB41003F
:1019B000006880B27047DFF88810096889B201EBCF
:1019C000C001DFF8880000EB4100006880B270477A
:1019D000DFF86C20126892B202EBC002DFF87000F0
:1019E00000EB420001607047DFF85420126892B2A9
:1019F00002EBC002DFF85C0000EB42000A463F2A1F
:101A00000ADB520911F01F0F00D1521E92B292024E
:101A100042F40042026070475208C90700D5521CC8
:101A200092B29202026070470549096889B201EBDF
:101A3000C001084800EB41000068C0F3090070478E
:101A4000505C0040005C00400060004008600040C6
:101A5000046000400C6000400146000AC9B240EA40
:101A600001207047AD4890F82010891E032900D945
:101A7000704780B5DFE801F00C150202002180F804
:101A800020104FF440510220BDE80440FFF70FBF83
:101A9000C17B282910D1816A406ABDE8044001F069
:101AA000C0B80121002000F019F94FF44051022084
:101AB000BDE80440FFF7FBBE01BD38B5974CE57BA0
:101AC0000220FFF7B1FF608402464FF48071944812
:101AD000FFF7B0FE94F82000002802D0012803D0C0
:101AE00016E0BDE831401FE02A2D05D1A16A606AE9
:101AF000BDE8344001F0C4B8012000F01BF92421F6
:101B0000052001F086F800210220BDE83440E5E020
:101B1000022000F00FF92421052001F07AF80021BD
:101B20000220BDE83440D9E010B500207B4C03E032
:101B30007B49095C2154401C618C0A469042F7D3D2
:101B4000784862684260A26882601F290DD0022036
:101B500000F0F0F8002020601A21052001F059F86B
:101B600000210120BDE81040B8E0E17B282901D028
:101B70002A290FD1607CA27C120442EA0062E07C38
:101B800042EA0022207D02436262A07DE27D42EAB9
:101B90000022A2622068644A90427AD163480068B9
:101BA000627B904204D3A07B002801D011280BDB7C
:101BB000022000F0BFF82421052001F02AF80021BE
:101BC0000120BDE8104089E000294AD003292CD02B
:101BD00008295AD00A2958D012292AD0152954D0B8
:101BE0001A292ED01B2928D01D294ED01E2924D0D9
:101BF00023292ED0252930D0282936D02A293AD099
:101C00002F293ED0552940D05A291ED088293CD0B2
:101C10008A293AD08F2938D09E2936D0A82934D0A5
:101C2000AA2932D0AF2930D033E0BDE8104000F00F
:101C3000E7BFBDE8104000F0ADBFBDE8104000F0C8
:101C4000ECBFBDE8104000F0D3BFBDE8104000F08D
:101C5000D3BFBDE8104000F0ACBFBDE8104000F0BD
:101C6000B7BFBDE8104001F054B8A16A606ABDE892
:101C7000104000F0D6BFA16A606ABDE8104000F0D5
:101C8000FFBFBDE8104001F029B8BDE8104001F0E9
:101C900044B8022000F04EF82021052000F0B9FFE2
:101CA00000210120BDE8104018E010B50C46224686
:101CB000C021FFF7ADFD21460120FFF789FE30214D
:101CC0000120FFF7DBFD0320144981F820001548AF
:101CD00081680C1B84600021017310BD10B50246A1
:101CE0000C4610481249016002730D22C021FFF713
:101CF0008FFD0D210120FFF76BFE0848052180F8BC
:101D00002010002C08D0042180F820103021012060
:101D1000BDE81040FFF7B2BD10BD0000003200204A
:101D20004C3100208832002055534243EC320020D1
:101D30005553425380B5002803D002280ED006D355
:101D400001BD10210120BDE80440FFF797BD4FF40D
:101D500080510220BDE80440FFF7A9BD10210120F9
:101D6000FFF78CFD4FF480510220BDE80440FFF7DF
:101D70009EBD0000F0B40024CA78134603F00F03A0
:101D8000D20601D58A7813430A88D2B2002A1AD023
:101D9000026815E0482D12D1066110E00126A64028
:101DA0000D883540B5420AD1A5000F27AF40BA4390
:101DB00003FA05F52A43CD78282DEBD14661641C42
:101DC000082CEBD302600A88B2F5807F1EDB4468E2
:101DD000002218E0012602F1080506FA05F50E8832
:101DE0002E40AE420ED196000F27B740BC4303FAF7
:101DF00006F63443CE78282E00D14561CE78482EA1
:101E000000D10561521C082AE4D34460F0BC70473D
:101E1000016170474161704770B4234A002801D5C1
:101E2000936900E01368C0F3034485B200F44016E0
:101E3000B6F5401F06D123F07063146824F0706477
:101E4000146010E0C60206D5032606FA04F4A34384
:101E500043F0706307E00446640D240105FA04F4BE
:101E6000A34343F07063002904D00146490D0901E2
:101E70008D402B43002801D5936100E0136070BCB6
:101E8000704730B48A0002F00C0221F00301074BC6
:101E90005C580F259540AC435C505C589040204303
:101EA000585030BC70470000040001400800014059
:101EB000F0B540F2FF7581EA030C0CF0004C15EA16
:101EC00011541DBF15EA1357AC42AF42E5E0BC41C7
:101ED000C1F31301C3F31303801A994143F4801330
:101EE00004D2641E4000494180185941C90241EAA8
:101EF0005051B1FBF3F603FB1611A2FB0675D7EBAD
:101F0000C020A94102D2761E80185941C90241EA77
:101F10005051B1FBF3FE03FB1E11A2FB0E75D7EB74
:101F2000C020A94103D2AEF1010E801859418902A7
:101F300041EA9051760546EA8E2EB1FBF3F603FB9B
:101F40001611A2FB0675D7EB8020A94102D2761E9E
:101F500080185941C90241EA50514EEA060EB1FBC0
:101F6000F3F603FB1611A2FB0675D7EBC020A941BF
:101F700002D2761E80185941C90241EA5051B1FB84
:101F8000F3F703FB1711A2FB0735D3EBC020A941E0
:101F900067F100070CBF004247F0010766F3D52741
:101FA0004FEA1E31B80814F5806412DDBD0775F1E3
:101FB000004250EB0E5051EB045111F5801F5CBFF5
:101FC00041EA0C01F0BD4CF07F6141F0E04100209E
:101FD000F0BDBD076D0840EA0E5041F48011D4F108
:101FE0000104B4F120060ADAC4F120060200E04040
:101FF00001FA06F3E1401843B24015430EE0342CD9
:1020000013DCC6F1200445EA40056D0820FA06F20B
:10201000154321FA06F0A1400D43002175F100425D
:1020200050F1000051EB0C01F0BD00205FEA0C0103
:10203000F0BDCFB992185B41B3FA83F704BFB2FA8F
:1020400082F6BF190B3FB7F120062FBF02FA06F345
:10205000BB40C7F1200622FA06F638BF3343BA4028
:102060001CB1E419641E33E77F4231F00041B1FA3C
:1020700081F404BFB0FA80F6A4190B3CB4F1200639
:102080002FBF00FA06F1A140C4F1200620FA06F69F
:1020900038BF3143A0403C1B1AE7AC421ABF05EAE7
:1020A0001357AF4212E050EA41061CBF52EA430602
:1020B000BFE750EA4107304661461CBF41EA05517F
:1020C000F0BD52EA430C08BFC143F0BD00204FF4FD
:1020D000001616EB410F98BF16EB430F08BF16EB27
:1020E000410F24BFC14305E016EB430F0CBF61460F
:1020F0004CEA0551F0BD000090EA010F7DF5B6AB4A
:1021000081F00041431A4FF000423EBF5340C01AD5
:10211000C91800BFD3095FEAD05C13EB400F34BF8E
:10212000B3EB410F40E07CEBD1530CD342EA0121E9
:1021300022D8D1EB402009D3400A28BF5FEA5001E2
:1021400040EBCC507047401A15D04002B0FA80F2F4
:10215000521C9040400A4FEA3C23B3EB026384BF19
:1021600000EB730007E040F400001A16DB07C2F131
:102170000102D04018437047182BFCDC31FA03F2FF
:1021800002FA03F3591A38BF42F00102D2EB4020A1
:102190003CBF4000ACF1010C5FEACC5CC20572F1BF
:1021A00000414CEB5020704713EB400F0FD2C94257
:1021B00009D0ACEBD153022B03DB4902172BDDDD39
:1021C00070479143401AC042D5D10020704713EBAD
:1021D000410FD0D36FF00000704700004FF4001C97
:1021E0001CEB410F94BF1CEB430F09E041EA030CC9
:1021F00050EA4C0C52EA0C0C03D2994208BF9042B0
:10220000704714BF8B4282427047000081B000903B
:102210000098411E00910028FAD101B0704780B5A6
:1022200001210820F7F70AFAC020ADF800001420B9
:102230008DF8030003208DF8020069465248FFF72D
:1022400099FD524801210160416001BD10B54F4C1C
:102250000120606020600520FFF7D8FF002060604B
:102260000520FFF7D3FF0020206010BD10B5474CBC
:102270000020206060600520FFF7C8FF012020607B
:102280000520FFF7C3FF0120606010BD38B50124B1
:1022900020463F4908600520FFF7B8FF3D4D2868FC
:1022A000002800D100240120E8670520FFF7AEFFD9
:1022B0000020E8670520FFF7A9FF204632BD10B5D2
:1022C000324C0020206060600520FFF79FFF012056
:1022D00020600520FFF79AFF0020206010BD10B598
:1022E0002A4C00202060012060600520FFF78EFF4F
:1022F000012020600520FFF789FF0020206010BD2D
:1023000070B50446214D0020286006460FE02046A7
:10231000C0B2C009686064000520FFF777FF0120A4
:1023200028600520FFF772FF00202860761C3046E9
:10233000C0B20828EBDB70BDF8B5044600250120CB
:10234000134908602E46134F0FE00020F867052060
:10235000FFF75CFF0120F8676D003868002800D0A7
:102360006D1C0520FFF752FF761C3046C0B20828CE
:10237000EBDB002C02D1FFF7B2FF01E0FFF79FFF7C
:102380002846C0B2F2BD0000000C014098812142F5
:102390009C8121421C81214238B504460D46FFF73D
:1023A00055FF64002046C0B2FFF7AAFFFFF76EFF9B
:1023B0002846FFF7A5FFFFF769FFFFF747FF44F047
:1023C00001042046C0B2FFF79BFFFFF75FFF00202C
:1023D000FFF7B2FF0446FFF749FF204632BDF8B5CC
:1023E00004460D4616461F46FFF730FF760030467E
:1023F000C0B2FFF785FFFFF749FF3846FFF780FFC0
:10240000FFF744FFFFF722FF46F001063046C0B257
:10241000FFF776FFFFF73AFF04E00120FFF78CFF9C
:1024200004F8010B2846451EC0B2002809D02846F2
:10243000C0B20028F1D10020FFF77EFF04F8010BA5
:10244000F0E7BDE8F14011E770B504460D461646C9
:10245000FFF7FCFE64002046C0B2FFF751FFFFF714
:1024600015FF2846FFF74CFFFFF710FF3046FFF738
:1024700047FFFFF70BFFBDE87040F7E6F8B50446ED
:102480000D4616461F46FFF7E1FE76003046C0B205
:10249000FFF736FFFFF7FAFE3846FFF731FFFFF789
:1024A000F5FE05E014F8010BFFF72AFFFFF7EEFE3B
:1024B0002846451EC0B20028F4D1BDE8F140D5E65B
:1024C00030B40468E443214A8179002926D01346B8
:1024D00019680C401C605C6801688C435C6004797E
:1024E0001419256801680D4325609C6801688C43B8
:1024F0009C60DC6801688C43DC60417904681029C9
:1025000007D199680C439C60D96800680143D96081
:1025100009E0521810680443146004E000791218AE
:1025200010680440146030BC704702460020074B1E
:10253000196811405B69134202D0002900D00120C4
:102540007047034908607047000000000004014024
:102550001404014080B55C4988420BD101214FF43D
:102560000070F7F781F800214FF40070BDE80440D7
:10257000F7F77AB8554988420BD101214FF48060B2
:10258000F7F772F800214FF48060BDE80440F7F7D8
:102590006BB84F4988420BD101214FF40040F7F747
:1025A00063F800214FF40040BDE80440F7F75CB841
:1025B00001BD4368474A13400A6813430A7943EA56
:1025C000022343608368444A1340CA6813438A68FD
:1025D00013434A7943EA42038360C26A22F47002D9
:1025E000097C491EC9B242EA0152C2627047002901
:1025F000816803D041F001018160704749084900BA
:1026000081607047816841F008018160704780688F
:10261000C00800F001007047816841F0040181604A
:1026200070478068800800F00100704700298168C9
:1026300003D041F4A0018160704721F4A0018160C2
:10264000704770B407240D460A2D0BDBC568A1F155
:102650000A0606EB4606B44025EA0404B3402343C9
:10266000C36008E0056901EB4106B44025EA0404B3
:10267000B3402343036113461F24072B09DA436B3E
:10268000521E02EB82029440A34391400B434363EA
:1026900014E00C2B09DC036BD21F02EB8202944086
:1026A000A34391400B43036308E0C36A0D3A02EB76
:1026B00082029440A34391400B43C36270BC7047B5
:1026C000C06C80B270470000002401400028014027
:1026D000003C0140FFFEF0FFFDF7F1FF0246002045
:1026E00012680A4200D001207047C9430160704758
:1026F00080B500B906A005490B681BB12222002154
:10270000984701E000F06AFB222002BDF43200206D
:10271000636F6E73747261696E742068616E646C4D
:1027200065723A20626164206D657373616765004C
:10273000C9B2830706D0521E22D310F8013B99423A
:10274000F7D11FE0083A13D302F1040241EA012154
:1027500041EA014150F8043B121F21BF4B40A3F155
:10276000013C2CEA030C1CF0803FF3D0C9B2001FDF
:10277000083210F8013B521E28BF91EA030FF8D827
:1027800018BF0120401E704710B5144600F002F833
:10279000226010BDC1F30A5343B14A0012F5001F75
:1027A00028D2A3F2FE32A1EB0251704750EA410C4D
:1027B00020D001F0004C31EA0C01B1FA81F204BFE3
:1027C000B0FA80F3D2180B3AB2F120032CBF00FA12
:1027D00003F1914041EA0C013EBFC2F1200C20FA06
:1027E0000CF319439040524240F2FD33D21A01EBF0
:1027F00003517047002270474FF4001C1CEB410F3F
:1028000094BF1CEB430F09E041EA030C50EA4C0C67
:1028100052EA0C0C03D28B4208BF8242704714BFAD
:102820009942904270470000124254D440F2FF7C1B
:102830001CEA11530FD0634531D09B1863453CBF50
:1028400001EB0251704701F0004141EA0C510020B8
:10285000AFF30080704750EA410320D001F0004CF4
:1028600091EA0C011CD0B1FA81F30B3B9A420DD9CD
:10287000D21A994051EA0C01C3F1200C20FA0CFC49
:1028800061449840531C40F2FF7CD7E7914041EAF5
:102890000C01C2F1200C20FA0CF319439040704750
:1028A000B0FA80F31533202BE0D3202AEED3203A60
:1028B000203B9A4209D9D21A00FA03F141EA0C01ED
:1028C0000020531C40F2FF7CB8E700FA02F141EA15
:1028D0000C0100207047524240F2FF7C1CEA115369
:1028E0000DD06345DBD0B2EB030C3CBFA1EB025132
:1028F00070470CF1010221EA035141F4801150EAC2
:10290000410CCCD001F0004C352A27DC30B481EAF0
:102910000C01B2F1200309DAC2F12003044601FAE6
:1029200003F5D0402843D1409C400CE0C3F1200285
:10293000450020FA03F418BF44F0010421FA03F023
:1029400091400C43002174F1004550F1000051EB1F
:102950000C01244230BC7FF47BAF704761460020FD
:1029600076E70000BBBBE1B1B2F5803F80F07E802E
:10297000022A1ED98C46B1FBF2F102FB11C31B04E3
:1029800043EA1043B3FBF2FC02FB1C3380B240EA83
:102990000343B3FBF2F002FB103240EA0C40002389
:1029A0007047022A05D98446B0FBF2F002FB10C240
:1029B00070474AB105D100F0010249085FEA3000D2
:1029C0007047002200237047F7F758BB0B00020046
:1029D000002100207047904271EB030CF6D3B3F551
:1029E000803F2FD2F0B5B3FA83F7B1FA81F4A7F1A3
:1029F0000F0E3D1B5340CEF1200602FA0EF2F341BA
:102A00005340B5F10F0746D80F3C2C444140C4F168
:102A10002006A040F1414140B1FBF3F603FB161143
:102A2000A2FB0645001BA94102D2761E801859411F
:102A300080EA010221FA0EF362FA0EF200215A40F6
:102A40003046F0BD30B4B1FBF3FC03FB1C11A2FB1C
:102A50000C45001BA94103D2ACF1010C801859416F
:102A600030BC02460B46604600217047B2F1807FC1
:102A700065D3F0B5B2FA82F7B1FA81F4C7F10F0667
:102A80003D1B22FA06F307F1110EF24120355A40A0
:102A9000B5F10F07B8D94140C4F12006A040F1417B
:102AA0004140B1FBF3FC03FB1C11A2FB0C45001BD6
:102AB000A94103D2BCF1010C801859410F2F12D348
:102AC0000F3FC90341EA5041B1FBF3F603FB161176
:102AD000A2FB0645D4EBC030A94102D2761E801875
:102AE000594146EACC3C07B34140C7F12006B84003
:102AF000F1414140B1FBF3F603FB1611A2FB064581
:102B0000001BA94102D2761E8018594180EA0102B9
:102B100021FA0EF3C7F1200462FA0EF20CFA07F064
:102B20005A402CFA04F13043F0BD80EA010221FA48
:102B30000EF3002162FA0EF260465A40F0BD8C4658
:102B4000B1FBF2F102FB11C31B0243EA1063B3FBBA
:102B5000F2FC02FB1C331B024CEA002043EA106328
:102B6000B3FBF2FC02FB1C331B024CEA002043EADD
:102B70001063B3FBF2FC02FB1C331B024CEA002087
:102B800043EA1063B3FBF2FC02FB1C324CEA002068
:102B9000002370478849087CC00702D58748052173
:102BA00005E08748C97C0A46252A00DB2421FFF777
:102BB0007CB8844800218180022181710021C1718B
:102BC0004172022181720021C1720C21FFF76DB8A0
:102BD0007D48002101800F218170FF21C1700021FB
:102BE0008180022181710021C1710821FFF75DB848
:102BF00004217648FFF759B808217548FFF755B802
:102C00006D48C17C0846132800DB12217148FFF78C
:102C10004CB8704A90701173704701210020FFF783
:102C20005DB870B504460D466B4E307800281FD154
:102C30002A462146282000F08DF800281FD05E4843
:102C4000007B000607D50220307029462046BDE8EB
:102C50007040FBF7BBB90220FFF76CF82421052078
:102C6000FFF7D7FF01210846BDE87040FFF736B8EF
:102C7000022804D12046BDE87040FBF7A7B970BD1B
:102C800010B50A46544C217800291FD101462A204C
:102C900000F060F8002820D04748007B000608D4E8
:102CA000012020704FF440510220BDE81040FEF793
:102CB000FEBD0020FFF73EF824210520FFF7A9FF05
:102CC00000210120BDE81040FFF708B8012904D118
:102CD0001146BDE81040FBF7CBB910BD80B53649B1
:102CE0008868002808D1087C400705D4012100200D
:102CF000BDE80440FEF7F2BF0220FFF71BF82421D5
:102D00000520FFF786FF00210120BDE80440FEF703
:102D1000E5BF01210020FEF7E1BF80B526498868A4
:102D2000002803D10020FFF705F809E0087B000622
:102D300003D50020FEF7FEFF02E00220FEF7FAFFB7
:102D400020210520FFF765FF00210120BDE8044098
:102D5000FEF7C4BF80B5511841F20103994211D367
:102D60002A2802D10220FEF7E5FF0020FEF7E2FF4D
:102D700021210520FFF74DFF00210120FEF7AEFFC6
:102D8000002002BD0C498968B1EB422F12D02A28DD
:102D900003D10220FEF7CEFF02E00020FEF7CAFFBB
:102DA00024210520FFF735FF00210120FEF796FFC3
:102DB000002002BD012002BD00320020D4320020DC
:102DC000544F010800070020DC320020E0060020FC
:102DD000E4060020EC06002020320020012000F054
:102DE00001B8000080B5AFF30080024A110018203E
:102DF000ABBEFBE72600020010B5DFF858480028FC
:102E000004D1012021680882002010BDDFF84808A5
:102E100000680068804720680A3010BD80B5DFF880
:102E200034080168CA78DFF83408407890420DD33E
:102E3000887800280AD18888002807D18A72DFF8AC
:102E40001808006840688047002002BD022002BDCB
:102E500010B5DFF80048002804D10120216808825D
:102E6000002010BDDFF8F007006880688047206808
:102E70000C3010BD10B5DFF8DC472068C178407910
:102E8000DFF8DC271268926990472268917A00295E
:102E900014D0002812D1107900280FD19078002882
:102EA0000CD1DFF8B4070068C0688047206841791A
:102EB000C1722068C1780173002010BD022010BDCE
:102EC00010B5DFF890170968002803D102200882A6
:102ED000002010BDDFF88C4700202080087810F01B
:102EE0007F0F19D1487A0021820603D541F00201F3
:102EF000217000E021702178400609D541F00101E0
:102F00002170DFF85407006800698047204610BD33
:102F100001F0FE012170F4E700F07F02012A01D1E7
:102F2000204610BD00F07F0002281BD14A7902F034
:102F30000F00DFF83417120651F8200008D500F012
:102F400030001028DDD1002040F001002070D8E7CB
:102F500000F44050B0F5805FD3D1002040F0010074
:102F60002070CEE7002010BDF8B5DFF8E806016854
:102F7000087810F07F0005D1487A00F0DF00487231
:102F80000020F2BD022859D14888002856D108797E
:102F9000002853D14879024622F08004DFF8C85651
:102FA000000655F8240002D500F0300001E000F4DE
:102FB0004050DFF8A8361B789C423FD200283DD015
:102FC000887A00283AD0100655F824000BD500F076
:102FD000300010282BD12046FEF7B2FC30212046CD
:102FE000FEF74CFC23E000F44050B0F5805F1ED1AA
:102FF00048F280064BF68F77002C0DD1DFF86C0677
:1030000090F82C100020FEF7EFFC2868074087F4AA
:1030100040573E432E600AE02046FEF77FFC55F8FD
:103020002400074087F440573E4345F82460DFF80A
:1030300028060068406980470020F2BD0220F2BDEA
:1030400038B5DFF8100604686079054625F080027F
:10305000DFF81436000653F8221002D501F03001D3
:1030600001E001F44051DFF8F4050078824207D214
:103070006088002804D1002902D0A07A002801D15C
:10308000022032BD48F28001280653F8224008D5BC
:1030900048F6BF70044084F01004214343F8221026
:1030A00007E04BF68F70044084F48054214343F8CA
:1030B0002210DFF8A405006880698047002032BD37
:1030C00080B5DFF890050068417A41F02001417237
:1030D000DFF884050068C0698047002002BDDFF882
:1030E00074251268538A002804D18888C31A138271
:1030F00000207047086818447047F8B5DFF8545549
:10310000286800F110063488B168002916D0002C18
:1031100014D0B088844200D9044620468847074628
:103120003088001B30807088201870800020FEF7E7
:1031300042FC224601463846FEF77CFB30880028D8
:103140000CD04FF44050DFF82815088000210846C5
:10315000FEF73EFC3020DFF81C1508803088B1886F
:10316000884203D3032029680872F1BD002803D0E8
:10317000052029680872F1BD10D10620296808725F
:103180000020DFF8F414096889B2DFF8F02402EBBC
:10319000410210603020DFF8DC140880F1BD2DE919
:1031A000F041DFF8B054286800F110073C88002C8B
:1031B0001DD1007A04281AD1DFF8B804DFF8C01452
:1031C0000A78012A0FD10022DFF8AC341B689BB2C9
:1031D000DFF8A84404EB4304226030220280042676
:1031E000002008702BE007261021018027E0B88816
:1031F000A04201D3042600E00226844200D90446FE
:103200002046B968884780460020FEF7C7FB224663
:1032100001464046FEF7FCFA21460020FEF7D8FBA7
:103220003888001B3880788824187C803020DFF8AC
:10323000441408804FF44050DFF8341408802868A4
:103240000672BDE8F08138B50220DFF80844226834
:103250005578117811F07F0F2DD1092D02D1FFF78C
:10326000DDFD3EE0052D0FD1D0787F2808DC907879
:10327000002805D19088002802D1907A002801D03A
:1032800008204EE000202CE0032D08D1D178012940
:1032900027D19188002924D1FFF712FF21E0012DC9
:1032A0001FD1D17801291CD19188002919D1517AD7
:1032B00089060FD415E001F07F02012A04D10B2DFD
:1032C0000FD1FFF7D7FD0CE001F07F01022908D1F3
:1032D000012D02D1FFF748FE03E0032D01D1FFF7D6
:1032E000AFFE01000AD02846DFF874130968496967
:1032F00088470146032901D1092012E0002801D0A6
:1033000008200EE006200021DFF86C23126892B23C
:10331000DFF8683303EB420319603021DFF85423F0
:1033200011802168087231BD38B5DFF82843226862
:103330005178002506291AD1107810F07F0F40F03F
:103340007F809078012804D1DFF814030068C569F4
:1033500076E0022804D1DFF808030068056A6FE010
:1033600003286DD1DFF8F8020068456A68E000299B
:1033700042D1508800283FD1D08802283CD1107912
:10338000002839D1117811F07F0F05D190880028DD
:1033900002D1DFF8F05253E001F07F0001280DD197
:1033A00029465079AE4A126892699047002847D161
:1033B0002068807A002843D0B24D41E001F07F01BF
:1033C00002293DD15379194601F00F0201F0700135
:1033D000A5481B0650F8220002D500F0300001E09D
:1033E00000F440509D4B1B789A4229D2002927D1E6
:1033F000002825D0A34D23E0082905D1107810F02E
:103400007F0F1DD1A04D1BE00A2919D1107800F0C3
:103410007F00012814D1907A002811D0508800280C
:103420000ED1107900280BD1D088012808D1294667
:1034300050798B4A126892699047002800D1934DC9
:103440002068290007D00021418220688561084654
:10345000A847002107E04078814909680969884741
:103460000146032805D02268108A4FF6FF73984260
:1034700003D109202168087231BD022901D000283A
:1034800002D10820107231BD1178090629D5D188E2
:103490000B460093009B0546AB4202D20098108277
:1034A00016E0884214D26E49096891F82C10024641
:1034B0000B469A4203D200207149087008E090FB45
:1034C000F1F201FB1200002802D101206C490870C2
:1034D0006348006890F82C0021688882BDE831407C
:1034E0005DE6032010724FF440506149088031BD01
:1034F00038B56148006880B2654901EB4001088831
:10350000644911EB4004534D2868017A092911D010
:1035100021780170607829684870A088FEF79CFACD
:10352000296848802089FEF797FA29688880A08951
:103530002968C8800120296808722868C088002886
:1035400002D1FFF780FE01E0FFF7EEFEBDE831405B
:1035500048E010B53F4C2068017A022901D00429C7
:1035600004D1FFF71CFE2068007A16E0062913D16B
:10357000417805290AD1017811F07F0F06D1C07872
:1035800000F04AF834480068006A80473448006810
:1035900080688047082000E0082021680872BDE8A4
:1035A00010401FE010B52B4C2068007A022801D093
:1035B000042801D1082011E0032801D0052804D1F6
:1035C000FFF79BFD2068007A08E0072805D1244812
:1035D0000068C0688047082000E008202168087261
:1035E000BDE8104080B5214890F82C100020FEF76F
:1035F000FBF918480068017A082906D14FF4805178
:103600001B4A118010211B4A1180007A092801D120
:10361000012002BD002002BD70B4104909780022CB
:10362000114C48F68F760CE01346DBB254F8235069
:1036300035401D4345F4004545F0800544F82350CE
:10364000521C8A42F0D340F080001349086070BCDD
:103650007047000048320020503200204E07002002
:103660004C3200200C330020005C00405406002047
:10367000E8320020EA320020505C00400460004044
:1036800019330020C12E0108F92D0108512E01081F
:1036900008600040006000404C5C00407047000043
:1036A000000000000000000000000000000000001A
:1036B000000070F8F87000000000000D0D00000020
:1036C000003838000038380000000000000000001A
:1036D0000020F8F820F8F82000020F0F020F0F0268
:1036E000003078CE8E18100000040C38390F060018
:1036F000183C24BCD86030000006030D1E121E0CBE
:1037000000B0F8487830000000070F0809070F09DB
:103710000000003838000000000000000000000039
:103720000000C0F0380800000000071F382000002B
:1037300000000838F0C00000000020381F0700001B
:103740000080A0E0C0E0A0800000020301030200AE
:10375000008080E0E08080000000000303000000A3
:1037600000000000000000000000002C3C1C0000D5
:103770000080808080808000000000000000000049
:1037800000000000000000000000000C0C0C000015
:1037900000000080E078180000181E0701000000FB
:1037A0000000F0F80868F8F00000070F0B080F079A
:1037B00000202030F8F80000000000000F0F00008B
:1037C0000030380888F87000000C0E0B090808005B
:1037D0000030388888F8700000060E08080F0700CF
:1037E0000000F8F800E0E00000030302020F0F02FF
:1037F00000F8F88888880800000808080C0703000B
:1038000000C0E07858C8800000070F08080F0700C4
:1038100000080888E878180000000E0F010000007A
:103820000070F8C888F8700000070F08090F07003B
:1038300000F0F80808F8F0000000090D0F0301007F
:1038400000000060606000000000000C0C0C000034
:1038500000000060606000000000002C3C1C0000C4
:103860000080C0603018080000000103060C08004A
:1038700000404040404040000001010101010100C2
:103880000008183060C0800000080C06030100002A
:1038900000303888C87830000000000D0D000000AE
:1038A000F0F80888C848F8F0070F08090B0A0B0B56
:1038B00000E0F01818F0E000000F0F01010F0F00FA
:1038C00000F8F88888F87000000F0F08080F07004C
:1038D00000F0F8080838300000070F08080E06004E
:1038E00000F8F80818F0E000000F0F080C070300BC
:1038F00000F8F88888880800000F0F0808080800FA
:1039000000F8F88888880800000F0F000000000009
:1039100000F0F8080838300000070F08090F0F0002
:1039200000F8F88080F8F800000F0F00000F0F007B
:10393000000008F8F80800000000080F0F08000059
:103940000000000000F8F80000060E08080F07004D
:1039500000F8F880E0781800000F0F00030F0C004B
:1039600000F8F80000000000000F0F080808080029
:1039700000F8F820C020F8F8000F0F0001000F0F2A
:1039800000F8F860C080F8F8000F0F0000010F0F7A
:1039900000F0F80808F8F00000070F08080F07000B
:1039A00000F8F88888F87000000F0F000000000091
:1039B00000F0F80808F8F00000070F08183F27008B
:1039C00000F8F88888F87000000F0F00010F0E0053
:1039D000003078C88818100000040C08090F060091
:1039E000000808F8F80808000000000F0F000000A9
:1039F00000F8F80000F8F80000070F08080F0700AB
:103A000000F8F80000F8F8000003070C0C070300AA
:103A100000F8F800C000F8F800010F0E010E0F01C9
:103A2000001838E0C0381800000E0F00010F0E001B
:103A30000078F88080F878000000000F0F00000088
:103A400000080888C8783800000E0F090808080028
:103A50000000F8F80808000000007F7F40400000E8
:103A6000001878E08000000000000001071E180028
:103A700000000808F8F80000000040407F7F0000C8
:103A80003018081830203018000000000000000036
:103A90000000000000000000404040404040404026
:103AA000000002060E0800000000000000000000F8
:103AB0000000202020E0C00000060F09090F0F00C1
:103AC00000F8F82020E0C000000F0F08080F0700E2
:103AD00000C0E0202060400000070F08080C040030
:103AE00000C0E02020F8F80000070F08080F0F00C2
:103AF00000C0E02020E0C00000070F090909010014
:103B00000080F0F88888880000000F0F0000000097
:103B100000C0E02020E0E00000474F48487F3F0021
:103B200000F8F82020E0C000000F0F00000F0F0089
:103B3000002020ECEC0000000008080F0F0808002F
:103B400000002020ECEC0000004040407F3F0000DF
:103B500000F8F80080E06000000F0F01030E0C0079
:103B6000000808F8F80000000008080F0F08080017
:103B700000E0E020E020E0C0000F0F0007000F0F82
:103B800000E0E02020E0C000000F0F00000F0F0059
:103B900000C0E02020E0C00000070F08080F070069
:103BA00000E0E02020E0C000007F7F08080F070051
:103BB00000C0E02020E0E00000070F08087F7F0041
:103BC00000E0E08040606000000F0F000000000097
:103BD00000C0E0202020200000080909090F06008D
:103BE0000020F8F8202020000000070F0808080037
:103BF00000E0E00000E0E00000070F08080F0F0001
:103C000000E0E00000E0E0000003070C0C07030008
:103C100000E0E000C000E0E000030F0C030C0F0325
:103C20000060E08080E06000000C0E03030E0C00DA
:103C300000E0E00000E0E00040474F68381F070068
:103C400000202020A0E06000000C0E0B09080800F6
:103C50001C14DCE02020E0C000000F1F10101C0C22
:103C600000000000FF00000000000000FF00000056
:103C70001C141CE0E02020200000001F1F01010098
:103C80000006010102020404000000000000000020
:103C900080B50020BB490968887200F093F9BA48E2
:103CA000002141604FF40441B84A118001600020B6
:103CB000B749086001BD10B50020B6498872B64802
:103CC000C079B049096848720020FDF7C3FD4FF480
:103CD00000710020FDF7C5FD20210020FDF7CEFD7D
:103CE00040210020FDF74CFEAC4C94F82C10002035
:103CF000FDF77AFE80210020FDF734FE0020FDF75D
:103D0000FFFD0020FDF7ECFD00210120FDF7A9FDDE
:103D1000C0210120FDF726FE20210120FDF7AEFD88
:103D200000210120FDF7C3FD00210220FDF799FDD0
:103D30004FF480710220FDF723FE94F82C1002202E
:103D4000FDF752FE4FF440510220FDF7B0FD002177
:103D50000220FDF793FD00210320FDF782FD4FF4C3
:103D6000A0710320FDF7FEFD20210320FDF786FD55
:103D700000210320FDF79BFD4FF4C0610420FDF7F7
:103D800070FD4FF4C0710420FDF7ECFD002104200C
:103D9000FDF78DFD20210420FDF770FD0021052099
:103DA000FDF75FFD4FF4C8710520FDF7E9FD4021E7
:103DB0000520FDF719FE4FF440510520FDF777FD72
:103DC00000210520FDF75AFD94F82C100020FDF786
:103DD0000BFE0020FDF784FD0020FFF71DFC0120F5
:103DE0006B4908606E486F49086000206E49087092
:103DF00010BD64480068807A002800D1704780B503
:103E00000520634908600120FDF79AFD0220FDF7B7
:103E100085FD00206449087001BD62480068604962
:103E2000884202D00220FDF785BF70470420584920
:103E3000086070475D480178202901D10021017098
:103E40007047704738B500214E4A13680446212C4C
:103E500007D11C7804F07F04212C0ED10FF2FD0154
:103E60000BE0202C09D11C7804F07F04212C01D117
:103E70000FF2FD0120244D4D2C701C7804F07F04BE
:103E8000212C0CD1FE280AD15888002807D1988807
:103E9000002804D1D888012801D10FF2AD01080013
:103EA00001D1022032BD99610020126850828847FA
:103EB000002032BD80B533490A68137803F07F01D2
:103EC000212918D10146FF2915D15188002912D185
:103ED000918800290FD1D18800290CD10120FDF74C
:103EE0002FFD0220FDF71AFD2D482E490860002005
:103EF0002D49087002BD03F07F03212B06D1014636
:103F0000022901D0222801D1002002BD022002BDD9
:103F1000002901D002207047002801D002207047FC
:103F2000002070472249FFF7DAB82249FFF7D7B8D7
:103F300014490968C978062901DB002070471E4A28
:103F400002EBC101FFF7CBB8002805D101200D49D4
:103F5000096808820020704718487047002805D17A
:103F600008200849096808820020704714487047F3
:103F7000002805D1082003490968088200207047FD
:103F80000F48704748320020405C00400E3300204C
:103F9000F03200202C320020984D010854060020F9
:103FA0005553424300320020203200201B330020B2
:103FB000A8060020B0060020B8060020EC32002041
:103FC0004C0600200648012101600021016041608B
:103FD0004FF4E051034A1180016000207047000057
:103FE000405C00400E330020560E4B0E410E360E44
:103FF0002B0E1F0E140E080EFD0DF00DE40DD80D46
:10400000CB0DBE0DB10DA40D960D890D7B0D6D0D63
:104010005E0D500D410D320D230D140D040DF50CE8
:10402000E50CD50CC40CB40CA30C920C810C700CD8
:104030005F0C4D0C3B0C290C170C040CF20BDF0B26
:10404000CD0BB90BA60B930B800B6C0B580B440BD1
:10405000300B1C0B080BF30ADF0ACA0AB60AA10AC6
:104060008C0A770A620A4C0A370A220A0C0AF709F4
:10407000E109CC09B609A0098B0975095F0949094D
:1040800033091D090809F208DC08C608B0089A08B7
:1040900085086F08590843082E0818080308ED071B
:1040A000D807C207AD07980783076E07580744076C
:1040B0002F071A070507F106DD06C806B406A00695
:1040C0008C067806650651063E062B061706040682
:1040D000F205DF05CC05BA05A8059605830572052E
:1040E00060054F053D052C051B050A05F904E9048B
:1040F000D804C804B804A8049804890479046A049C
:104100005B044C043D042F04200412040404F60351
:10411000E803DB03CD03C003B303A60399038C03B9
:104120008003740367035B034F03440338032D03C9
:10413000210316030B030003F502EB02E002D60293
:10414000CC02C202B802AE02A5029B029202890210
:10415000800277026E0265025C0254024B02430247
:104160003B0233022B0223021C0214020D02050241
:10417000FE01F701F001E901E201DB01D501CE0109
:10418000C801C101BB01B501AF01A901A3019D0196
:10419000970192018C01870181017C0177017101F6
:1041A0006C01670162015D01590154014F014B012E
:1041B000460142013D013901350131012C0128013F
:1041C000240120011C011901150111010D010A0131
:1041D00006010301FF00FC00F800F500F200EF000B
:1041E000EB00E800E500E200DF00DC00D900D700CA
:1041F000D400D100CE00CC00C900C600C400C1006C
:10420000BF00BC00BA00B700B500B300B000AE00FC
:10421000AC00AA00A800A600A300A1009F009D007A
:104220009B009900970096009400920090008E00E9
:104230008C008B008900870086008400820081004A
:104240007F007E007C007B0079007800760075009E
:104250007300720071006F006E006D006B006A00E9
:1042600069006800660065000901020002D44F4839
:10427000815470474E4802F00F02104400F8041CAD
:10428000704710B5401EB0F1807F01D3012010BDF2
:10429000484C60600F214FF0FF30FFF7E5FF002032
:1042A000A06007202060002010BD80B501210846D5
:1042B000F5F7C4F901214048BDE80440FDF7ACBD65
:1042C00030B4002302E0401C491C5B1C934206D220
:1042D00004780D78AC42F6D0002030BC7047012045
:1042E000FBE7000080B586B0002003AA04E0334954
:1042F000091809781154401C0C28F8DB0020694685
:1043000003E0121812780A54401C2D4A0C28F8DBDE
:10431000009850400090486850404860886842408B
:104320008A600C2203A96846FFF7CAFF00280BD158
:104330000020F5F7BCFE00235AA219460C20F4F722
:10434000A2F8F6F7E2F8FEE707B000BD38B504467C
:104350000D4645F25550F5F7A3FA2046F5F7A3FAB6
:104360002846F5F7A3FAF5F7A4FABDE83140F5F7CA
:10437000A5BAF5F79EBA3EB504460D4601214FF4A5
:104380000060F5F75BF9ADF80450ADF8004000208F
:10439000ADF80600ADF802000A4C69462046F5F774
:1043A00097F901212046F5F71CFA37BD00E400E03B
:1043B00018ED00E010E000E000023000E8F7FF1F19
:1043C000F27F0008002C014080B5FBF77FFB4FF423
:1043D0000040FBF7C1FB4BF68030FFF752FFFFF7C1
:1043E00064FF0020FBF77CFA4FF49670FBF757FB55
:1043F0000120FBF775FAFBF70EFBF5F76BFAF8F700
:10440000DFFEF7F79CFFF9F7BCFBF9F78DFB4CF2E9
:104410004F312F20FFF7AFFFFDF701FFF4F7A7FEA5
:10442000FBF750F9F3F730FFF9F716FFFCF7B3FF8E
:10443000FBF77CFCFBF776FAFBF7DAFAFBF7C0FA3E
:10444000FBF7A7FAFBF7A8FB002140F2DF10FAF711
:1044500005FF2F2140F2E730F4F7C9FC2F21092096
:10446000F4F7FCFC4FF49670FBF719FBFFF73AFFEB
:10447000F7F76CFFF4F770FBF8F7B6FA40F271212A
:104480000420FFF763FFF9F7CAFF012803D1F4F70F
:1044900018FDFAF789FBFFF76CFFFAF760FCF8F7F5
:1044A00005FEF0E744656D6F204D6F646500000008
:1044B0000000000000000000002F000000000700C6
:1044C000070000147F147F1400242A7F2A12006240
:1044D00064081323003649552250000005030000EC
:1044E00000001C224100000041221C000014083E74
:1044F00008140008083E0808000000A0600000083A
:10450000080808080000606000000020100804028D
:10451000003E5149453E0000427F4000004261514B
:104520004946002141454B31001814127F100027E5
:1045300045454539003C4A494930000171090503A8
:1045400000364949493600064949291E00003636D9
:10455000000000005636000000081422410000143C
:104560001414141400004122140800020151090619
:1045700000324959513E007C1211127C007F49499A
:104580004936003E41414122007F4141221C007FCB
:1045900049494941007F09090901003E4149497AD9
:1045A000007F0808087F0000417F41000020404153
:1045B0003F01007F08142241007F40404040007FBF
:1045C000020C027F007F0408107F003E4141413E03
:1045D000007F09090906003E4151215E007F09194B
:1045E00029460046494949310001017F0101003F48
:1045F0004040403F001F2040201F003F4038403FC8
:10460000006314081463000708700807006151492B
:10461000454300007F41410000552A552A550000BE
:1046200041417F000004020102040040404040403C
:10463000000001020400002054545478007F4844D4
:10464000443800384444442000384444487F00380B
:104650005454541800087E0901020018A4A4A47C34
:10466000007F080404780000447D400000408084FE
:104670007D00007F102844000000417F4000007C46
:1046800004180478007C0804047800384444443852
:1046900000FC242424180018242418FC007C08049E
:1046A000040800485454542000043F444020003C77
:1046B0004040207C001C2040201C003C4030403CFE
:1046C000004428102844001CA0A0A07C004464548E
:1046D0004C44141414141414EB3C904D53444F5395
:1046E000352E3000020108000200025000F80C00D4
:1046F000010001000000000000000000000029A2ED
:1047000098E46C4E4F204E414D45202020204641DC
:1047100054313220202033C98ED1BCF07B8ED9B8E1
:1047200000208EC0FCBD007C384E247D248BC199B6
:10473000E83C01721C83EB3A66A11C7C26663B07B1
:10474000268A57FC750680CA0288560280C31073F9
:10475000EB33C98A461098F7661603461C13561E9B
:1047600003460E13D18B7611608946FC8956FEB83C
:104770002000F7E68B5E0B03C348F7F30146FC11FC
:104780004EFE61BF0000E8E600723926382D74172E
:1047900060B10BBEA17DF3A66174324E740983C76C
:1047A000203BFB72E6EBDCA0FB7DB47D8BF0AC988C
:1047B00040740C487413B40EBB0700CD10EBEFA08F
:1047C000FD7DEBE6A0FC7DEBE1CD16CD19268B55EA
:1047D0001A52B001BB0000E83B0072E85B8A562425
:1047E000BE0B7C8BFCC746F03D7DC746F4297D8C13
:1047F000D9894EF2894EF6C606967DCBEA030000B3
:10480000200FB6C8668B46F86603461C668BD066DA
:10481000C1EA10EB5E0FB6C84A4A8A460D32E4F789
:10482000E20346FC1356FEEB4A525006536A016AF5
:1048300010918B4618969233D2F7F691F7F642878D
:10484000CAF7761A8AF28AE8C0CC020ACCB801020A
:10485000807E020E7504B4428BF48A5624CD136117
:1048600061720B40750142035E0B497506F8C34146
:10487000BB000060666A00EBB04E544C44522020EE
:10488000202020200D0A52656D6F766520646973C3
:104890006B73206F72206F74686572206D65646938
:1048A000612EFF0D0A4469736B206572726F72FF8F
:1048B0000D0A507265737320616E79206B657920E3
:1048C000746F20726573746172740D0A00000000C9
:1048D000000000ACCBD855AAF8B50020ADF8000018
:1048E000604D4BF6BF7648F2800729E055F820105E
:1048F000ADF80010BDF8001009040DD555F82010D2
:1049000040F68F72114045F820105748217800EB8F
:10491000810050F8040C8047BDF8000000060FD558
:10492000207855F8201089B248F60F72114045F8EA
:1049300020104E48217800EB810050F8040C80478D
:10494000686C4B490880000440F18B80088810F0A7
:104950000F00484C2070C9D1474C2868208020881F
:1049600000F030006080208800F4405020802868EB
:1049700080B2304080F4005080F02000384328603E
:104980000888C0062BD52868ADF80000BDF80000E7
:10499000000546D4BDF800000004D1D5296840F6D2
:1049A0008F7001402960FEF7FDFD286880B2064047
:1049B0002088C00401D586F480562088800401D563
:1049C00086F400566088C00601D586F0100660881F
:1049D000800601D586F020063E432E60F1BD296891
:1049E00089B248F60F7001402960FEF7B2FD2868D1
:1049F00080B206402088C00401D586F48056208805
:104A0000800401D586F400566088C00601D586F082
:104A100010066088800601D586F020063E432E6091
:104A2000F1BD296840F68F7001402960FEF760FDF6
:104A3000286880B206402088C00401D586F48056DC
:104A40002088800401D586F400566088C00601D510
:104A500086F010066088800601D586F020063E4369
:104A60002E60F1BD005C00403006002014060020DE
:104A7000103300201A330020E832002080B5394975
:104A8000086840F0010008604A68374802404A6000
:104A90000A68364802400A60086820F480200860EE
:104AA000486820F4FE0048604FF41F00886000F062
:104AB00005F84FF000602E49086001BD00BF82B0CC
:104AC0000020009001902749086840F48030086079
:104AD000086800F4003001900098401C0090019894
:104AE000002803D10098B0F5A06FF1D10868400C00
:104AF00000F0010001900198012830D11D480268A2
:104B000042F010020260026892089200026002689D
:104B100042F002020260486848604868486048689D
:104B200040F480604860486820F47C104860486821
:104B300040F4E8104860086840F080700860086839
:104B40008001FCD54868800880004860486840F0D3
:104B500002004860486800F00C000828FAD102B052
:104B600070470000001002400000FFF8FFFFF6FE53
:104B700008ED00E0002002407047000080B50020F2
:104B8000F5F795FA5FF0000322A204211420F3F751
:104B90005CFCF5F7BAFCFEE7FEE7FEE7FEE77047D0
:104BA00070477047FAF7E4BF80B52020FDF7BDFCE1
:104BB000002806D02020FDF7C4FCBDE80140FAF72C
:104BC000EDBB01BD80B501214FF08040F4F744FEFC
:104BD000012808D101214FF08040F4F749FEBDE8DB
:104BE0000140F4F775B901BD10B5084C012120460C
:104BF000F4F732FE012807D101212046F4F738FEF0
:104C0000BDE81040F4F769B910BD0000000800408D
:104C100000F006B848617264204661756C7400004B
:104C200070B5144C144D28682080144E21883088AB
:104C30000140480505D51248406880474FF6FF30CF
:104C40002860218830880140080403D5BDE8704001
:104C5000FFF742BE70BDFCF705BFFCF72EBF7047E3
:104C600080B50849052000F00FF80520BDE8024096
:104C7000FCF736BE10330020445C00400E330020A9
:104C8000540600208C31002070B504460D4604F017
:104C90007F042046FCF7C8FE06462046FCF78BFE44
:104CA000014632462846FCF7C5FD304670BDF0B4DB
:104CB0000246106895681318506803EB5004C0074B
:104CC0001CD54D441AE013F8017B05F8017B491E01
:104CD000F9D198B113F8011BC6F38106032E08BF62
:104CE00013F8016B01EB06214942801C294405D0D1
:104CF00011F8016B05F8016B401EF9D1A3420ED0EB
:104D000013F8016B16F0030104BF13F8011BC91C53
:104D100030090F28DBD113F8010B0F30D7E7F0BCB7
:104D200002F10C00704700004253333000000000D5
:104D3000000064005A006E00414C33300000000057
:104D40000000000000000F0042533430000000005B
:104D50000000330029003D00414C343000000000C9
:104D6000000078006E0082004750333000000000E1
:104D7000000096008C00A000434D5233000000005C
:104D80000000B400AA00BE0041534C3300000000F4
:104D90000000C800BE00D20009026200030100C08A
:104DA0003209040000020806500407058102400091
:104DB0000007050202400000080B01020202010187
:104DC000090401000102020100052400100105246C
:104DD00001000104240202052406000107058403E2
:104DE0000800FF09040200020A000000070505028E
:104DF00040000007058302400000000000000000A2
:104E00000080C06030180C000000000000000000AE
:104E1000000103060C183000000000000000000034
:104E2000000C183060C0800000000000000000008E
:104E30000030180C06030100000000000000000014
:104E4000C0F0FC0EFCF0C0000000000060707C7F31
:104E50007F7F7F487F7F7F7F7C70600010188CC6CB
:104E60006363C68C1810426331180C0C183163420E
:104E700042C68C183030188CC64208183163C6C63A
:104E8000633118086363C6C66363C6C663630006FE
:104E900006FEFE060600003060C080003060C08064
:104EA000003060C0800000180C060301180C0603D7
:104EB00001180C06030100002603530054004D00A6
:104EC0006900630072006F0065006C00650063009C
:104ED000740072006F006E006900630073000000D0
:104EE0002603530054004D003300320020004D00D3
:104EF0006100730073002000530074006F007200A3
:104F0000610067006500000010B507497944183159
:104F1000064C7C44163404E00A68081D1144884796
:104F20000146A142F8D110BD500000006C00000005
:104F300020202020202328303A43656E7469677250
:104F400061646520313A46616872656E68656974AE
:104F5000290D0A0000800202200000004D696E69E0
:104F60002044534F4469736B2020202020202020B0
:104F70002020202020202020AF31FFFFC82B000060
:104F8000540700200000000027FDFFFFC8020000BA
:104F9000A60200004002002000F00DF8002801D019
:104FA000FFF7B2FFAFF300800020AFF30080FFF700
:104FB0000BFA00F002F80120704700F001B8000081
:104FC00007463846FDF70EFFFBE700002023284385
:104FD0003A3130307E33353020463A3231327E3607
:104FE0003632290D0A00000020202020232852619B
:104FF0006E67653A204F46462C357E313230290D9A
:105000000A00000020202020202328303A566F6C10
:10501000742020313A506F776572290D0A00000024
:1050200020202020202020232852616E67653A200E
:1050300020307E202035290D0A000000202020206D
:10504000232852616E67653A2020317E2031302955
:105050000D0A00002020202328303A4F4646202009
:10506000313A4F4E290D0A0012010002EF020140B1
:10507000160401DC00020102030100005072736596
:105080007454656D70313D3232300000507273657A
:105090007454656D70323D32353000005072736566
:1050A0007454656D70333D33303000004C6F77437E
:1050B000757272656E743D31000000003C8B54EADD
:1050C0006C5A3745D78AEC5F3858CAE5183C66C336
:1050D0008100000000000081C3663C1810035300EB
:1050E000540020004D0061007300730001488047A8
:1050F000014800477D4A01089951010850727365C3
:105100007454656D70310000507273657454656D30
:1051100070320000507273657454656D7033000016
:10512000536C65657054696D650000004261636B86
:105130006C6967687400000053686F775479706514
:10514000000000004C6F7743757272656E7400004A
:1051500054656D705479706500000000536C65658E
:105160007054696D653D30004261636B6C696768BE
:10517000743D360053686F77547970653D30000098
:10518000566F6C756D653D330000000054656D70A1
:10519000547970653D300000AFF30080AFF30080BC
:1051A000FFF7FAFE566F6C756D650000686A6C74E7
:1051B0007A4C000004030904FFF7FEBFFFF7FEBFAF
:1051C000FFF7FEBFFFF7FEBFFFF7FEBFFFF7FEBF13
:1051D000FFF7FEBFFFF7FEBFFFF7FEBFFFF7FEBF03
:1051E000FFF7FEBFFFF7FEBFFFF7FEBFFFF7FEBFF3
:1051F000FFF7FEBFFFF7FEBFFFF7FEBFFFF7FEBFE3
:10520000FFF7FEBFFFF7FEBFFFF7FEBFFFF7FEBFD2
:10521000FFF7FEBFFFF7FEBFFFF7FEBFFFF7FEBFC2
:10522000FFF7FEBFFFF7FEBFFFF7FEBFFFF7FEBFB2
:10523000FFF7FEBFFFF7FEBFFFF7FEBFFFF7FEBFA2
:10524000FFF7FEBFFFF7FEBFFFF7FEBFFFF7FEBF92
:10525000FFF7FEBFF20200016002CC4F010804120A
:10526000E80410033C500108040412200412540402
:105270001230141003542F002074041003542D0016
:10528000207C14128C04129C0410035C51010868E9
:105290000412740412800422AC1C1108F2FF0001F5
:1052A000F1F2011AFC1C1A081C1214041220041238
:1052B0002C0412380412A404124404125004F802FC
:1052C0004B010000023C52FF01F10464920116916F
:1052D0000CF1022E711E611C61115A98FA12060718
:1052E0002002C409B80B1A92033FF21D03DD716856
:1052F00010051A034D0069006E04900577006100E7
:10530000720065485007574C01089D3601085F0838
:10531000E104925B1892610C2300C25F1005080043
:10532000913C0108B7041003353E010843041245BF
:105330000412B5041003113F01082504122B044F79
:10534000313FD403124005213CC3F33D64831B3E2F
:105350000C122D0C1668EC12122C1003984D01083B
:10536000620816B4DC1204081003B84E01082608BF
:1053700052E0081003F80500201A0812DC3057101C
:1053800000204206DD427007D60A3331882925F015
:105390000207AA8A00080465E8F2007E148700006C
:0753A000570002060101FFA6
:040000050801519904
:00000001FF
